:100000000C94671B0C94981B0C94981B0C94981BD5
:100010000C94981B0C94981B0C94981B0C94981B94
:100020000C94981B0C94981B0C94981B0C94981B84
:100030000C94981B0C94981B0C94981B0C94981B74
:100040000C94981B0C94A99C0C94981B0C94981BD2
:100050000C94981B0C94981B0C9447890C94E7748F
:100060000C94981B0D94771F0D946D1F0C94981B86
:100070000C94981B0C94981B0C94981B0C94981B34
:100080000C94E4F50C94981B0C94981B0C94981BFE
:100090000C94981B0C94981B0C94981B0C94981B14
:1000A0000C94981B0C94981B0C94B6F50C94981B0C
:1000B0000C94981B0C94981B0C94981B0C94981BF4
:1000C0000C94981B0C94981B0C94981B0C9499F608
:1000D0000C9463F60C94981B0C94981B0C94981B2E
:1000E0000C94981B084AD73B3BCE016E84BCBFFDE5
:1000F000C12F3D6C74319ABD56833DDA3D00C77FF8
:1001000011BED9E4BB4C3E916BAAAABE0000008090
:100110003F05A84CCDB2D44EB93836A9020C50B91F
:10012000918688083CA6AAAA2ABE000000803F004B
:100130000C943D730C942FF70C943BC70C948BDFFD
:100140000C9442C80C94C9C70D941D200C9410C87F
:100150000D9411200C9421D60C944FD70D940920A6
:100160000C94BD720C949ADA0C94DA6F0C9437F7F5
:100170000C94F7C70D9415200C9424C80C94287285
:100180000C9406F70C94576F0D94E41F0C944AF7E7
:100190000C94DE720C9491D50C94D5DA0C9430C783
:1001A0000D94B51F0C9466D80C9443CE0C9414CFC8
:1001B0000C944A450C9445720C9424F70C944BC74C
:1001C0000C9445C70C9467C70C9422730C94D3C746
:1001D0000D940D200C94DBC70C946BC70C9438C89D
:1001E0000C9434C70C94A3DA0C94A0DA0D94A426D2
:1001F0000C9452430C94D96F0C94E8D60C94B5C768
:100200000C942EC80C94E9DA0C943BF70C94D7DBD1
:100210000C94BCDA0C9433F70C9453C70C9411D79C
:100220000C94BFC70C94CBDA0C94A3D70C9455F75D
:100230000C94FA730C94ABDC0D943B200C942BF7CC
:100240000C945DF70D9433200C942CD30C9415F77B
:100250000C94F5D40C94B0C70C941E450C9443F741
:100260000C94ABCA0C941AC80D94F31F0C94BB7376
:100270000C94E3C70C94CD730C941AC70C94C5D698
:100280000C9457D60C9459C70C942CC70C94034368
:100290000D9421200C9461D70C9415C70C944FC772
:1002A0000C94C1D40C9401C80D9428200C9430D720
:1002B0000C94B1CC0C94D7F60C94DBCC0C9472D487
:1002C0000C94C3450C9492D00C94A5D40C9473DA7E
:1002D0000D9486260D9419200C945DC70C94E8DBD0
:1002E0000C9438C70C94B6D70C948B450C94C474FA
:1002F0000C94EDC70C943FF70C9441C70C94F6DABC
:100300000C94CCCB0D9402200C9456430C9461C7F2
:100310000C94A8C74E414E494E495459494E46CDBA
:10032000CCCC3D0AD7233C17B7D13877CC2B3295AC
:1003300095E6241FB14F0A000020410000C842008A
:10034000401C4620BCBE4CCA1B0E5AAEC59D740054
:10035000407A10F35A00A0724E18090010A5D4E894
:100360000000E87648170000E40B54020000CA9A27
:100370003B000000E1F50500008096980000004079
:10038000420F000000A086010000001027000000BE
:1003900000E803000000006400000000000A000004
:1003A0000000000100000000002C76D888DC674FB8
:1003B0000823DFC1DFAE59E1B1B796E5E3E453C6E8
:1003C0003AE651997696E8E6C28426EB898C9B62E0
:1003D000ED407C6FFCEFBC9C9F40F2BAA56FA5F48A
:1003E00090055A2AF75C936B6CF9676DC11BFCE0B2
:1003F000E40D47FEF520E6B500D0ED902E03009405
:100400003577050080841E080000204E0A00000099
:10041000C80C333333330F986E12831141EF8D21A3
:1004200014893BE65516CFFEE6DB18D1844B381B0A
:10043000F77C1D901DA4BBE424203284725E2281CF
:1004400000C9F124ECA1E53D27434F4D4D554E49E0
:10045000434154494F4E0044525952554E00455263
:10046000524F525300494E464F004543484F004FAC
:100470004646004F4E0020204D61783A2000200073
:1004800020204D696E3A2000536F667420656E64BB
:1004900073746F70733A20003D3D4F6E506F7765F7
:1004A000724C6F7373526573756D653D3D004D32CF
:1004B000342053256C642054256C64004739322E57
:1004C00039204525730047312046256400473932DD
:1004D0002E39205A2573004731205A3020463230B9
:1004E000300047312058257320592573204633307A
:1004F0003030004D34323020532569205A257300A6
:100500004D3130362050256920532569004D323059
:10051000302044257300473238523058590047394B
:10052000322E39204530205A300A47315A2573007F
:100530004D31303920532569004D31393020532554
:1005400069004D343230205330205A300020496E3B
:1005500076616C69642065787472756465722000D8
:1005600047322F47332062616420706172616D658C
:10057000746572730A00536C6565702E2E2E005AD6
:100580002050726F62652050617374204265640A66
:10059000005A2050726F626520506173742042656A
:1005A00064004732384C30004D3131372050726F83
:1005B0006265206661696C65642E0A4732380A00FC
:1005C00070726F62655F7265776970650047323976
:1005D000205265747279696E670050726F62696E3D
:1005E00067204661696C6564004D31313720426592
:1005F00064206C6576656C696E67206661696C6500
:10060000642E0A4730205A31300A4D3330302050A2
:10061000323520533838300A4D33303020503530A1
:100620002053300A4D333030205032352053383883
:10063000300A4D333030205035302053300A4D339E
:1006400030302050323520533838300A4D33303076
:10065000205035302053300A473420533100707217
:100660006F62655F6661696C6564004D313137208A
:10067000426564206C6576656C696E6720646F6E98
:10068000652E00205A3A200020593A200042656425
:1006900020583A20004D65736820706F696E742091
:1006A0006F7574206F662072616E67650A004D3049
:1006B0002053746F70004D312053746F7000436F7E
:1006C0006E74696E756500436C69636B20746F208E
:1006D000526573756D652E2E2E004E6F204D6F7610
:1006E000652E00456E642066696C65206C697374C4
:1006F0000A00426567696E2066696C65206C6973E3
:10070000740A004E6F206D656469610A005265735A
:10071000756D696E6720534400286E6F2066696CA2
:1007200065290043757272656E742066696C653A5E
:1007300020005072696E742074696D653A20000A59
:1007400053746174733A2046696C616D656E7420F0
:10075000757365643A20002C204C6F6E6765737466
:10076000206A6F623A2000546F74616C2074696D66
:10077000653A200053746174733A20002C2046615E
:10078000696C65643A20002C2046696E697368655F
:10079000643A20005072696E74733A200053746199
:1007A00074733A2000436F6F6C696E672E2E2E00B3
:1007B00048656174696E672E2E2E00452025530012
:1007C0006F6B006F6666006A0465045E0457044937
:1007D0000444454255473A004D31313320530042DD
:1007E000656420436F6F6C696E672E2E2E00426524
:1007F000642048656174696E672E2E2E00544D3357
:100800004420453520506C7573204F46462E002FEE
:100810002F00205200416363656C65726174696FDB
:100820006E3A2050004D32303620580046523A0081
:1008300020466C6F773A20003A200020536572768C
:100840006F2000206F7574206F662072616E67657F
:100850000A00536572766F200020643A0020693ADE
:100860000020703A00496E76616C69642065787486
:1008700072756465720A0020643A0020693A0020AB
:10088000703A0064697300656E0043290A00616272
:100890006C656420286D696E2074656D702000435E
:1008A0006F6C64206578747275646573206172651D
:1008B0002000504944204175746F74756E65005076
:1008C0004944204175746F74756E65206661696C6A
:1008D00065642120426164206865617465722069E5
:1008E000640A0046696C616D656E742072756E6F86
:1008F00075742064697374616E636520286D6D2959
:100900003A200046696C616D656E742072756E6F79
:10091000757420004D34323120696E636F727265D8
:10092000637420706172616D6574657220757361A6
:1009300067650A004D65736820706F696E74206F7B
:100940007574206F662072616E67650A004F666677
:1009500073657473204170706C69656400457272D0
:100960003A20546F6F206661722100546F6F2066C9
:1009700061722066726F6D207265666572656E6366
:100980006520706F696E740A00454550524F4D20C6
:100990004F4B0A00506F7765722D6C6F7373207226
:1009A00065636F7665727920004D383400446F6E50
:1009B00065207072696E74696E672066696C650A7D
:1009C000004D3737004D3331004361703A004D45DB
:1009D00041545041434B00434F4F4C45525F5445A7
:1009E0004D5045524154555245004348414D4245B2
:1009F000525F54454D504552415455524500424175
:100A000042595354455050494E47004152435300B8
:100A10004D4F54494F4E5F4D4F4445530054484548
:100A2000524D414C5F50524F54454354494F4E0034
:100A30004C4F4E475F46494C454E414D4500415550
:100A4000544F5245504F52545F53445F5354415496
:100A500055530053445F5752495445005245504541
:100A60004154005344434152440050524F4D50545E
:100A70005F535550504F525400454D455247454ED7
:100A800043595F50415253455200434153455F4CD7
:100A9000494748545F4252494748544E45535300D2
:100AA000544F47474C455F4C494748545300534FB8
:100AB0004654574152455F504F57455200425549A1
:100AC0004C445F50455243454E54004C4556454CAE
:100AD000494E475F44415441005A5F50524F42458E
:100AE0000052554E4F5554004155544F4C455645B4
:100AF0004C005052494E545F4A4F420050524F47AB
:100B000052455353004155544F5245504F52545F34
:100B100054454D5000564F4C554D45545249430095
:100B2000454550524F4D0042494E4152595F46494A
:100B30004C455F5452414E5346455200534552492D
:100B4000414C5F584F4E5F584F4646004649524D04
:100B5000574152455F4E414D453A4D61726C696E49
:100B600020322E302E375F4457372E3320544D33EA
:100B70004420453550534D44424220284170722054
:100B8000323420323032312031393A35343A32364B
:100B90002920534F555243455F434F44455F5552BB
:100BA0004C3A68747470733A2F2F67697468756271
:100BB0002E636F6D2F496E73616E69747941757420
:100BC0006F6D6174696F6E2F4D61726C696E2F74F9
:100BD0007265652F437265616C6974794477696EDB
:100BE0005F322E302050524F544F434F4C5F56458A
:100BF0005253494F4E3A312E30204D414348494ED1
:100C0000455F545950453A544D33442045352050A2
:100C10006C75732045585452554445525F434F55A7
:100C20004E543A3120555549443A63656465326102
:100C300032662D343161322D343734382D396231FA
:100C4000322D6335356336326633363766660A00D1
:100C500050726F6265204F6666736574205A00504B
:100C6000726F6265204F6666736574205A00290AA8
:100C70000020746F20003F5A206F7574206F66202B
:100C800072616E6765202800290A0020746F2000B9
:100C90003F59206F7574206F662072616E67652002
:100CA000282D00290A0020746F20003F58206F75FE
:100CB00074206F662072616E676520282D00507267
:100CC0006F6265204F666673657420580043616EDD
:100CD0006E6F74206F70656E207375626469722028
:100CE000002569730025696D2025697300256968F1
:100CF0002025696D202569730025696420256968B0
:100D00002025696D2025697300256979202569648E
:100D1000202569682025696D20256973003D3D44C3
:100D200077696E20496E697420436F6D706C6574CD
:100D3000653D3D002A2A2A4E6F7A7A6C6554656DAE
:100D4000705374617475735B325D203D003D3D48A6
:100D5000656174696E6720446F6E65204368616EDB
:100D600067652046696C616D656E743D3D002020AD
:100D7000737461727470726F677265737320003D73
:100D80003D7761697477617920353D3D003D3D7760
:100D900061697477617920343D3D003D3D7761693B
:100DA0007477617920333D3D003D3D77616974770B
:100DB000617920313D3D003D3D6F6E5072696E742A
:100DC00054696D657253746F707065643D3D003D8C
:100DD0003D6F6E466163746F727952657365743DE1
:100DE0003D00270A0A0000272027002027002D00A9
:100DF0006E6F74696669636174696F6E2000636108
:100E00006E63656C005072696E742041626F72741B
:100E10006564004469736D697373005549204162CC
:100E20006F7274656400726573756D65004D323460
:100E3000002A2A2A43506C617920546F6E652A2A51
:100E40002A003D3D6F6E5072696E7454696D657213
:100E50005061757365643D3D00486F6D696E672034
:100E60004661696C6564006F70656E005452494755
:100E70004745524544003A200066696C616D656ED5
:100E800074007A5F6D696E00795F6D617800785FDC
:100E90006D6178005265706F7274696E6720656E5F
:100EA0006473746F70207374617475730A002074B6
:100EB0006F6F206C6F6E6720657874727573696FE1
:100EC0006E2070726576656E7465640A0020636FCB
:100ED0006C6420657874727573696F6E20707265CA
:100EE00076656E7465640A00486F6D65202573250C
:100EF000732573204669727374005761726E696E50
:100F0000673A20486F6D696E672042756D702044A6
:100F1000697669736F72203C20310A000202040076
:100F200000B0430000B443000000000000B04300E4
:100F300000B4430000C8430000004100000041002D
:100F40000000400101FF000000010000000100005E
:100F50008000555555000000400033333300AAAAE5
:100F60002A004992240000002000C7711C009999B2
:100F70001900D1451700555515003BB11300244900
:100F8000120011111100000010000F0F0F00E338C4
:100F90000E0043790D00CCCC0C00C3300C00E8A24D
:100FA0000B0064210B00AAAA0A00703D0A009DD81C
:100FB0000900427B090092240900DCD308008888DC
:100FC00008001042080000000800F0C107008787F1
:100FD000070075500700711C07003EEB0600A1BC1E
:100FE00006006990060066660600703E06006118FD
:100FF000060017F4050074D105005BB00500B2903F
:101000000500627205005555050078390500B81EC7
:101010000500050505004EEC040087D40400A1BDC1
:10102000040090A7040049920400C17D0400EE6909
:101030000400C7560400444404005C320400082144
:10104000040041100400000004003FF00300F8E039
:10105000030026D20300C3C30300CCB503003AA8A3
:1010600003000A9B0300388E0300C08103009F75B4
:101070000300D0690300505E03001D530300344891
:101080000300913D03003333030016290300381F8A
:10109000030097150300300C0300030303000BFA51
:1010A000020049F10200BAE802005CE002002DD81B
:1010B00002002DD0020059C80200B0C0020031B9B0
:1010C0000200DAB10200AAAA0200A0A30200BC9C9E
:1010D0000200FA9502005C8F0200DF880200828223
:1010E0000200457C02002776020027700200436A56
:1010F00002007C640200D05E02003F590200C85327
:101100000200FFFDFCFAF8F6F4F2F0EEECEAE9E793
:10111000E5E3E1E0DEDCDAD9D7D5D4D2D0CFCDCB50
:10112000CAC8C7C5C3C2C0BFBDBCBAB9B7B6B4B3DD
:10113000B2B0AFADACAAA9A8A6A5A4A2A1A09E9D3D
:101140009C9A99989795949392908F8E8D8B8A897B
:1011500088878684838281807F7E7D7B7A79787799
:10116000767574737271706F6E6D6C6B6A69686797
:10117000666564636261605F5E5D5C5B5A59585886
:101180005756555453525150504F4E4D4C4B4A4A5E
:101190004948474646454443424241403F3E3E3D22
:1011A0003C3B3B3A393838373635353433323231D7
:1011B00030302F2E2E2D2C2B2B2A2929282727267D
:1011C000252524232322212120201F1E1E1D1C1C17
:1011D0001B1B1A19191818171616151514131312A4
:1011E000121111100F0F0E0E0D0D0C0C0B0A0A0927
:1011F000090808070706060505040403030202019F
:1012000000003D3D6F6E5072696E7454696D657279
:10121000537461727465643D3D000000B04300008A
:10122000B4430000C84300000000000000000000BC
:1012300000003D3D6F6E53746F7265536574746941
:101240006E67733D3D003D3D6F6E436F6E6669672F
:1012500075726174696F6E53746F726557726974D9
:1012600074656E3D3D0053657474696E67732053F9
:10127000746F726564000A20696E6974207A7072F6
:101280006F62655F7A6F6666736574203D20003D0E
:101290003D6F6E436F6E66696775726174696F6EDC
:1012A00053746F7265526561643D3D00454550520F
:1012B0004F4D20496E697469616C697A65640A00F2
:1012C0003B20003A0A0020204D36303320002044D5
:1012D0000020204D34313220530046696C616D6529
:1012E0006E742072756E6F75742073656E736F7295
:1012F0003A002055004C0046696C616D656E7420A3
:101300006C6F61642F756E6C6F6164206C656E67C5
:101310007468733A0020204D3835312058005A2D1A
:1013200050726F6265204F66667365740020204DB1
:10133000343133205300506F7765722D4C6F7373C7
:10134000205265636F766572793A00204400204927
:101350000020204D3330342050002044002049002C
:1013600020204D33303120500050494420736574A3
:1013700074696E67733A00204A0020204732392092
:101380005720490020204D343230205300417574DD
:101390006F20426564204C6576656C696E673A0023
:1013A00020204D323036205800486F6D65206F6622
:1013B000667365743A0020580020530020204D3297
:1013C0003035204200416476616E6365643A2042A4
:1013D0003C6D696E5F7365676D656E745F74696D92
:1013E000655F75733E20533C6D696E5F666565642D
:1013F000726174653E20543C6D696E5F74726176F3
:10140000656C5F66656564726174653E20583C6D0D
:1014100061785F785F6A65726B3E20593C6D6178D8
:101420005F795F6A65726B3E205A3C6D61785F7AC6
:101430005F6A65726B3E20453C6D61785F655F6AEF
:1014400065726B3E0020540020520020204D323047
:1014500034205000416363656C65726174696F6E1E
:101460002028756E6974732F7332293A20503C70AE
:1014700072696E745F616363656C3E20523C726595
:1014800074726163745F616363656C3E20543C7485
:10149000726176656C5F616363656C3E0020204D10
:1014A0003230312058004D6178696D756D2041638F
:1014B00063656C65726174696F6E2028756E6974FE
:1014C000732F7332293A0020204D323033205800D8
:1014D0004D6178696D756D206665656472617465CE
:1014E000732028756E6974732F73293A00537465DD
:1014F00070732070657220756E69743A0020440024
:1015000020204D3230302053002044697361626CDA
:1015100065640A0046696C616D656E74207365745C
:1015200074696E67733A0020286D6D29002020478A
:101530003231202020203B20556E69747320696E63
:10154000206D6D003D3D6F6E4C6F6164536574742A
:10155000696E67733D3D0000803B4400803B440062
:10156000002041000096420000A0420000A042007E
:101570000048440080CC43D0070000D0070000643E
:101580000000004B00000024F4D43050C38E20C271
:10159000A24017828B7011127A910D816CD90AA822
:1015A00061E108C7586607615143061E4B5D05C1DE
:1015B00045A7041A411104093D98037139310340CC
:1015C00036DB0265339102D4305402802E1D026353
:1015D0002CEE01752AC501B028A001102781018FCA
:1015E0002564012B244B01E0223401AC211F018D25
:1015F000200D01801FFC00841EED00971DDF00B848
:101600001CD200E61BC600201BBC00641AB200B24C
:1016100019A8000A19A0006A189900D11791004072
:10162000178B00B516840031167E00B31579003A89
:10163000157300C7146F0058146A00EE1366008813
:1016400013630025135E00C7125B006C1257001570
:10165000125400C111510070114F0021114B00D6DE
:101660001049008D1047004610440002104200C08F
:101670000F4000800F3E00420F3C00060F3B00CBA6
:101680000E3800930E37005C0E3500270E3400F341
:101690000D3200C10D3100900D3000600D2E003272
:1016A0000D2D00050D2C00D90C2B00AE0C2900854A
:1016B0000C29005C0C2700350C27000E0C2600E8D6
:1016C0000B2400C40B2400A00B23007D0B23005A25
:1016D0000B2100390B2100180B2000F80A1F00D93C
:1016E0000A1E00BB0A1E009D0A1D00800A1D006321
:1016F0000A1C00470A1B002C0A1B00110A1A00F7DB
:10170000091A00DD091900C4091900AB0919009272
:101710000917007B091800630917004C09160036E9
:10172000091600200916000A091500F5081500E041
:10173000081400CC081400B8081400A40814009081
:101740000813007D0812006B0813005808120046A9
:1017500008120034081100230811001208110001BA
:10176000081100F0071000E0071000D0071000C0BB
:10177000071000B0070F00A107100091070E0083AB
:10178000070F0074070F0065070E0057070E00498A
:10179000070E003B070D002E070E0020070D00135B
:1017A000070D0006070D00F9060C00ED060D00E020
:1017B000060C00D4060C00C8060C00BC060C00B0D9
:1017C000060C00A4060B0099060C008D060B008287
:1017D000060B0077060B006C060B0061060A00572B
:1017E000060B004C060A0042060A0038060A002EC4
:1017F000060A0024060A001A060A00100609000755
:10180000060A00FD050900F4050900EB050900E2E0
:10181000050900D9050900D0050900C7050900BE62
:10182000050900B5050800AD050800A50509009CDF
:10183000050800940508008C050800840508007C54
:10184000050800740508006C050700650508005DC3
:10185000050700560508004E05070047050700402C
:1018600005080038050700310507002A0507002391
:101870000507001C050600160507000F05070008F0
:1018800005060002050700FB040600F5040700EE4C
:10189000040600E8040600E2040700DB040600D5A5
:1018A000040600CF040600C9040600C3040600BDF8
:1018B000040600B7040600B1040500AC040600A647
:1018C000040600A00405009B040600950405009092
:1018D0000406008A04050085040500800406007AD9
:1018E00004050075040500700405006B040500661E
:1018F000040500610405005C04050057040500525E
:101900000405004D04050048040500430405003E9D
:101910000404003A04050035040500300404002CDA
:1019200004050027040400230405001E0404001A13
:1019300004040016040500110404000D0404000949
:101940000405000404040000040400FC030400F87F
:10195000030400F4030400F0030400EC030400E8B3
:10196000030400E4030400E0030400DC030400D8E3
:10197000030400D4030400D0030400CC030400C813
:10198000030300C503030024F404D9201BC40C5C2A
:101990000E9804C4095F0265077101F405F900FBA4
:1019A00004B30048048700C10369005803550003CD
:1019B000034500BE023A008402310053022A002986
:1019C00002250004022000E4011C00C8011900AF38
:1019D00001170098011400840113007101100061C7
:1019E00001100051010E0043010D0036010B002BC8
:1019F000010B0020010B00150109000C0109000377
:101A0000010800FB000800F3000800EB000700E4F9
:101A1000000600DE000600D8000600D2000600CC5A
:101A2000000500C7000500C2000500BD000400B9A4
:101A3000000400B5000400B1000400AD000400A9DA
:101A4000000400A5000300A20003009F0004009B07
:101A5000000300980003009500020093000300902B
:101A60000003008D0002008B000300880002008646
:101A700000020084000300810002007F0002007D5C
:101A80000002007B0002007900020077000100766E
:101A90000002007400020072000100710002006F79
:101AA0000002006D0001006C0002006A0001006984
:101AB000000200670001006600010065000100648B
:101AC0000002006200010061000100600001005F8F
:101AD0000002005D0001005C0001005B0001005A93
:101AE0000001005900010058000100570001005694
:101AF0000001005500010054000100530000005394
:101B00000001005200010051000100500001004F8F
:101B10000001004E0000004E0001004D0001004C8D
:101B20000001004B0000004B0001004A0001004989
:101B30000001004800000048000100470001004685
:101B4000000000460001004500000045000100447F
:101B50000001004300000043000100420000004279
:101B60000001004100000041000100400001003F71
:101B70000000003F0001003E0000003E0001003D6B
:101B80000000003D0001003C0000003C0000003C63
:101B90000001003B0000003B0001003A0000003A59
:101BA0000001003900000039000100380000003851
:101BB0000000003800010037000000370001003647
:101BC000000000360000003600010035000000353E
:101BD0000000003500010034000000340000003433
:101BE0000001003300000033000000330001003228
:101BF000000000320000003200010031000000311E
:101C00000000003100010030000000300000003012
:101C10000001002F0000002F0000002F0000002F07
:101C20000001002E0000002E0000002E0001002DFB
:101C30000000002D0000002D0000002D0001002CF0
:101C40000000002C0000002C0000002C0001002BE4
:101C50000000002B0000002B0000002B0001002AD8
:101C60000000002A0000002A0000002A00010029CC
:101C700000000029000000290000002900000029C0
:101C800000010028000000280000002800000028B3
:101C900000000028000100270000002700000027A6
:101CA0000000002700000027000100260000002699
:101CB000000000260000002600000026000100258C
:101CC0000000002500000025000000250000002580
:101CD0000000002500010024000000240000002472
:101CE0000000002400000024000100230000002365
:101CF0000000002300000023000000230000002358
:101D00000000002300010022000000220000002249
:101D1000000000220000002200000022000100213B
:101D2000000000210000002100000021000000212F
:101D30000000002100000021000100200000002020
:101D40000000002000000020000000200000002013
:101D500000000020000000200001001F0000001F04
:101D60000000001F0000001F0000001F0000001FF7
:101D70000000001F0001001E0000001E0000001EE9
:101D80000000001E000000393000003325000087ED
:101D9000190000B00F0000DB080000BD0400007453
:101DA0000200003F01000020436F756E7420583A16
:101DB0000023646566696E652044454641554C5470
:101DC0005F0000626564004B6420004B6920004B9B
:101DD000702000504944204175746F74756E652001
:101DE00066696E6973686564212050757420746833
:101DF00065206C617374204B702C204B6920616EE0
:101E000064204B6420636F6E7374616E747320661C
:101E1000726F6D2062656C6F7720696E746F2043FE
:101E20006F6E66696775726174696F6E2E680A00FD
:101E3000504944204175746F74756E652066616900
:101E40006C6564212074696D656F75740A00504972
:101E500044204175746F74756E65206661696C65A8
:101E600064212054656D70657261747572652074AB
:101E70006F6F20686967680A00204B643A20002071
:101E80004B693A2000204B703A200020436C61736C
:101E900073696320504944200A00204E6F206F76FA
:101EA000657273686F6F740A002054753A200020C1
:101EB0004B753A2000206D61783A2000206D696EE4
:101EC0003A200020643A200020626961733A2000C1
:101ED000504944204175746F74756E652073746148
:101EE00072740A00504944204175746F74756E65B0
:101EF000206661696C6564212054656D706572614E
:101F00007475726520746F6F20686967680A004293
:101F1000656400453100626564002C207379737438
:101F2000656D2073746F70706564212048656174FD
:101F300065725F49443A200048656174696E6720A4
:101F40004661696C65640048656174696E67206606
:101F500061696C6564004D31313220536875746479
:101F60006F776E001000C90210012C0140012201A0
:101F700070011801B0010E01F00104015002FA00D5
:101F8000B002F0003003E600D003DC009004D20081
:101F90007005C800A006BE000008B400B009AA0081
:101FA000D00BA000600E960060118C00001582001E
:101FB00020197800C01D6E00A0226400B0275A00CE
:101FC000902C500000314600E0343C0010383200C4
:101FD000903A2800603C1E00A03D1400803E0A009C
:101FE000203F0000544845524D414C2052554E412F
:101FF00057415900546865726D616C2052756E616D
:10200000776179004572723A204D415854454D50E0
:10201000004D415854454D50207472696767657290
:102020006564004572723A204D494E54454D50004A
:102030004D494E54454D502074726967676572650D
:102040006400202F002042403A0020403A002057F0
:102050003A0020573A00496E76616C6964206578D1
:102060007472756465720A007C3C3E5E2B3D3F2FA6
:102070005B5D3B2C2A225C0043616E6E6F74206FA7
:1020800070656E2073756264697220005344204944
:102090006E6974204661696C005344206361726408
:1020A000206F6B0A006F70656E526F6F74206661EF
:1020B000696C65640A00766F6C756D652E696E6972
:1020C00074206661696C65640A004E6F2053442079
:1020D000636172640A000A4D3234004D32332025A8
:1020E00073002E0A006F70656E206661696C65640E
:1020F0002C2046696C653A200046696C6520736542
:102100006C65637465640A002053697A653A20003F
:1021100046696C65206F70656E65643A2000454EB7
:102120004420535542524F5554494E450A002220EF
:10213000706F73002220706172656E743A220053D2
:102140005542524F5554494E452043414C4C207402
:1021500061726765743A220053756263616C6C202A
:102160004F766572666C6F77004578636565646568
:1021700064206D617820535542524F5554494E4565
:102180002064657074683A002E0A0044656C6574BA
:10219000696F6E206661696C65642C2046696C65A8
:1021A0003A200046696C652064656C657465643A24
:1021B000005344207072696E74696E67206279748E
:1021C0006520004E6F74205344207072696E7469EC
:1021D0006E670A0057726974696E6720746F2066B3
:1021E000696C653A2000667265736800646F696E99
:1021F00067002066696C653A20004E6F7720002FDB
:102200006175746F25632E67002020506C616E6EBF
:10221000657242756666657242797465733A20002C
:102220002046726565204D656D6F72793A200043D6
:102230006F6D70696C65643A204170722032342091
:10224000323032310A00204C617374205570646161
:102250007465643A20323032312D30342D313820DB
:102260007C20417574686F723A2054696E794D61B3
:102270006368696E657333440A00322E302E375F0F
:102280004457372E330A004D61726C696E0020533B
:102290006F6674776172652052657365740A0020F9
:1022A0005761746368646F672052657365740A00D0
:1022B0002042726F776E206F75742052657365745B
:1022C0000A002045787465726E616C2052657365F2
:1022D000740A00506F77657255700A0073746172EA
:1022E000740A004732385859004D3130303100659A
:1022F00072726F722077726974696E6720746F20D2
:1023000066696C650A00446F6E6520736176696E5C
:10231000672066696C652E0A004D323900456E648F
:1023200073746F7073002553202563202563202567
:102330006320256300205A3A0020593A0020583A79
:1023400000656E6473746F7073206869743A20005E
:1023500070012C0190012701B0012201C0011D0173
:10236000F00118011002130130020E016002090190
:1023700090020401C002FF000003FA004003F500D0
:102380008003F000D003EB002004E6007004E100BD
:10239000E004DC004005D700C005D2004006CD00B7
:1023A000D006C8008007C3003008BE00F008B9009E
:1023B000C009B400B00AAF00B00BAA00D00CA50051
:1023C000000EA000500F9B00C0109600501291000C
:1023D00000148C00C0158700B0178200B0197D0072
:1023E000D01B7800001E730040206E009022690010
:1023F000F024640040275F0090295A00E02B55002C
:10240000102E500020304B0010324600E0334100C7
:1024100090353C001037370070383200A0392D005D
:10242000B03A2800A03B2300603C1E00103D19007C
:10243000903D1400103E0F00703E0A00C03E0500A3
:10244000003F0000403FFBFF803FF6FFC03FF1FF31
:1024500000000A0B02090C0D0E080703040100001E
:10246000000000000000000000000000000000006C
:102470000000000000000000000000001211100029
:10248000000000000000000000000000000000004C
:1024900000000000000050726F62696E67204661A4
:1024A000696C656400205A3A200020593A200042A5
:1024B000656420583A20003D3D6F6E557365724348
:1024C0006F6E6669726D52657175697265643D3DC6
:1024D00000220A00556E6B6E6F776E20636F6D6D14
:1024E000616E643A2022002042002050006F6B0091
:1024F000204500205A00205900204D393220580034
:1025000020453A00205A3A0020593A00583A002013
:10251000746F6F206C6F6E67206578747275736965
:102520006F6E2070726576656E7465640A00206354
:102530006F6C6420657874727573696F6E20707249
:102540006576656E7465640A0043616E6E6F742013
:10255000656E746572207375626469723A20004D0D
:10256000323520500A4D323400526573756D650066
:102570005549205061757365004E6F204D6174633D
:1025800068203A0050675570005067446F776E00BE
:1025900049732046696C65200049732044697220A4
:1025A00000476F557044697200486173204D65643F
:1025B00069610046696C656E616D652053656C6587
:1025C00063746564004D3130303043004D3130303C
:1025D000300046696C616D656E74205374617420BF
:1025E00030202D20330046696C616D656E74205378
:1025F0007461742030202D20320046696C616D6555
:102600006E7420537461742030202D2031002046D8
:10261000696C616D656E7420526573706F6E736561
:10262000204E6F00526573756D6520596573206487
:102630007572696E67207072696E74000A204E6F41
:102640002046696C616D656E7400496E76616C69D7
:1026500064204F7074696F6E004D353030005374D4
:102660006F72652053657474696E677300426564A8
:10267000205049442053746172746564004D3939A7
:10268000390A4D32383050305331363000424C54D4
:102690006F756368205265736574004D3530320A7A
:1026A0004D35303000496E697420454550524F4DCC
:1026B00000486F74656E6420504944205374617201
:1026C00074656400456E676C69736820416C72655F
:1026D00061647920536574004368696E6573652091
:1026E0004E6F7420537570706F7274656400496E1C
:1026F0004C616E6743686F696365000A202A2A2A65
:102700007265636461742E646174615B305D203D49
:10271000004732380A4731204631303030205A31B4
:102720003000556E737570706F72746564204F70F1
:1027300074696F6E2053656C65637465640047321D
:102740003652323535004D3139305335350A47323E
:10275000380A47333449380A4732390A4D34303061
:102760000A4D313034533231350A4732380A4D314F
:102770003039533231350A4D34323053310A473112
:10278000583130305931303046353030300A4731E9
:102790005A300A4D3530300A4D3131372053657487
:1027A000205A204F666673657400473120463130E9
:1027B0003030205A302E30004732380A4731204618
:1027C00031303030205A302E30004D353030005A04
:1027D000204F6666736574203A202573004D3530AE
:1027E00030005A204F6666736574203A20257300C6
:1027F0004732380A473146313530305A302E3000B2
:102800004732385A0A473146313530305A302E3047
:10281000004D383400473146313030305A302E3098
:10282000004732380A473146313030305A302E3086
:10283000004D616E75616C53657454656D70005A1E
:10284000204F6666736574203A2025730053746FB9
:1028500070205472696767657265640053746F70A5
:10286000204E6F0053746F705072696E740048612F
:102870006E646C6520446174612041646A75737490
:1028800020322053657474696E67205363726565E6
:102890006E200048616E646C652044617461205054
:1028A00072696E7446696C6520332053657474696F
:1028B0006E672053637265656E200048616E646CBC
:1028C000652044617461205072696E7446696C655C
:1028D00020322053657474696E6720536372656596
:1028E0006E20004D38340048616E646C6520446190
:1028F0007461205072696E7446696C6520506F7304
:10290000740048616E646C6520446174612050728B
:10291000696E7446696C652050726500426567692E
:102920006E537769746368003D3D20436865636B4F
:102930006B65793D3D007265636461742E6164640A
:1029400072203D3D007265636461742E6461746140
:102950005B305D203D3D0077616974776179203D92
:102960003D0020202A2A2A2A2A2A2A5254535F4824
:10297000616E646C65446174612A2A2A2A2A2A2AB3
:102980002A2000526573656E643A20000000220020
:10299000250028002B002E00310034000201000029
:1029A000050108010B0100002100240027002A0076
:1029B0002D003000330001010000040107010A016D
:1029C00005050505070508080808020202020A0AAB
:1029D00008080404040401010101010101010303C9
:1029E000030303030303040707070C0C0C0C0C0C74
:1029F0000C0C0202020206060606060606060B0B71
:102A00000B0B0B0B0B0B01021020200808102040B1
:102A100010204080020102010804020101020408A2
:102A20001020408080402010080402018004020130
:102A30008040201008040201080402010102040879
:102A4000102040800102040810204080544D33447F
:102A500020453520506C75732052656164792E00D5
:102A60005072696E74696E672E2E2E005072696EF8
:102A70007420506175736564006E6F746966696374
:102A80006174696F6E20005049442054756E652052
:102A900046696E6973686564004572726F7220776B
:102AA000726974696E6720746F20454550524F4DAE
:102AB000210A0053544F505045442E200050726953
:102AC0006E7465722073746F7070656420647565D0
:102AD00020746F206572726F72732E2046697820A1
:102AE000746865206572726F7220616E6420757300
:102AF00065204D39393920746F20726573746172A5
:102B0000742E202854656D7065726174757265202D
:102B100069732072657365742E205365742069741F
:102B20002061667465722072657374617274696E77
:102B300067290A004E6F20436865636B73756D20CB
:102B400077697468206C696E65206E756D62657258
:102B50002C204C617374204C696E653A20004E6FD6
:102B600020436865636B73756D2077697468206CAA
:102B7000696E65206E756D6265722C204C61737490
:102B8000204C696E653A2000636865636B73756DF0
:102B9000206D69736D617463682C204C61737420BF
:102BA0004C696E653A20004C696E65204E756D6209
:102BB0006572206973206E6F74204C617374204CB1
:102BC000696E65204E756D6265722B312C204C61EB
:102BD0007374204C696E653A20004D3131300053DA
:102BE000657269616C20737461747573206D6973AB
:102BF0006D617463680A00776169740A0053442048
:102C000072656164206572726F720A002121204B27
:102C1000494C4C2063617573656420627920746F40
:102C20006F206D75636820696E61637469766520D5
:102C300074696D65202D2063757272656E742063F2
:102C40006F6D6D616E643A2000486F74656E64202C
:102C500049646C652054696D656F757400486F74C4
:102C6000656E642049646C652054696D656F757488
:102C70000A003D3D6F6E46696C616D656E745275FC
:102C80006E6F75743D3D007061757365004D363033
:102C900030002066696C616D656E745F72756E6F71
:102CA0007574200066696C616D656E745F72756E17
:102CB0006F757420540046696C616D656E74527551
:102CC0006E6F75742054002A2A2A496E6974696EE1
:102CD000672063617264206973204F4B2A2A2A009F
:102CE0004D6564696120496E736572746564004D59
:102CF000656469612052656D6F766564004D3130A1
:102D000030305300627573793A2070617573656471
:102D100020666F7220696E7075740A00627573792F
:102D20003A2070617573656420666F7220757365F3
:102D3000720A00627573793A2070726F63657373FB
:102D4000696E670A002A2A2A6B696C6C2A2A2A0093
:102D5000706F7765726F6666004B494C4C45442E28
:102D600020005072696E7465722068616C746564CD
:102D70002E206B696C6C28292063616C6C65642162
:102D80000A0053544F505045442E20005072696E33
:102D90007465722073746F7070656420647565204B
:102DA000746F206572726F72732E2046697820747A
:102DB0006865206572726F7220616E64207573653C
:102DC000204D39393920746F2072657374617274C3
:102DD0002E202854656D7065726174757265206966
:102DE000732072657365742E205365742069742096
:102DF00061667465722072657374617274696E675E
:102E0000290A006563686F3A004572726F723A0072
:102E100042696C696E656172204C6576656C696E9D
:102E20006720477269643A0A0021212053544F50A9
:102E30002063616C6C6564206265636175736520F5
:102E40006F6620424C546F756368206572726F72B2
:102E5000202D207265737461727420776974682004
:102E60004D3939390A0021212053544F50206361D4
:102E70006C6C65642062656361757365206F6620A4
:102E8000424C546F756368206572726F72202D20FA
:102E9000726573746172742077697468204D393972
:102EA000390A002F2F616374696F6E3A0070726F78
:102EB0006D70745F00656E640053656E64204D3103
:102EC000303820746F20726573756D650A00496E25
:102ED000736572742066696C616D656E7420616ED5
:102EE000642073656E64204D3130380A0052656885
:102EF0006561742066696E69736865642E00526549
:102F00006865617420446F6E650052656865617420
:102F1000696E672E2E2E00526568656174004865E3
:102F2000617465722054696D656F75740053656EC8
:102F300064204D31303820746F2068656174206ED4
:102F40006F7A7A6C650A004E6F7A7A6C65205061F0
:102F5000726B656400486F74656E6420746F6F20D7
:102F6000636F6C640A00706175736564005061750D
:102F700073650044697361626C6552756E6F757438
:102F80000050757267654D6F7265005061757365AD
:102F9000640073686F7700627574746F6E006265A9
:102FA00067696E004C6F61642046696C616D656E87
:102FB00074004C6F61642046696C616D656E7420AD
:102FC0005400496E736572742066696C616D656E3C
:102FD0007420616E642073656E64204D3130380A50
:102FE00000726573756D656400526573756D696E09
:102FF000670057616974696E6720666F7220686543
:10300000617475702E0A004C656176696E672047A1
:103010003236003F53706563696669656420582CD9
:103020005920636F6F7264696E617465206F757487
:10303000206F6620626F756E64732E0A003F2852FF
:103040002965706561742076616C7565206E6F749A
:1030500020706C61757369626C653B206D7573746B
:10306000206265206174206C6561737420312E0AC2
:10307000003F2852296570656174206D7573742056
:103080006265207370656369666965642077686549
:103090006E206E6F74207573696E6720616E204CB0
:1030A00043442E0A003F5370656369666965642076
:1030B0006E6F7A7A6C652074656D70657261747577
:1030C0007265206E6F7420706C61757369626C65D7
:1030D0002E0A003F537065636966696564206669FE
:1030E0006C616D656E742073697A65206E6F7420F3
:1030F000706C61757369626C652E0A003F53706570
:10310000636966696564207072696D65206C656EBF
:10311000677468206E6F7420706C61757369626C7F
:10312000652E0A003F5072696D65206C656E67748C
:1031300068206D75737420626520737065636966BD
:10314000696564207768656E206E6F742075736999
:103150006E6720616E204C43442E0A003F53706519
:10316000636966696564206E6F7A7A6C652073693D
:103170007A65206E6F7420706C61757369626C651E
:103180002E0A003F52657472616374696F6E204D40
:10319000756C7469706C696572206D7573742062EA
:1031A00065207370656369666965642E0A003F5324
:1031B00070656369666965642052657472616374E1
:1031C000696F6E204D756C7469706C696572206EE4
:1031D0006F7420706C61757369626C652E0A003FB4
:1031E000537065636966696564206C6179657220F6
:1031F000686569676874206E6F7420706C617573A0
:1032000069626C652E0A0043292E0A003F537065DF
:10321000636966696564206265642074656D7065C4
:10322000726174757265206E6F7420706C61757355
:1032300069626C65202834302D0047323620737463
:10324000617274696E672E2E2E0A004F46460A0080
:10325000466164652048656967687420004265645A
:10326000204C6576656C696E6720004661696C6507
:103270006420746F20656E61626C65204265642015
:103280004C6576656C696E670A00496E76616C699B
:1032900064206D6573682E0A0050726F62696E67F4
:1032A00020506F696E740025532025692F25690011
:1032B0002E0A002F0050726F62696E67206D657371
:1032C0006820706F696E742000202844525952554E
:1032D0004E2900473239204175746F2042656420C1
:1032E0004C6576656C696E67003F20284C2C522C2B
:1032F000462C4229206F7574206F6620626F756EB0
:1033000064732E0A003F2856296572626F73652028
:103310006C6576656C20696D706C61757369626C43
:10332000652028302D34292E0A00426164205A205D
:1033300076616C75650A004E6F2062696C696E6516
:10334000617220677269640A004163637572616328
:10335000792044656372656173696E672100446515
:103360006372656173696E6720416363757261633F
:10337000792044657465637465642E0A00473238A9
:10338000004732385A0041636375726163793A20AD
:1033900000206F66200044696420004733342061B8
:1033A000626F727465642E0A0041636375726163B3
:1033B0007920416368696576656400546172676568
:1033C0007420616363757261637920616368696504
:1033D0007665642E0A004469666673205A312D5A58
:1033E000323D2573000A444946464552454E434501
:1033F000205A312D5A323D0050726F62696E67203B
:103400004661696C65640050726F62696E67206620
:1034100061696C65640A00473334204974657261E0
:1034200074696F6E3A202569000A47333420497465
:1034300065726174696F6E3A20003F2841296D7092
:103440006C696669636174696F6E206F7574206F53
:103450006620626F756E64732028302E352D322EF3
:1034600030292E0A003F2854296172676574206153
:1034700063637572616379206F7574206F66206273
:103480006F756E64732028302E30312D312E302927
:103490002E0A003F2849297465726174696F6E2095
:1034A0006F7574206F6620626F756E6473202831AB
:1034B0002D3330292E0A003F285929206F7574209A
:1034C0006F6620626F756E64732E0A003F2858295C
:1034D000206F7574206F6620626F756E64732E0A9C
:1034E000003F2853292050726F62652D706F7369F9
:1034F00074696F6E20696E64657820696E76616CA0
:1035000069642E0A003F285329206973207265716F
:1035100075697265642E0A004D34323220530044BE
:103520006576696174696F6E0025533A20257300D2
:1035300046696E6973686564210A003A207A3A2008
:1035400000206F662000476F696E6720746F3A2015
:10355000580043570A00206469723A0020616E6780
:103560006C653A005374617274207261646975739A
:103570003A004D343820506F696E740025533A205C
:1035800025642F256400506F736974696F6E696ECE
:1035900067207468652070726F62652E2E2E0A0097
:1035A0003F4C656773206F66206D6F76656D656E45
:1035B0007420696D706C61757369626C6520283068
:1035C0002D3135292E0A003F2028582C5929206FEB
:1035D0007574206F6620626F756E64732E0A0050DA
:1035E000726F6265206F7574206F6620626F756EF2
:1035F0006473003F53616D706C652073697A652058
:103600006E6F7420706C61757369626C652028340C
:103610002D3530292E0A004D3438205A2D50726F26
:103620006265205265706561746162696C69747964
:1036300020546573740A003F2856296572626F73BF
:1036400065206C6576656C20696D706C6175736959
:10365000626C652028302D34292E0A005374616E67
:103660006461726420446576696174696F6E3A20A2
:10367000002052616E67653A2000204D61783A2043
:1036800000204D696E3A2000205369676D613A2031
:10369000004D65616E3A20005741524E494E472118
:1036A000204C6F77205A204A65726B206D6179201B
:1036B0006C65616420746F20756E77616E746564EB
:1036C000207061757365732E0A00F600680111247D
:1036D0001FBECFEFD1E2DEBFCDBF00E00CBF14E0D4
:1036E000A0E0B2E0EEE2FFE602E00BBF02C007900E
:1036F0000D92A431B107D9F726E1A4E1B4E001C0ED
:103700001D92A734B207E1F71BE1C6E6DBE100E05A
:1037100006C021970109802FFE010F94C433C536DE
:10372000D10780E00807A9F70F9436210D9485375B
:103730000C9400009F92AF92BF92CF92DF92EF92D3
:10374000FF920F931F93CF93DF9300D01F921F928E
:10375000CDB7DEB7E2E0F1E10027BB27462F572FB8
:10376000A82FAA2341F4A52F542FB85FAA2319F438
:10377000A52F5527B85FA03138F45295A295452F53
:103780004F70507FA42BBC5FA03428F4550FAA1FA4
:10379000550FAA1FBE5FA03818F4550FAA1FB39586
:1037A000550FAA1FEA0FF01F449151E0AA27B85005
:1037B00081F1C8F0B0FF02C0440F551FB1FF04C033
:1037C000440F551F440F551FB2FF06C05295429536
:1037D000142F1F70407F512BB3FF1BC0A52F542FF8
:1037E00044270C94091CB195B0FF02C0559547952C
:1037F000B1FF04C05595479555954795B2FF05C053
:103800005295407F4295452B5F70B3FF02C0452F14
:103810005527DD24CC24BB24B2E0649FD018C10816
:10382000B00AB00B749FC018B108B00B849FB018D9
:10383000B109659FC018B108B00B759FB018B109E8
:10384000859FB0196A9FB018B1097A9FB0194D9D34
:10385000A12C99243327992722275D9DA00C911C28
:10386000301F901F201FAD9D900C311D901F201FF9
:103870004C9DA00C911C301F901F201F5C9D900C34
:10388000311D901F201FAC9D300D911D201F4B9DA1
:10389000900C311D901F201F5B9D300D911D201F2E
:1038A000AB9D900D211D4B9F300D911D201F5B9FE7
:1038B000900D211DAB9F200DB1E0BB24CC24DD2455
:1038C000639FD018C108B00AB00B739FC018B1082D
:1038D000B00B839FB018B109699FC018B108B00B35
:1038E000799FB018B109899FB019629FB018B109CA
:1038F000729FB019D61AC70AB80A20F0B1E03B0F80
:10390000901F201F1124792F632F90E0822F0F909A
:103910000F900F900F900F90DF91CF911F910F910B
:10392000FF90EF90DF90CF90BF90AF909F90089561
:10393000AF92BF92CF92DF92EF92FF920F931F93BD
:10394000CF93DF93C0E5DBE00FE018E080E6A82E20
:103950008BE0B82EC12CD12C7601C394699179915A
:10396000899199910F94022D288939894A895B8917
:103970000F94632D0F944035F801619371938193F7
:1039800091938F01C616D706E806F90610F46B016D
:103990007C01AC16BD0611F76FEF7FEFCB01A701DD
:1039A00096010F94413320931F08309320084093D1
:1039B000210850932208DF91CF911F910F91FF9022
:1039C000EF90DF90CF90BF90AF900895CF93DF93AB
:1039D00024E0829FC0011124EC01CE50D84FFC019D
:1039E000E85DF84F845E984FDC012D913D914D913B
:1039F0005C9160817181828193810F94CD33688362
:103A000079838A839B83DF91CF91089580919B1165
:103A100090919C11891B877089F48091A30C81116E
:103A20000DC08091980B9091990B892B39F481E00E
:103A30009091CA05911103C080E0089581E0089536
:103A400090E080E00895282F90911607833021F4AC
:103A500095FD0FC094FD0FC0892F90E0B0E0A0E06D
:103A600004C0B695A795979587952A95D2F781704A
:103A7000089581E0089580E00895CF93C82FCB0189
:103A80000E94A9F786E79EE00E94A9F787E69EE0DC
:103A9000CC2311F08CE69EE00E94A9F78AE0CF913A
:103AA0000C9481F70F931F93CF938C01C62F89EC51
:103AB00099E00E94A9F7C8010E94A9F78AE30E9431
:103AC00081F780E38C0F0E9481F78AE0CF911F91EC
:103AD0000F910C9481F78CE49BE00E94A9F760E0C1
:103AE0008CE39BE00E94521D60E087E29BE00E9415
:103AF000521D61E080E29BE00E94521D61E085E181
:103B00009BE00E94521D61E085E09BE00E94521DF7
:103B100060E08CEF9AE00E94521D61E082EF9AE033
:103B20000E94521D61E088EE9AE00E94521D61E001
:103B300081EE9AE00E94521D61E089ED9AE00E94B8
:103B4000521D61E08BEC9AE00E94521D61E08DEB0A
:103B50009AE00E94521D60E08EEA9AE00E94521D97
:103B600060E080EA9AE00E94521D60E08AE89AE0F4
:103B70000E94521D61E089E79AE00E94521D61E0B7
:103B80008AE69AE00E94521D61E083E69AE00E9474
:103B9000521D60E08CE59AE00E94521D61E083E5D1
:103BA0009AE00E94521D61E08EE39AE00E94521D4D
:103BB00061E080E39AE00E94521D61E08DE19AE0AD
:103BC0000E94521D60E080E19AE00E94521D61E077
:103BD0008BE09AE00E94521D61E08EEF99E00E9416
:103BE000521D60E08AEE99E00E94521D60E087ED70
:103BF00099E00E94521D60E086E493E10E94201D3E
:103C0000682F61708EEC99E00C94521DCF93DF9376
:103C100080919B1190919C11891B8095877019F45C
:103C20000F94440FF5CF80919B118F5F8770A09107
:103C30009B119CE5A99FD0011124FD01E85DF74F80
:103C4000EF0119929A95E9F798E09083A35CB74F3A
:103C500090E1EDE9F1E101900D929A95E1F7209163
:103C60009B1190919C11291303C094E69093981195
:103C700080939B11DF91CF910C94BCF22F923F92D5
:103C80004F925F926F927F928F929F92AF92BF926C
:103C9000CF92DF92EF92FF920F931F93CF93DF9318
:103CA000D62FC72FFC0180809180A280B380C501F0
:103CB000B40120E831E541E050E00F944133C901FF
:103CC0006DE671E00F94B0336B017C01C501B40166
:103CD00020E13EE040E050E00F944133CA01B901D9
:103CE00028E130E040E050E00F944133362E272E9B
:103CF000062F172F8CE3482E512C612C712CC501F7
:103D0000B401A30192010F944133B62EA72ECA012C
:103D1000B901A30192010F944133CB01C114D10425
:103D200079F1AF92BF927F936F932F923F92FF9260
:103D3000EF92DF92CF9289E09DE09F938F93CF9394
:103D4000DF930F94942C8DB79EB70E960FB6F89410
:103D50009EBF0FBE8DBF8D2F9C2FDF91CF911F91E6
:103D60000F91FF90EF90DF90CF90BF90AF909F901A
:103D70008F907F906F905F904F903F902F9008951D
:103D8000E114F104C9F0AF92BF927F936F932F9229
:103D90003F92FF92EF9289EF9CE09F938F93CF9396
:103DA000DF930F94942CEDB7FEB73C960FB6F894C2
:103DB000FEBF0FBEEDBFCFCF012BB9F0AF92BF92C8
:103DC0007F936F932F923F928DEE9CE09F938F9302
:103DD000CF93DF930F94942C8DB79EB70A960FB6AE
:103DE000F8949EBF0FBE8DBFB6CF892BA9F0AF92BE
:103DF000BF927F936F9385EE9CE09F938F93CF93B9
:103E0000DF930F94942CEDB7FEB738960FB6F89465
:103E1000FEBF0FBEEDBF9FCFAF92BF9281EE9CE081
:103E20009F938F93CF93DF930F94942C0F900F90C9
:103E30000F900F900F900F908ECFCF93DF9300D005
:103E40001F92CDB7DEB784EF91E0A0E0B0E08983A8
:103E50009A83AB83BC83BE016F5F7F4F8CE30E946C
:103E600045F584E99EE00E94A9F78CB16EE87EE0FA
:103E700085FB882780F90E943D1D8091030168E839
:103E80007EE0869581700E943D1D89B162E87EE0EA
:103E900083FB882780F90E943D1D8CB169E77EE095
:103EA000829581700E943D1D4B9909C00E9480F54A
:103EB0000F900F900F900F90DF91CF9108950E9477
:103EC00065F50F900F900F900F90DF91CF910895AF
:103ED00080910A06882319F010920A06089540E09E
:103EE00070E060E089E59EE00F94730ECF93C0917F
:103EF0009B04CF7739F50E94D8F3882319F180917C
:103F00003B1390913C13A0913D13B0913E13009749
:103F1000A105B105B9F0BC01CD016D597F4F8F4F9F
:103F20009F4F24E630E040E050E00F944133609131
:103F30003F137091401380914113909142130F945D
:103F40004133C22F8C2FCF910895CF93DF93EB0194
:103F50000E9476EE882319F00E94C6EDEB01CE0197
:103F6000DF91CF9108954F925F926F927F928F92DF
:103F70009F92AF92BF92CF92DF92EF92FF921F93E8
:103F8000CF93DF9300D01F92CDB7DEB719821A828C
:103F90001B821C82CE0101964C0186E9C82E86E068
:103FA000D82E9AE4E92E92E0F92E22EFA22E27E0F5
:103FB000B22E10E088E5810F0E9476EEF401819325
:103FC0004F01882309F4E0C00E94FEED2B013C0163
:103FD000812F0E94231D882309F4CCC0F701208182
:103FE000318142815381C301B2010F94CD33F60177
:103FF00060837183828393831F5FF4E0CF0ED11CB3
:1040000084E0E80EF11C94E0A90EB11C133091F687
:1040100085E40E9476EE8C83882309F4C0C00E9458
:10402000FEED6B017C0183E00E94231D882371F06B
:1040300020915602309157024091580250915902F6
:10404000C701B6010F94CD336B017C01C092A2066B
:10405000D092A306E092A406F092A5068091DC041B
:10406000882359F18091431382FF27C08C818823D4
:1040700021F18981811103C08A818823F1F02DEC1F
:104080003CEC4CE45DE360913D0770913E0780910C
:104090003F07909140070F94CD339B01AC01609195
:1040A00052027091530280915402909155020F94E4
:1040B0002D36181614F40E944CC240E050E0BA01AC
:1040C00086E40E94E3EE20E030E0A9010F942D3653
:1040D000181684F40E94FEED20E030E040E752E440
:1040E0000F94C73460932A0270932B0280932C02A2
:1040F00090932D028091080B83FD28C08091B50517
:10410000882321F1209156023091570240915802A4
:10411000509159026091A2067091A3068091A40665
:104120009091A5060F94CC332091C2053091C30520
:104130004091C4055091C5050F94CD336093C205DD
:104140007093C3058093C4059093C5050F900F909D
:104150000F900F90DF91CF911F91FF90EF90DF9024
:10416000CF90BF90AF909F908F907F906F905F9017
:104170004F900895F5012081318142815381C3011F
:10418000B2010F94CC3333CFF70180819181A281AA
:10419000B381F60180839183A283B3832DCF809175
:1041A000560290915702A0915802B0915902809303
:1041B000A2069093A306A093A406B093A5064ECFA3
:1041C000CF9384E50E9476EEC0E08823D9F00E9468
:1041D000D6EDC82F1816B4F40F94990B8DE40E94F5
:1041E00081F780918C0490918D040E9418AD6C2F02
:1041F000CC0F770B8DE495E00E94FCF98AE00E94D9
:1042000081F7CFEF8C2FCF910895CF92DF92EF926D
:10421000FF920F931F93CF93DF93CDB7DEB7A09795
:104220000FB6F894DEBF0FBECDBF0E94E02087FD21
:10423000CCC085E40E9428EE882309F4D5C00E94F2
:10424000FEED6B017C0120E030E0A9010F942D36DA
:1042500087FF04C0F7FAF094F7F8F094F7FAF094B7
:10426000F7F8F094CD8EDE8EEF8EF8A28CE0EBE8BE
:10427000F2E0DE01119601900D928A95E1F78AE550
:104280000E9476EE882351F040E050E0BA018AE5C2
:104290000E94E3EE69877A878B879C8788E50E9476
:1042A00076EE882351F040E050E0BA0188E50E94A4
:1042B000E3EE69837A838B839C8389E50E9476EEA3
:1042C000882351F040E050E0BA0189E50E94E3EE16
:1042D0006D837E838F83988785E50E9428EE8823EF
:1042E00009F489C00E94FEED6B017C0120E030E002
:1042F000A901C701B6010F942D3687FF04C0F7FA54
:10430000F094F7F8F094F7FAF094F7F8F094C98E77
:10431000DA8EEB8EFC8E1D8A1E8A1F8A188E8CE424
:104320000E9428EE882309F46FC00E94FEED6B0105
:104330007C0120E030E0A901C701B6010F942D36C1
:1043400087FF04C0F7FAF094F7F8F094C98ADA8A84
:10435000EB8AFC8A62E070E082E40E94FAEEF82EBA
:1043600080913510811131C021E0AE01475E5F4F71
:10437000BE016F5F7F4FCE014D960F94F31D8823D2
:1043800021F16F2D81E00F94C51E82E50E9476EE2B
:10439000882309F442C00E94FAED40E050E060EA50
:1043A00071E44D875E876F87788B209135102223CB
:1043B00061F08C012F2DAE01435F5F4FBE016F5E38
:1043C0007F4FCE0145960F94B01CA0960FB6F8947F
:1043D000DEBF0FBECDBFDF91CF911F910F91FF9038
:1043E000EF90DF90CF900895C12CD12C80E8E82E7B
:1043F00080E4F82E33CFC090D404D090D504E09060
:10440000D604F090D70472CFC090D804D090D904CD
:10441000E090DA04F090DB048CCF90E080E0BDCF38
:10442000CF92DF92EF92FF920F931F93CF93DF9380
:10443000CDB7DEB76C970FB6F894DEBF0FBECDBF19
:104440008CE40E9428EE882309F4B0C00E94FEED9F
:104450006B017C0120E030E0A9010F942D3687FF2D
:1044600004C0F7FAF094F7F8F094F7FAF094F7F83C
:10447000F094C98EDA8EEB8EFC8E8CE0EBE8F2E0E5
:10448000DE01119601900D928A95E1F788E50E9470
:1044900076EE8823A1F040E050E0BA0188E50E9462
:1044A000E3EE2091F2073091F3074091F407509129
:1044B000F5070F94CC3369837A838B839C8389E5DA
:1044C0000E9476EE8823A1F040E050E0BA0189E531
:1044D0000E94E3EE2091F2073091F3074091F40738
:1044E0005091F5070F94CC336D837E838F8398872B
:1044F0008AE50E9476EE882351F040E050E0BA0150
:104500008AE50E94E3EE69877A878B879C871D8600
:104510001E861F86188A80913510811138C020E0D0
:10452000AE01435F5F4FBE016F5F7F4FCE01499683
:104530000F94F31D882359F18091DC0481110E94AE
:104540004CC260E080E00F94C51E898D9A8DAB8DC2
:10455000BC8DB0588D8B9E8BAF8BB88F198A1A8A01
:104560001B8A1C8A1D861E861F86188A809135101C
:10457000882369F010E000E020E0AE014B5E5F4F61
:10458000BE016F5E7F4FCE010D960F94B01C6C96EE
:104590000FB6F894DEBF0FBECDBFDF91CF911F9154
:1045A0000F91FF90EF90DF90CF900895C12CD12C08
:1045B00080E8E82E80E4F82E58CF84E690E09093CF
:1045C000D3048093D20410920305109202050C9438
:1045D000BEA60F93AB010091010521E0022722E066
:1045E00035E0BC0182ED94E00E9402F40F91089541
:1045F000CF93DF9300D01F92CDB7DEB78091B50582
:104600008823C1F083E390E09C838B831A82198214
:104610009E012F5F3F4F40E150E066EB75E0CE0119
:1046200003960F94030E86E492E10E94A9F78AE0B4
:104630000E9481F70F900F900F900F90DF91CF9114
:104640000895CF93DF9300D01F921F92CDB7DEB7AE
:1046500081E08093B50580E1E6EBF5E0DF011D9296
:104660008A95E9F70E94F82286E18D8382E390E043
:104670009C838B831A8219829E012F5F3F4F41E0FA
:1046800050E0BE016B5F7F4FCE0103960F94030E87
:104690000F900F900F900F900F90DF91CF91089592
:1046A000CF92DF92EF92FF92CF93DF93EC010896C7
:1046B0000E94E6E96B017C0120E030E0A9010F9443
:1046C000FD2C20E030E0A901882359F0CE010E94A2
:1046D000CFEF9B01AC01C701B6010F94632D9B0185
:1046E000AC01688579858A859B850F94CC33688772
:1046F00079878A879B87DF91CF91FF90EF90DF903A
:10470000CF9008958C3221E0920714F08CE291E072
:10471000909300118093FF100C9486C80F931F9301
:10472000CF93DF9304E61BE0C8E7D0E1F8012191C5
:104730003191419151918F0160E070E080E89FE3F9
:104740000F94C7346993799389939993F0E1C838AA
:10475000DF0761F70E948BC0DF91CF911F910F910E
:104760000C94981C90919B1180919C11981306C0F9
:104770008091260890912708892B21F080E00F94E2
:10478000440FF0CF089590919B1180919C11981344
:1047900008C08091260890912708892B11F40C9469
:1047A000BEF380E00F94440FEECFCF92DF92EF92F2
:1047B000FF92CF93DF9320914B0B222329F1EC0141
:1047C00008960E94E6E96B017C0120E030E0A90137
:1047D0000F94FD2C20E030E0A901882359F0CE0190
:1047E0000E94CFEF9B01AC01C701B6010F94632D6E
:1047F0009B01AC01688579858A859B850F94CD33B3
:10480000688779878A879B87DF91CF91FF90EF90A8
:10481000DF90CF900895CF92DF92EF92FF92809138
:104820001B07882309F457C0C0901707D0901807BA
:10483000E0901907F0901A0720E030E0A901C701C5
:10484000B6010F94FD2C882309F445C020E030E028
:1048500040E05FE3C701B6010F94632D9B01AC01FB
:104860000F94632D2BED3FE049E450E40F94632D4A
:104870009B01AC0160E070E080E89FE30F94C734D7
:104880006B017C01C0924C0BD0924D0BE0924E0B11
:10489000F0924F0B60915E0270915F02072E000C48
:1048A000880B990B0F94042D2AE037ED43E25CE36B
:1048B0000F94632DA70196010F94632D60935A0204
:1048C00070935B0280935C0290935D02FF90EF9087
:1048D000DF90CF900895C12CD12C80E8E82E8FE393
:1048E000F82ED0CF0F931F93CF93DF9350E0FC01AE
:1048F000E40FF51F8081440F551F440F551F4E5480
:104900005B4FEA01882329F188819981AA81BB81C3
:10491000EB01088119812A813B810097A105B1052E
:1049200069F40C591F4F2F4F3F4FDA010D931D9320
:104930002D933C9313978FEF808306C0081B190BB0
:104940002A0B3B0B37FDF7CFDF91CF911F910F91D2
:104950000895188219821A821B82F6CF2F923F92F5
:104960004F925F926F927F928F929F92AF92BF927F
:10497000CF92DF92EF92FF920F931F93CF93DF932B
:10498000CDB7DEB76C970FB6F894DEBF0FBECDBFC4
:104990008C015B015A834983FC01EA5BFF4F208154
:1049A00031814281538129873A874B875C87CA01CD
:1049B000B9010F94022D6B017C01D5012D913D9120
:1049C0004D915C910F94632D0F94AB342B013C01FE
:1049D000E981FA812081318142815381C701B60189
:1049E0000F94632D0F94AB344B015C01C301B201F2
:1049F0000F944035698B7A8B8B8B9C8B6837710554
:104A00008105910540F428E730E040E050E0298B33
:104A10003A8B4B8B5C8BC501B4010F9440356D878D
:104A20007E878F87988B683771058105910540F4E3
:104A300048E750E060E070E04D875E876F87788BD5
:104A4000F801EE5AFF4F4080518062807380C301AD
:104A5000B2010F94042D69837A838B839C836989C7
:104A60007A898B899C890F94022D6D8B7E8B8F8B1D
:104A7000988F20E030E0A90169817A818B819C8147
:104A80000F94FD2C882309F4E1C1A7019601C70109
:104A9000B6010F94632D4B015C012D893E894F892E
:104AA000588DCA01B9010F94632D9B01AC01C5015A
:104AB000B4010F94CC334B015C0129813A814B81C5
:104AC0005C81CA01B9010F94CD339B01AC01C501D2
:104AD000B4010F94C7340F94AB340F9440356D83F9
:104AE0007E838F83988766277727CB0164197509A2
:104AF000860997090F94042D4B015C016D857E8515
:104B00008F8598890F94022D2B013C0120E030E025
:104B1000A901C501B4010F94FD2C882309F49AC1A1
:104B2000A3019201C301B2010F94632D698F7A8FA3
:104B30008B8F9C8FA7019601C701B6010F94632D3F
:104B40009B01AC01698D7A8D8B8D9C8D0F94CC333C
:104B50006B017C01A5019401C501B4010F94CD3313
:104B60009B01AC01C701B6010F94C7340F946F3598
:104B7000D80195968D909D90AD90BC9098977501B9
:104B800064012D813E814F815885C21AD30AE40AFF
:104B9000F50A0F944035C61AD70AE80AF90AF7FE53
:104BA0008EC02D893E894F89588DCA01B9010F9455
:104BB000632D6B017C0129813A814B815C81CA01A3
:104BC000B9010F94CD3369877A878B879C8720E062
:104BD00030E0A90169817A818B819C810F94FD2C41
:104BE000882309F43BC1C501B4010F94022D298526
:104BF0003A854B855C850F94632DA70196010F9430
:104C0000CC336D837E838F839887A3019201C30188
:104C1000B2010F94632D9B01AC016D817E818F8168
:104C200098850F94CD332B013C0120E030E040E823
:104C300050E469817A818B819C810F94632D9B0163
:104C4000AC01C301B2010F94C7340F94AB342B01F4
:104C50003C0120E030E0A9010F942D3618161CF01D
:104C6000412C512C3201C301B2010F9440356D83A8
:104C70007E838F83988786169706A806B90620F448
:104C80008D829E82AF82B8866D817E818F8198856C
:104C90000F94022D29853A854B855C850F94632DF1
:104CA000A70196010F94CD330F947B360F944035B6
:104CB00069877A878B879C87C12CD12C760169857F
:104CC0007A858B859C8529893A894B895C89621B09
:104CD000730B840B950B0F94022D29813A814B8124
:104CE0005C810F94C73420E034E244EF59E40F9420
:104CF000632D0F9440354B015C0169857A858B8566
:104D00009C852D853E854F855889621B730B840BCE
:104D1000950B0F94022D29813A814B815C810F9470
:104D2000C73420E034E244EF59E40F94632D0F942C
:104D300040352B013C013FE683169104A104B104E8
:104D400008F090C0F401EE0FFF1FEE0FFF1FEA5BAB
:104D5000F04F85919591A591B4918983292E3A2E92
:104D6000BD8B4FE6441651046104710408F083C002
:104D7000F201EE0FFF1FEE0FFF1FEA5BF04F4591B0
:104D80005591659174919A01CB014D815E816F813E
:104D90007885D80199964D935D936D937C939C97FC
:104DA0004C0D5D1D6E1D7F1DF80145A756A767A719
:104DB00070ABE65BFF4F49895A896B897C894083D8
:104DC000518362837383D5968D929D92AD92BC92EE
:104DD000D897F80141AE52AE63AE74AEFD964981EC
:104DE0004083218232825D895383349620833183CC
:104DF0008283938369857A858B859C85D1966D9313
:104E00007D938D939C93D4973D962D853E854F85BC
:104E1000588920833183428353836C960FB6F8946C
:104E2000DEBF0FBECDBFDF91CF911F910F91FF90DD
:104E3000EF90DF90CF90BF90AF909F908F907F903A
:104E40006F905F904F903F902F90089560E070E0DA
:104E5000CB0141CE60E070E0CB0188CE60E070E035
:104E6000CB01F3CEC501B4010E949A1B6983272EA2
:104E7000382E9D8B76CFC301B2010E949A1B9B01F5
:104E800084CF80919B1190919C11891B877019F49C
:104E900090E080E0089590919811992351F083302B
:104EA00030F48FEF890F19F080939811F1CF1092A1
:104EB000981180919C112CE5829FC0011124885D7E
:104EC000974FFC01208120FDE3CF20919C112F5FA3
:104ED00027702093991130919C1120919A113213CF
:104EE00004C02091991120939A11089590916F0018
:104EF00081E091FD02C080E0089590916F009D7F58
:104F000090936F000895FC0120813181428153818B
:104F10006091700B7091710B8091720B9091730B7B
:104F20000F94632D0F943A366093A9117093AA11D0
:104F30008093AB119093AC1190919B1180919C1137
:104F400098130C94061E0E94B2230E94762740916B
:104F5000A9115091AA116091AB117091AC114093BD
:104F60002E0550932F056093300570933105811104
:104F70000C94BCF208954F925F926F927F928F9241
:104F80009F92AF92BF92CF92DF92EF92FF920F93D8
:104F90001F93CF93DF93EC018B015A01F90120910C
:104FA000700B3091710B4091720B5091730B6081BB
:104FB0007181828193810F94632D0F943A366B0136
:104FC0007C0120916C0B30916D0B40916E0B5091D8
:104FD0006F0BF50160817181828193810F94632D44
:104FE0000F943A364B015C012091680B3091690BAC
:104FF00040916A0B50916B0BF80160817181828145
:1050000093810F94632D0F943A362B013C0120912C
:10501000640B3091650B4091660B5091670B688172
:1050200079818A819B810F94632D0F943A36609326
:105030009D1170939E1180939F119093A0114092A7
:10504000A1115092A2116092A3117092A4118092AA
:10505000A5119092A611A092A711B092A811C0928A
:10506000A911D092AA11E092AB11F092AC119091DB
:105070009B1180919C11981791F0DF91CF911F9116
:105080000F91FF90EF90DF90CF90BF90AF909F90E7
:105090008F907F906F905F904F900C94061E0E94AF
:1050A000B2230E9476274091A5115091A6116091DC
:1050B000A7117091A8110091A1111091A211209136
:1050C000A3113091A411C0909D11D0909E11E09039
:1050D0009F11F090A011C0922205D0922305E0927A
:1050E0002405F092250500932605109327052093AB
:1050F00028053093290540932A0550932B0560938A
:105100002C0570932D054091A9115091AA11609121
:10511000AB117091AC1140932E0550932F05609305
:10512000300570933105882391F0DF91CF911F9165
:105130000F91FF90EF90DF90CF90BF90AF909F9036
:105140008F907F906F905F904F900C94BCF2DF91A6
:10515000CF911F910F91FF90EF90DF90CF90BF9074
:10516000AF909F908F907F906F905F904F90089539
:10517000CF92DF92EF92FF92CF93DF93C82F0E94DE
:10518000762794E0C99FE0011124FE01EE5DFA4FFD
:10519000C080D180E280F38081110E94BCF2C858A7
:1051A000DF4EC701B6010F94042D288139814A8151
:1051B0005B810F94632DDF91CF91FF90EF90DF9093
:1051C000CF9008953F924F925F926F927F928F920D
:1051D0009F92AF92BF92CF92DF92EF92FF920F9386
:1051E0001F93CF93DF93CDB7DEB768970FB6F894D0
:1051F000DEBF0FBECDBFD82E2A013B0148015901A9
:105200003E2C20E030E0A901C501B8010F94FD2C2F
:10521000811110C081E08D1508F0B6C060E070E02B
:1052200080E793E420E030E040E752E40F94C73495
:105230004B015C018D8A9E8AAF8AB88E0D2D10E0DD
:10524000F801ED5BF04FE491BB24B3941E160CF40F
:10525000B12CCC24C39420E030E0A901C301B201F9
:105260000F942D3618160CF0C12CBC1471F092E07E
:10527000D9120BC0332049F081E00E9413C469E1C8
:1052800070E080E090E00E94D9F280E00E94B828AF
:1052900069837A838B839C8381E00E94B8286D8325
:1052A0007E838F83988782E00E94B82869877A87F7
:1052B0008B879C8783E00E94B8286D877E878F87C5
:1052C000988B000F111F000F111FE1E0F0E0EC0FB1
:1052D000FD1F0E0F1F1FF801108211821282138210
:1052E0009E01235F3F4FAE01475F5F4FBE016B5F83
:1052F0007F4FCE0101960E94BB27F8014082518268
:1053000062827382198A1A8A1B8A1C8A80912608F3
:1053100090912708892B91F4CE0141967C018E0152
:105320000B5E1F4F9E01235F3F4FAE01475F5F4FF4
:10533000BE016B5F7F4F40970E94BDB20E94B223B7
:10534000BC1451F092E0D91205C0332019F080E06E
:105350000E9413C40E94681F68960FB6F894DEBFBF
:105360000FBECDBFDF91CF911F910F91FF90EF90B6
:10537000DF90CF90BF90AF909F908F907F906F9075
:105380005F904F903F90089560E070E88BE395E464
:1053900049CFCF92DF92EF92FF92CF93DF93C82F46
:1053A0000E94762794E0C99FE0011124FE01EA5E85
:1053B000FA4FC080D180E280F38081110E94BCF25C
:1053C000C858DF4EC701B6010F94042D28813981DA
:1053D0004A815B810F94632DDF91CF91FF90EF9015
:1053E000DF90CF9008950E94762790919C11909322
:1053F0009B1190939A119093991194E69093981120
:1054000020ED33E0309327082093260881110E9475
:10541000BCF281E080931505089580FF04C090914F
:105420004A0B90FD8E7F81FF05C090914A0B9695A7
:1054300090FD8D7F82FF06C090914A0B96959695C0
:1054400090FD8B7F08958F929F92AF92BF92CF92E3
:10545000DF92EF92FF92CF93DF9320912E022223CF
:1054600009F49EC0EC0180918604C82ED12CF12C49
:10547000E12C80FF2CC08090300290903102A090EF
:105480003202B0903302288139814A815B81C501A3
:10549000B4010F942D36181624F488829982AA82BA
:1054A000BB8280903C0290903D02A0903E02B09062
:1054B0003F02288139814A815B81C501B4010F9483
:1054C000FD2C87FF04C088829982AA82BB82D70103
:1054D000C601B695A7959795879580FF2CC08090BB
:1054E000340290903502A0903602B09037022C81A1
:1054F0003D814E815F81C501B4010F942D36181690
:1055000024F48C829D82AE82BF8280904002909073
:105510004102A0904202B09043022C813D814E8115
:105520005F81C501B4010F94FD2C87FF04C08C82FC
:105530009D82AE82BF8282E0F694E794D794C794AE
:105540008A95D1F7C0FE2CC0C0903802D0903902A5
:10555000E0903A02F0903B02288539854A855B85C8
:10556000C701B6010F942D36181624F4C886D986C3
:10557000EA86FB86C0904402D0904502E090460245
:10558000F0904702288539854A855B85C701B601B9
:105590000F94FD2C87FF04C0C886D986EA86FB8657
:1055A000DF91CF91FF90EF90DF90CF90BF90AF90C1
:1055B0009F908F9008952F923F924F925F926F929B
:1055C0007F928F929F92AF92BF92CF92DF92EF9293
:1055D000FF920F931F93CF93DF93CDB7DEB7A697BC
:1055E0000FB6F894DEBF0FBECDBF86E996E00E94ED
:1055F000232A8091080B83FD7EC0209156023091B2
:10560000570240915802509159026091A206709140
:10561000A3068091A4069091A5060F94FD2C8823E3
:1056200009F469C010912508111161C080914802E8
:105630009091490201972091FD103091FE1028179A
:1056400039073CF40F94990B8DEC9EE00E94A9F76A
:1056500011E020915602309157024091580250912A
:1056600059026091A2067091A3068091A4069091C0
:10567000A5060F94CC336B017C0120E030E0A9013A
:105680000F942D3687FF04C0F7FAF094F7F8F094E2
:1056900020915A0230915B0240915C0250915D0270
:1056A000C701B6010F94632D20E030E84BE354E4CA
:1056B0000F942D361816ECF40F94990B8EEA9EE099
:1056C0000E94A9F78091A2069091A306A091A4063A
:1056D000B091A5068093560290935702A09358026A
:1056E000B093590282EA96E00E94832704C010E03A
:1056F000B0CF1111E7CF2AE037ED43E25CE36091D0
:105700002A0270912B0280912C0290912D020F940D
:10571000632D6B017C016091600270916102072E24
:10572000000C880B990B0F94042D9B01AC01C70151
:10573000B6010F94632D698B7A8B8B8B9C8B809138
:105740004B0B882309F18090EE079090EF07A09013
:10575000F007B090F107C0909E06D0909F06E090B1
:10576000A006F090A10620E030E0A901C501B40137
:105770000F94FD2C8823D1F1A7019601C501B40136
:105780000F942D36181694F1C12CD12C76018E0170
:105790000F5E1F4F22EA36E04EE956E06AE976E0F6
:1057A00086E996E00E9487BF80E1E6E9F6E0AAE498
:1057B000B2E001900D928A95E1F7A6960FB6F894A3
:1057C000DEBF0FBECDBFDF91CF911F910F91FF9034
:1057D000EF90DF90CF90BF90AF909F908F907F9091
:1057E0006F905F904F903F902F90089520914A02C4
:1057F00030914B0240914C0250914D0260919606BF
:105800007091970680919806909199060F94CC33E9
:105810006D8B7E8B8F8B988F20914E0230914F0233
:10582000409150025091510260919A0670919B06EE
:1058300080919C0690919D060F94CC33698F7A8F4E
:105840008B8F9C8F209152023091530240915402D1
:1058500050915502C701B6010F94CC336D8F7E8FE6
:105860008F8F98A320915602309157024091580291
:10587000509159026091A2067091A3068091A406EE
:105880009091A5060F94CC336B017C0120E030E0B1
:10589000A9016D897E898F89988D0F94FD2C8111C6
:1058A0000CC020E030E0A901698D7A8D8B8D9C8D34
:1058B0000F94FD2C882309F467CF2D893E894F89E9
:1058C000588DCA01B9010F94632D4B015C01298DDC
:1058D0003A8D4B8D5C8DCA01B9010F94632D9B01EC
:1058E000AC01C501B4010F94CD334B015C012D8D8A
:1058F0003E8D4F8D58A1CA01B9010F94632D9B01B4
:10590000AC01C501B4010F94CD334B015C01A7017B
:105910009601C701B6010F94632D9B01AC01C5012F
:10592000B4010F94CD330F947B364B015C012DEB0A
:1059300037E346E855E30F94FD2C87FF0FC020E0C6
:1059400030E0A901C701B6010F942D364601570179
:1059500087FF04C0B7FAB094B7F8B0942DEB37E3E3
:1059600046E855E3C501B4010F94FD2C87FD1CCF1B
:1059700020E030E040EA51E4C501B4010F94C7349F
:105980000F9440351B01672B19F422242394312CEA
:10599000B10190E080E00F94022D9B01AC0160E02A
:1059A00070E080E89FE30F94C7342B013C01AC0109
:1059B0009B01C501B4010F94632D4B015C01A30150
:1059C00092016D897E898F89988D0F94632D6D8BDF
:1059D0007E8B8F8B988FA3019201698D7A8D8B8D31
:1059E0009C8D0F94632D698F7A8F8B8F9C8FA30171
:1059F00092016D8D7E8D8F8D98A10F94632D6D8F8B
:105A00007E8F8F8F98A3A3019201C701B6010F94D7
:105A1000632D69A37AA38BA39CA380E1EAE4F2E05F
:105A20008E010F5F1F4FD80101900D928A95E1F70B
:105A30000E947AC82B013C0128EC420E511C611CCB
:105A4000711C0DA31EA381E0281A310809F460C05F
:105A50000E947AC88B019C0104191509260937098F
:105A600037FD59C02B013C0128EC420E511C611C32
:105A7000711C80E00F94440F2D893E894F89588D09
:105A800069817A818B819C810F94CD3369837A837C
:105A90008B839C83298D3A8D4B8D5C8D6D817E81AE
:105AA0008F8198850F94CD336D837E838F83988704
:105AB0002D8D3E8D4F8D58A169857A858B859C856E
:105AC0000F94CD3369877A878B879C8729A13AA168
:105AD0004BA15CA16D857E858F8598890F94CD3310
:105AE0006D877E878F87988B750164018E010F5EAD
:105AF0001F4F9E01235F3F4FAE01475F5F4FBE01C7
:105B00006B5F7F4F8DA19EA10E9487BF81119BCFAC
:105B1000750164013CCE0E94F98CAECF8091AE0439
:105B20009091AF04A091B004B091B10480932A0287
:105B300090932B02A0932C02B0932D028091AC0481
:105B40009091AD04909361028093600208958091DA
:105B50002A0290912B02A0912C02B0912D028093E9
:105B6000AE049093AF04A093B004B093B1048091BD
:105B70006002909161029093AD048093AC0484E63E
:105B800090E0909361028093600208958F929F92BB
:105B9000AF92BF92CF92DF92EF92FF92CF93DF93BB
:105BA00080902A0290902B02A0902C02B0902D029F
:105BB000FC01C080D180E280F38020E030E0A901C8
:105BC000C701B6010F94FD2C882341F0C0922A0230
:105BD000D0922B02E0922C02F0922D02C091600232
:105BE000D091610284E690E090936102809360021C
:105BF000C0905A02D0905B02E0905C02F0905D028F
:105C000080E090E0A0E8BFE380935A0290935B02AB
:105C1000A0935C02B0935D020E94DB2A80922A026C
:105C200090922B02A0922C02B0922D02D09361028E
:105C3000C0936002C0925A02D0925B02E0925C0272
:105C4000F0925D02DF91CF91FF90EF90DF90CF90C7
:105C5000BF90AF909F908F9008950F931F93CF9315
:105C6000DF9300D01F92CDB7DEB79C0106E916E0A6
:105C700090E1EAE4F2E0D80101900D929A95E1F703
:105C8000F9012081318142815381F801608571855C
:105C9000828593850F94CD33F80160877187828761
:105CA000938780E090E0A0EAB0E489839A83AB8395
:105CB000BC83CE0101960E94C62D0F900F900F90CD
:105CC0000F90DF91CF911F910F910895AF92BF92E6
:105CD000CF92DF92EF92FF920F931F93CF93DF93B8
:105CE000CDB7DEB764970FB6F894DEBF0FBECDBF59
:105CF0000E94E02087FDAFC08AE50E9476EE8823EF
:105D000009F4BAC040E050E0BA018AE50E94E3EE2F
:105D10007B018C0120915202309153024091540238
:105D20005091550260E070E088EC93E40F94CC331E
:105D30005B016C019701A8010F942D36181614F021
:105D40007501860120E030E0A901B701C8010F9478
:105D50002D36181624F4E12CF12C00E010E0B701E8
:105D6000C8010F943935072E000C880B990B0F943E
:105D7000042D698B7A8B8B8B9C8B20E030E0A90102
:105D80000F94FD2C882321F0CE0141960E942D2EE8
:105D900080E090E0A0EAB1E48D879E87AF87B88B62
:105DA00019861A861B861C868CE40E9428EE88239E
:105DB00009F467C00E94FEED6B017C0120E030E039
:105DC000A901C701B6010F942D3687FF04C0F7FA69
:105DD000F094F7F8F094CD82DE82EF82F88620917D
:105DE000FF10309100112430310574F08091FD10C6
:105DF0009091FE10821B930B97FF03C091958195A4
:105E0000910901E004970CF400E080E00F944F1C2E
:105E1000882359F022E0AE01435F5F4FBE016B5F04
:105E20007F4FCE0109960F946C1B69897A898B8903
:105E30009C898B019C01305809831A832B833C83F6
:105E400020E030E0A9010F94FD2C882321F0CE0141
:105E500001960E942D2E64960FB6F894DEBF0FBEF9
:105E6000CDBFDF91CF911F910F91FF90EF90DF9009
:105E7000CF90BF90AF900895E12CF12C00E211E497
:105E800049CFC090D804D090D904E090DA04F090C3
:105E9000DB0494CFCF92DF92EF92FF920F931F9388
:105EA000C12CD12C76018C0126E532E042E552E08E
:105EB0006EE472E08AE492E00E9487BF1F910F9126
:105EC000FF90EF90DF90CF9008954F925F926F9286
:105ED0007F928F929F92AF92BF92CF92DF92EF927A
:105EE000FF920F931F93CF93DF93CDB7DEB72C971D
:105EF0000FB6F894DEBF0FBECDBF2B013C01298742
:105F00003A874B875C8747015801F601E080F180B2
:105F10000281138120E030E0A901B701C8010F948C
:105F2000FD2C882309F488C05E2D4F2D302F212FA2
:105F3000852F942FA32FB22F89839A83AB83BC83A1
:105F400020E030E0A901B701C8010F94FD2C8111B8
:105F500008C0E0902602F0902702009128021091DC
:105F60002902C701D8018D839E83AF83B887A5011D
:105F70009401609152027091530280915402909169
:105F800055020F94FD2C87FF0CC080925202909214
:105F90005302A0925402B0925502CE0101960E9483
:105FA0004A2F40924A0250924B0260924C027092E9
:105FB0004D0289859A85AB85BC8580934E0290936E
:105FC0004F02A0935002B0935102CE0105960E9459
:105FD0004A2FA50194016091520270915302809161
:105FE0005402909155020F942D36181664F4809245
:105FF000520290925302A0925402B0925502CE01E6
:1060000001960E944A2F0E94B2232C960FB6F89454
:10601000DEBF0FBECDBFDF91CF911F910F91FF90DB
:10602000EF90DF90CF90BF90AF909F908F907F9038
:106030006F905F904F90089550E040E030E820E48A
:1060400077CFCF92DF92EF92FF920F931F936A0167
:10605000E0905202F09053020091540210915502C8
:10606000FB012081318142815381FC01608171817A
:10607000828193810E94652F1F910F91FF90EF9075
:10608000DF90CF900895CF92DF92EF92FF920F931F
:106090001F936B01FC01E080F18002811381EAE42F
:1060A000F2E024813581468157816081718182814E
:1060B00093810E94652F1F910F91FF90EF90DF90C9
:1060C000CF900895AF92BF92CF92DF92EF92FF925E
:1060D0000F931F93CF93DF9300D01F92CDB7DEB7FE
:1060E000FC01E080F18002811381611112C0A09057
:1060F0005202B0905302C0905402D09055029501C4
:10610000A601B701C8010F94FD2C87FF02C07501DD
:10611000860120E030E048EC53E4B701C8010F9459
:10612000FD2C87FD04C0E12CF12C08EC13E4C70121
:10613000D80189839A83AB83BC8366EE72E0CE017B
:1061400001960E9443300F900F900F900F90DF91B7
:10615000CF911F910F91FF90EF90DF90CF90BF9064
:10616000AF900895EF92FF920F931F93CF93DF9319
:106170007C018B010E948DF3CAE4D2E020915A0287
:1061800030915B0240915C0250915D02F7016081A9
:106190007181828193810F94C7342C853D854E8512
:1061A0005F850F94CD336C877D878E879F87C8016D
:1061B0000E944A2FDF91CF911F910F91FF90EF9096
:1061C0000C94B2238F929F92AF92BF92CF92DF92A4
:1061D000EF92FF921F93CF93DF93CDB7DEB7609717
:1061E0000FB6F894DEBF0FBECDBF182F80E00E941F
:1061F000B8284B015C018092A0049092A104A09267
:10620000A204B092A30481E00E94B8286B017C0133
:10621000C092A404D092A504E092A604F092A70430
:1062200082E00E94B8286093A8047093A904809328
:10623000AA049093AB041D861E861F86188A898245
:106240009A82AB82BC82CD82DE82EF82F886698739
:106250007A878B879C8783E00E94B8286D877E872A
:106260008F87988B80914B0B882321F0CE0101966C
:106270000E9450231E3FD9F480E1FE013196AAE42A
:10628000B2E001900D928A95E1F760960FB6F8940E
:10629000DEBF0FBECDBFDF91CF911F91FF90EF907A
:1062A000DF90CF90BF90AF909F908F90089584E043
:1062B000189FF0011124DF01A65BBD4F81E090E043
:1062C0008C0F9D1FE80FF91F4081518162817381FE
:1062D0004D935D936D937C931397D7CF0C948BC0A4
:1062E0000F931F93CF93DF93EC018B0181E00E940A
:1062F00013C469E170E080E090E00E94D9F2B80137
:10630000CE010E944330C0910A0680E00E9413C46F
:1063100010920A0682E00E94E2300E946E31C2FBB7
:10632000CC27C0F981E08C27DF91CF911F910F918D
:106330000895CF93DF93CDB7DEB72C970FB6F894BF
:10634000DEBF0FBECDBF0E9469C10E9476279CE0D0
:10635000E2E2F5E0DE01119601900D929A95E1F7E7
:1063600081110E94BCF2CE0101960E9439912C96B7
:106370000FB6F894DEBF0FBECDBFDF91CF91089569
:106380002F923F924F925F926F927F928F929F9245
:10639000AF92BF92CF92DF92EF92FF920F931F9333
:1063A000CF93DF9300D0CDB7DEB780904A029090B4
:1063B0004B02A0904C02B0904D0240904E02509083
:1063C0004F026090500270905102C0905202D090E3
:1063D0005302E0905402F09055020E94981C0E94D3
:1063E0000B2406E212E180E392E09B838A838AE138
:1063F000282E82E1382E198289810E94E61CC8016C
:106400000E948BE8EA81FB81619371938193919360
:10641000FB83EA83C1010E948BE8EA81FB816087EC
:10642000718782879387F981FF5FF9830C5F1F4F24
:1064300084E0280E311CF330F9F68DEF94E00E94D1
:10644000CEC10E945FF20E948E23A501940160914B
:106450004A0270914B0280914C0290914D020F9430
:10646000FD2C81111CC0A301920160914E0270911C
:106470004F0280915002909151020F94FD2C811196
:106480000EC020915202309153024091540250911B
:106490005502C701B6010F94FD2C8823B9F00F9067
:1064A0000F900F90DF91CF911F910F91FF90EF9080
:1064B000DF90CF90BF90AF909F908F907F906F9024
:1064C0005F904F903F902F900C9499310F900F90C8
:1064D0000F90DF91CF911F910F91FF90EF90DF9080
:1064E000CF90BF90AF909F908F907F906F905F9074
:1064F0004F903F902F90089580919F04659B6EC0B0
:10650000806180939F049091030180919F0491FF8B
:1065100067C0806280939F0480919F044B9B62C000
:10652000846080939F0480919F0490919E049817AB
:1065300009F45AC092E090939D0480939E04809148
:10654000C705811105C08091A606882309F459C0AA
:106550008091140580FF10C08091C80580FD0CC09B
:1065600080919C0484FF08C080910A06806180931A
:106570000A0680E00E94599180911405869580FF5B
:1065800011C08091C805869580FD0CC080919C0447
:1065900085FF08C080910A06806280930A0681E028
:1065A0000E945991809114058695869580FF29C097
:1065B0008091C8058695869580FF23C08091A606A8
:1065C0008823F9F080919C0482FF1BC080910A0609
:1065D000846080930A0682E00C9459918F7E91CF5B
:1065E0008F7D98CF8B7F9DCF80919D04882309F468
:1065F000A6CF815080939D048111A1CF90939C04DC
:106600009ECF08958091C705811104C08091A60690
:10661000882331F062E070E080E090E00C94D9F2E1
:1066200008953F924F925F926F927F928F929F92C6
:10663000AF92BF92CF92DF92EF92FF920F931F9390
:10664000CF93DF9300D01F92CDB7DEB7382E80E016
:1066500090E0A0E2B1E489839A83AB83BC83C090CD
:106660009211D0909311E0909411F090951120E048
:1066700030E0A901C701B6010F94FD2C87FF0CC0C3
:10668000A701960160E070E080E291E40F94CC33C2
:1066900069837A838B839C8360E0CE0101960E949C
:1066A000623040904A0250904B0260904C027090D1
:1066B0004D0280904E0290904F02A0905002B090F8
:1066C0005102332089F10F94BA0D19821A821B826C
:1066D0001C82E0905202F0905302009154021091FB
:1066E0005502CE0101966C01A5019401C301B201CE
:1066F0000E94652F3092A6060E9402330F900F90E1
:106700000F900F90DF91CF911F910F91FF90EF901D
:10671000DF90CF90BF90AF909F908F907F906F90C1
:106720005F904F903F9008950F94770DCECF2F92AA
:106730003F924F925F926F927F928F929F92AF9211
:10674000BF92CF92DF92EF92FF920F931F93CF935E
:10675000DF93CDB7DEB766970FB6F894DEBF0FBEF6
:10676000CDBFF82E282E312CF101ED5BF04FD490E7
:1067700022E0821335C08091A606811103C081E01A
:106780000E9411330F94BA0D811139C18FE39FE03C
:106790000E948BE820E030E0A9010F94FD2C8823B3
:1067A000F9F06D2DDD0C770B880B990B0F94042DF0
:1067B0002B013C018FE39FE00E948BE84B015C01C1
:1067C00020E030E040EA50E40F94FD2C11E087FF18
:1067D0001CC0812C912C90EAA92E90E4B92E15C0F2
:1067E0006D2DDD0C770B880B990B0F94042D2B016D
:1067F0003C01C101880F991F880F991F895C904F38
:106800000E948BE84B015C0110E0A3019201C501DD
:10681000B4010F94632D4B015C016101CC0CDD1CB4
:10682000CC0CDD1CC601855D904F0E948BE8EE24E8
:10683000E394E12620E030E040EC5FE30F94632D29
:10684000A30192010F94632DAB01BC0100E010E0A5
:1068500098018F2D0E94E22820E030E0A901C501B7
:10686000B4010F94FD2CF601E15EF04FFA8BE98B39
:10687000882309F44DC0F2E000E010E020E431E4A8
:10688000FF1619F000E010E09801B501A40170585E
:10689000E12C8F2D0E94E228A5019401C501B401CD
:1068A0000F94CD336B8B7C8B8D8B9E8B22E0F216FD
:1068B000E9F0F101E45EF04F6491611107C00F94BB
:1068C000990B8AEF9EE00E94A9F76AE070E090E0E1
:1068D00080E00F94022D9B01AC0160E070E088E441
:1068E00092E40F94C7348B019C0104C000E010E0D7
:1068F00020EC30E4EE24E3944B895C896D897E8939
:106900008F2D0E94E22832E0F312D0C00F94770D51
:1069100081E090E0A0E0B0E00F2C04C0880F991F48
:10692000AA1FBB1F0A94D2F720914A0B282B209351
:106930004A0B20918604822B8093860489899A8948
:106940000E948BE8F601E65BFD4F608371838283D2
:10695000938382E0F8121AC0209192113091931122
:10696000409194115091951160915202709153028F
:1069700080915402909155020F94CC33609352024F
:10698000709353028093540290935502F601E45E93
:10699000F84F10821182128213828F2D0E94E61C02
:1069A0000E946E31F601E65BFD4F80819181A281EC
:1069B000B381F601EA56F94F80839183A283B383B2
:1069C00092E0F916A9F18CE0E7E9F2E0DE01119618
:1069D00001900D928A95E1F7E1E0F0E0EC0FFD1FE8
:1069E000EC0DFD1D80809180A280B38020E030E01E
:1069F000A901C501B4010F94FD2C81111EC066963A
:106A00000FB6F894DEBF0FBECDBFDF91CF911F91BF
:106A10000F91FF90EF90DF90CF90BF90AF909F903D
:106A20008F907F906F905F904F903F902F90089540
:106A30000E9491E88111E3CFC6CF20E030E0A901A8
:106A4000C501B4010F942D3687FF04C0B7FAB09486
:106A5000B7F8B094F601E65BFD4F6F01A301920118
:106A6000C501B4010F94632D9B01AC01F601608157
:106A70007181828193810F94CC33F601608371839D
:106A800082839383F2E080E090E0A0E4B1E4FF161B
:106A900021F080E090E0A8E4B2E48D879E87AF8784
:106AA000B88BCE010D960E944A2FA9CF81E090E0CD
:106AB000A0E0B0E00F2C04C0880F991FAA1FBB1FD5
:106AC0000A94D2F720914A0B282B20934A0B20914D
:106AD0008604822B8093860489899A890E948BE898
:106AE000F601E65BFD4F60837183828393834ECF13
:106AF0000F931F9380913610813019F50E947AC848
:106B00000091BA041091BB042091BC043091BD04E3
:106B1000601B710B820B930B28EE33E040E050E0DA
:106B20000F9441336091BE047091BF048091C00402
:106B30009091C104620F731F841F951F1F910F91C5
:106B400008956091C2047091C3048091C40490912F
:106B5000C504D6CF109236101092BA041092BB041E
:106B60001092BC041092BD041092C2041092C3048F
:106B70001092C4041092C5041092BE041092BF0477
:106B80001092C0041092C10408958F929F92AF9208
:106B9000BF92CF92DF92EF92FF920F931F93CF930A
:106BA000DF93CDB7DEB72C970FB6F894DEBF0FBEDC
:106BB000CDBF8B0140E050E068E472E44D835E831A
:106BC0006F83788740E050E060EA70E449875A8735
:106BD0006B877C878130B9F1823009F459C020E09D
:106BE00030E040E050E46091520270915302809195
:106BF0005402909155020F94CD334B017C0120E05B
:106C000030E048EC53E40F942D36181634F4812C00
:106C1000912C88ECE82E93E4F92EF801A084B1843D
:106C2000C284D3849401A701B501C6010F942D3607
:106C3000181614F054016701C501D60189839A839F
:106C4000AB83BC8348C0BE01675F7F4FC801089615
:106C50000E944330B8016C5F7F4FAE014B5F5F4FC6
:106C6000C8010E9421300E9499312C960FB6F894E9
:106C7000DEBF0FBECDBFDF91CF911F910F91FF906F
:106C8000EF90DF90CF90BF90AF909F908F9008953E
:106C9000F8012085318542855385609152027091BB
:106CA000530280915402909155020F94CD336B01A1
:106CB0007C0120E030E048EC53E40F94FD2C87FD8C
:106CC00006C0C12CD12C28ECE22E23E4F22EC9827E
:106CD000DA82EB82FC82BE01675F7F4FCE010196B4
:106CE000B7CFCF92DF92EF92FF92CF93DF93C62F71
:106CF000FC01C080D180E280F38020E030E0A90177
:106D0000C701B6010F94FD2C20E030E0A90187FDFA
:106D100014C020E030E048EC52E4C701B6010F9403
:106D20002D3624E630E040E050E0181634F0C7017C
:106D3000B6010F9439359B01AC01C230A0F4D0E00C
:106D4000CD5DD74FAFEFB0E00F94823324E630E053
:106D500040E050E00F9463332F3F310519F010F0FD
:106D60002FEF30E02883DF91CF91FF90EF90DF90FD
:106D7000CF900895E4E3F5E010821182128213822D
:106D800014820C9486C8EF92FF920F931F93CF93B7
:106D9000DF93CDB7DEB78C01EDB6FEB60F944A2C6B
:106DA00001962DB73EB7281B390B0FB6F8943EBF9E
:106DB0000FBE2DBF8DB79EB70196B8010F94432C1F
:106DC0000E9473C40FB6F894FEBE0FBEEDBEDF91F5
:106DD000CF911F910F91FF90EF900895809109013D
:106DE00080FD06C08091431383FB882780F90895B6
:106DF00080E00895CF92DF92EF92FF92FC01C08075
:106E0000D180E280F380663019F510923905109236
:106E10003A0510923B0510923C0510923D050E94E8
:106E20007F8920E030E0A901C701B6010F94FD2C55
:106E300087FF1DC0C12CD12C7601C701B6010F946C
:106E40003A36CB01FF90EF90DF90CF900C947AED23
:106E50000E94BA3620E030E0A901C701B6010F94C4
:106E6000FD2C87FF15C0C12CD12C760121C020E05C
:106E700030E04CE053E4C701B6010F942D361816EC
:106E8000E4F6C12CD12C9CE0E92E93E4F92ED5CF69
:106E900020E030E046E953E4C701B6010F942D36F7
:106EA000181634F4C12CD12C86E9E82E83E4F82E90
:106EB000C701B6010F943A36CB01FF90EF90DF90F7
:106EC000CF900C94822390914A0B977081E0973079
:106ED00009F080E008952091850420FF14C020E887
:106EE0003EE3629FA001639F500D729F500D1124DD
:106EF000CA019695879596958795009731F08A9562
:106F00000000E9F708950C94D9F20895CF93DF9328
:106F10001092090B10929C0B10929E0B10929D0BDD
:106F200010929A0410929904CFEFDFEF80914313EF
:106F300085FD07C00E949875D093C211C093C111FE
:106F4000F5CF8FEF9FEF9093C2118093C111DF9126
:106F5000CF9108958F929F92AF92BF92CF92DF927E
:106F6000EF92FF920F931F93CF93DF937C0121E564
:106F7000E20EF11CD7014C914A3509F0A4C06C0116
:106F8000B2E5CB0ED11CF6013081353A09F09BC039
:106F9000EC01C05BDF4F2881233008F494C08C01E2
:106FA00000561F4FD8014C93E15BFF4F3083319661
:106FB0002083EF54F1093081E05BFF4F308330389C
:106FC000B1F43196AC54B1093C913083E854F109E5
:106FD000AF5ABF4F50E040E02250330B42175307E7
:106FE000CCF4808132968D934F5F5F4FF7CF233083
:106FF00031F5313809F074C0FC01EC55FF4FDC016C
:10700000AC5ABF4F2C9120833196885A9F4FDC0198
:107010008C9180834801B12CA12C888190E002964C
:107020008A159B050CF43FC0F40181914F010E9429
:1070300012F60E9402ACFFEFAF1ABF0AEECF323851
:1070400021F5FC01EC5AFF4F30814181E05BFF4F9D
:10705000408331963083DC01AA55BF4F50E040E0B9
:107060002350330B42175307ACF6FA01EE7FE45A74
:10707000FF4FE80FF91F608171817C9311966C932B
:1070800011974E5F5F4F1296EDCF243019F63338CB
:1070900009F6FC01EC5AFF4F20813181E05BFF4F84
:1070A00030833196B0CF80E5DE011D928A95E9F7F5
:1070B0008AE1F80111928A95E9F78AE5D7018C9364
:1070C00085EAF6018083DF91CF911F910F91FF90A8
:1070D000EF90DF90CF90BF90AF909F908F900895EA
:1070E000323809F097CFADCFCF93DF93D0913610E0
:1070F00082E092E10E94A9F78AE00E9481F78091E4
:10710000B50B873009F449C083E08093B30B81E06D
:107110008093670280E190E09093DA128093D91215
:1071200085E08093CD12C2E8C093D01284E190E153
:10713000A0E0B0E08093D1129093D212A093D3122A
:10714000B093D4128DE792E10E94AA3761E070E01B
:1071500080E090E00E946B3781E09AE59093DA122C
:107160008093D91285E390E09093DC128093DB1238
:1071700087E08093CD12C093D01284E890E0A0E025
:10718000B0E08093D1129093D212A093D312B09317
:10719000D4128DE792E10E94AA3780913610813097
:1071A00089F1823061F50E9478356093BE04709356
:1071B000BF048093C0049093C10481E08093361093
:1071C0000E947AC86093BA047093BB048093BC0495
:1071D0009093BD04D23089F08091B6059091B705A7
:1071E00001969093B7058093B6051092870410928C
:1071F00088041092890410928A0481E004C00E94DD
:10720000AA35DBCF80E0DF91CF9108950E949CAF3B
:107210001092490B109225020E94D8F3882351F056
:107220008091431382FD06C08DE29EE09093990BFE
:107230008093980B61E086E29EE00E94B8F80C947F
:107240007438809136108130C1F582E49EE00E944E
:10725000A9F78AE00E9481F781E09AE59093DA121B
:107260008093D91287E590E09093DC128093DB1233
:1072700087E08093CD1282E88093D01284E890E07A
:10728000A0E0B0E08093D1129093D212A093D312D9
:10729000B093D4128DE792E10E94AA3782E08093E6
:1072A00036100E947AC86093C2047093C30480931E
:1072B000C4049093C50481E0089580E008950F937D
:1072C0001F930E947AC80091B1051091B2052091D8
:1072D000B3053091B405011511052105310509F0FB
:1072E00067C02091AF11222309F45FC0E091AD1176
:1072F00021502093AF1121E02E0F2093AD1130913A
:10730000B011231302C01092AD1124E0E29FF001EE
:107310001124EF54FE4E00811181228133810093AC
:10732000AD051093AE052093AF053093B005600F07
:10733000711F811D911D6093B1057093B2058093FB
:10734000B3059093B4058091AF059091B005892B5A
:1073500061F11FB7F89481E39EE00E94A9F78AE0EB
:107360000E9481F784E096E09093DA128093D9121C
:1073700080EA90E89093DC128093DB1287E08093A0
:10738000CD1282E88093D01280EA90E0A0E0B0E0D5
:107390008093D1129093D212A093D312B093D412AF
:1073A0008DE792E10E94AA371FBF1F910F910895A8
:1073B000601B710B820B930B97FDF7CF40981092D7
:1073C000B1051092B2051092B3051092B405EDCF3D
:1073D0000F931F93CF93DF938C01EB019091AF112B
:1073E0002091B011921305C00E945F390E94F98C60
:1073F000F5CF8091AE1134E0839FF0011124EF545A
:10740000FE4E11830083D383C2839F5F9093AF119D
:107410008F5F281739F08093AE11DF91CF911F91C4
:107420000F9108951092AE11F8CF2F923F924F9284
:107430005F926F927F928F929F92AF92BF92CF9204
:10744000DF92EF92FF920F931F93CF93DF930097FA
:1074500009F0AAC110929E0B10929D0B90939A0472
:1074600080939904BAE0CB2EB0E2DB2EE12CF12C14
:1074700015E002E846015701C4E1D0E01092201265
:1074800010921F121093131200931612809217126B
:1074900090921812A0921912B0921A1283EC91E1F4
:1074A0000E94AA3721972FEF821A920AA20AB20AE3
:1074B000209721F744E1C40ED11CE11CF11C8AE5A0
:1074C000C81680E2D806E104F104A1F6C12CA0E2BE
:1074D000DA2EE12CF12CD5E0C2E8109220121092A5
:1074E0001F12D0931312C0931612C0921712D0928B
:1074F0001812E0921912F0921A1283EC91E10E9494
:10750000AA371092201210921F12D0931312C09318
:107510001612D701C6018C529F4FAF4FBF4F8093B9
:10752000171290931812A0931912B0931A1283ECA9
:1075300091E10E94AA37EFEFCE1ADE0AEE0AFE0AA8
:10754000FAE0CF16F0E2DF06E104F10431F6FEEDD9
:10755000CF2EF0E2DF2EE12CF12CD5E0C2E8109224
:10756000201210921F12D0931312C0931612C092C1
:107570001712D0921812E0921912F0921A1283EC9C
:1075800091E10E94AA372FEFC21AD20AE20AF20A48
:1075900046EEC41640E2D406E104F10401F7CC241F
:1075A000C394E2E1DE2EE12CF12C0AE010E0D5E0FC
:1075B000C2E81093201200931F12D0931312C093AD
:1075C0001612C0921712D0921812E0921912F0926D
:1075D0001A1283EC91E10E94AA37109320120093B3
:1075E0001F12D0931312C0931612D701C6018096B2
:1075F000A11DB11D8093171290931812A093191218
:10760000B0931A1283EC91E10E94AA378FEFC81A47
:10761000D80AE80AF80AE5E0CE16E2E1DE06E1045F
:10762000F10439F600919D0B10919E0B0115110587
:1076300009F0D6C080919C0B882309F4E1C02AE0B0
:1076400030E240E050E065EA73E083EC91E10E94B3
:1076500007ACC1E0D0E003E010E0E0909D0BF090BB
:107660009E0B35E0332E42E8242E44244A94542CB9
:1076700064E0662E712C7FE1C72E74E0D72E8091D6
:107680009D0B90919E0B800F911FE816F90608F054
:10769000D5C0C7010E941EAD882309F481C0809126
:1076A000B11064EA70E1882311F061EB70E1FB0135
:1076B00001900020E9F7CF010197861B970BF4E1B9
:1076C000FC9F9001FD9F300D1124265F3F4D50E03F
:1076D00040E0459710F0FB01128A83EC91E10E9493
:1076E00007ACCE018F5F9D4EB0E0A0E021964E0129
:1076F00024E0880C991C2A95E1F7FDEF8F1AFFE929
:107700009F0AB12CA12C2091431324FF7EC07092BC
:10771000201260921F123092131220921612809340
:10772000171290931812A0931912B0931A1283ECA7
:1077300091E10E94AA37D0922012C0921F1230927B
:107740001312209216128092171290921812A09281
:107750001912B0921A1283EC91E10E94AA37B70174
:107760008EEE9DE00E94C8F98091B11061EB70E14E
:10777000811102C064EA70E18BEE9DE00F948B0BE7
:1077800069E07BE087EE9DE00F948B0B64EA70E18B
:1077900086EE9DE00F948B0B82EE9DE00E94A9F790
:1077A0002FEFE21AF20A6BCF20919D0B30919E0BC6
:1077B000A901415051096091990470919A04681788
:1077C000790738F42C5F3F4F30939E0B20939D0B2D
:1077D00045CE4430510508F43DCE24503109F4CF54
:1077E0000430110569F480919C0B882331F083E00B
:1077F00090E090939E0B80939D0BD0E0C0E02DCF46
:10780000D0E0C0E004E010E028CF109220121092E7
:107810001F12309213122092161280931712909317
:107820001812A0931912B0931A1283EC91E10E94DE
:10783000AA375092201240921F1281CFDF91CF9130
:107840001F910F91FF90EF90DF90CF90BF90AF907E
:107850009F908F907F906F905F904F903F902F9070
:107860000895AF92BF92CF92DF92EF92FF920F9363
:107870001F93CF93DF93EC0184E6C82E80E2D82ECD
:10788000E12CF12C02E8A12C90E2B92E15E0009336
:10789000D012C092D112D092D212E092D312F092B2
:1078A000D412B092DA12A092D9121093CD128DE7B1
:1078B00092E10E94AA378FEFC81AD80AE80AF80A9C
:1078C00088E7C81680E2D806E104F10401F724E64F
:1078D00030E240E050E0BE018DE792E1DF91CF91D0
:1078E0001F910F91FF90EF90DF90CF90BF90AF90DE
:1078F0000C9407AC0F931F93CF93DF938C016F3FD2
:1079000019F41092771060E020917710862F062EE0
:10791000000C990B2817190609F08CF56093771065
:1079200060E080EF9DE00E94B8F8C8010E94A9F7CE
:107930008AE00E9481F7C8010F944A2C800F911FA2
:10794000EC01C01BD10BC034D1053CF00197FC0108
:107950002491207C2038D1F3F3CFDD27AE01B8018C
:1079600087E390E10F946B2CC95CDF4E188287E3AC
:1079700090E1DF91CF911F910F910C94313CDF91F9
:10798000CF911F910F910895DF92EF92FF920F9385
:107990001F93CF93DF93CDB7DEB7CA5AD1090FB685
:1079A000F894DEBF0FBECDBFCF55DF4F18821982CE
:1079B0001A821B82C15AD0408091B2039091B303C6
:1079C000A091B403B091B503CB55DF4F8883998361
:1079D000AA83BB83C55AD04084E690E09093D30439
:1079E0008093D204109203051092020510920405B0
:1079F00022E035E044E050E0BE016B557F4F82ED60
:107A000094E00F94030E8091D2049091D3040296D7
:107A10009093D3048093D204109203051092020530
:107A200081E0C655DF4F8883CA5AD040CE018655C3
:107A30009F4F0E94049D22E035E048E450E060E55D
:107A40007BE082ED94E00F94030E22E035E040E10C
:107A500050E06FEF77E082ED94E00F94030E8AE040
:107A600097EDA3EABCE3CF55DF4F88839983AA83C0
:107A7000BB83C15AD040CE018F559F4F0E94FB9CC3
:107A800088E297E00E94169D8FE092E00E940D9D93
:107A90008BE092E00E94FB9C8091EE079091EF07B3
:107AA000A091F007B091F10789839A83AB83BC83DF
:107AB0008E010F5F1F4FC8010E94FB9CCF55DF4F07
:107AC000188219821A821B82C15AD0407E018DE62B
:107AD000E80EF11C83E0D7018C938983CE018F558A
:107AE0009F4F0E94FB9CC7010E94049DC8010E94F9
:107AF000049D4AE0D42EDA94DD2031F0CE018F557A
:107B00009F4F0E94FB9CF7CF8AE891E10E94169D4F
:107B1000CF55DF4F188219821A821B82C15AD0407A
:107B20003AE0D32EDA94DD2031F0CE018F559F4F0D
:107B30000E94FB9CF7CF85E0D82ED982F701D08236
:107B4000C8010E94049DC7010E94049D22E035E007
:107B500048E050E065EF74E082ED94E00F94030E8E
:107B600022E035E048E050E06DEE74E082ED94E014
:107B70000F94030E22E035E044E650E062EB76E03D
:107B800082ED94E00F94030E19828FEFD7018C934E
:107B9000C8010E940D9DC7010E94049D22E035E0AE
:107BA00044E050E06AEE72E082ED94E00F94030E40
:107BB0008091C9058983C8010E940D9D22E035E0AE
:107BC00040E150E06DED74E082ED94E00F94030E1F
:107BD000198A1A8A1B8A1C8A80E090E0A0E8BFE319
:107BE0008D879E87AF87B88B80910211909103118A
:107BF000A0910411B091051189839A83AB83BC8352
:107C00002CEA35EC47E25EE36091061170910711B2
:107C100080910811909109110F94C7346D837E8370
:107C20008F8398872CEA35EC47E25EE360910A1176
:107C300070910B1180910C1190910D110F94632D87
:107C400069877A878B879C8722E035E044E150E0A2
:107C5000B80182ED94E00F94030E84E190E09A83E2
:107C60008983C8010E94E99C809197109091981097
:107C7000A0919910B0919A1089839A83AB83BC83A9
:107C80002CEA35EC47E25EE360919B1070919C100A
:107C900080919D1090919E100F94C7346D837E83C8
:107CA0008F8398872CEA35EC47E25EE360919F1062
:107CB0007091A0108091A1109091A2100F94632D4B
:107CC00069877A878B879C87C8010E94F29C8CE029
:107CD000E3EAF2E0D80101900D928A95E1F7C8013C
:107CE0000E94F29C1982C8010E94049D8FE790E0D7
:107CF0009A838983C8010E94E99CEFEAF2E0D801E7
:107D000001900D92DA94E1F722E035E045E050E091
:107D1000B80182ED94E00F94030E8091DC04898316
:107D2000C8010E940D9D80E2E4EBF2E0D8010190D1
:107D30000D928A95E1F722E035E040E250E0B8018B
:107D400082ED94E00F94030EF7011082C7010E94A8
:107D50000D9D8BE197E00E940D9D87E197E00E94C9
:107D6000FB9CCF55DF4F188219821A821B82C15AA1
:107D7000D040CE018F559F4F0E94FB9C80E2D801DE
:107D80001D928A95E9F722E035E040E250E0B80123
:107D900082ED94E00F94030EFE01F99688E0DF0176
:107DA0001D928A95E9F744E650E060E070E049836F
:107DB0005A836B837C834D835E836F83788783E0F4
:107DC00090E0A0E0B0E089879A87AB87BC874D87B9
:107DD0005E876F87788B498B5A8B6B8B7C8B8D8BF7
:107DE0009E8BAF8BB88F898F9A8FAB8FBC8F8D8F07
:107DF0009E8FAF8FB8A38EE190E0A0E0B0E089A3A2
:107E00009AA3ABA3BCA38DA39EA3AFA3B8A789A736
:107E10009AA7ABA7BCA78DA79EA7AFA7B8AB89AB06
:107E20009AABABABBCAB8DAB9EABAFABB8AF22E00C
:107E300035E040E450E0B80182ED94E00F94030E89
:107E400090E1D92EF8018D2D11928A95E9F722E063
:107E500035E040E150E0B80182ED94E00F94030E6C
:107E6000D8011D92DA94E9F722E035E040E150E0D4
:107E7000B80182ED94E00F94030ECF55DF4F1882C6
:107E800019821A821B82C15AD040CE018F559F4F52
:107E90000E94FB9C2CE0D22EF8018D2D11928A9528
:107EA000E9F722E035E04CE050E0B80182ED94E0E3
:107EB0000F94030E8CE6D8011D928A95E9F722E013
:107EC00035E04CE650E0B80182ED94E00F94030EEB
:107ED00086EC94E00E94F29C22E035E048E050E01D
:107EE00064ED74E082ED94E00F94030EF7011192BB
:107EF000DA94E9F7C755DF4F1882C95AD04080E0BD
:107F000090E0A0E4B0E4C356DF4F88839983AA834E
:107F1000BB83CD59D040C7010E94169DCE01875525
:107F20009F4F0E94049DCE0183569F4F0E94FB9C51
:107F300080E3D7011D928A95E9F782E392E10E94DE
:107F4000A9F78AE00E9481F722E035E040E350E0A3
:107F5000B70182ED94E00F94030E80910405811126
:107F600028C00091D2041091D30480910205909111
:107F70000305F7019183808384E690E09093D30416
:107F80008093D20422E035E044E050E06EEE72E0EF
:107F900082ED94E00F94030EC7010E94E99C91E0EA
:107FA0000537134009F490E080910405892B8093F4
:107FB000040580910405811105C060E086E692E128
:107FC0000E947A3C86E492E10E94A9F78AE00E942E
:107FD00081F79091040581E08927C655DF4F0FB6E0
:107FE000F894DEBF0FBECDBFDF91CF911F910F91EF
:107FF000FF90EF90DF9008951092490B10922502A8
:108000008091431380648093431361E08EEF9DE081
:108010000E94B8F843E15EE06BE17EE085E00E94FB
:1080200021AE60E085E09EE00C947A3CCF92DF9236
:10803000EF92FF920F931F93CF93DF93CDB7DEB7ED
:108040007C01CDB6DEB60F944A2C01962DB73EB713
:10805000281B390B0FB6F8943EBF0FBE2DBF0DB7CE
:108060001EB70F5F1F4FB701C8010F94432CF801D3
:1080700001900020E9F73197E01BF10B759720F094
:1080800084ED92E0F801848BC8010E94313C0FB668
:10809000F894DEBE0FBECDBEDF91CF911F910F9140
:1080A000FF90EF90DF90CF900895CF93DF9300D0B3
:1080B0001F92CDB7DEB787EB9DE00E94A9F78AE05B
:1080C0000E9481F78091B50B8330D9F119821A8211
:1080D0001B821C8260E0CE0101960E9471361982DB
:1080E0001A821B821C8261E0CE0101960E947136C9
:1080F00081E0809366021092B20B8093670281E068
:108100009AE59093DA128093D91283E390E09093EA
:10811000DC128093DB1287E08093CD1282E880939B
:10812000D01284E890E0A0E0B0E08093D112909368
:10813000D212A093D312B093D4128DE792E10E9491
:10814000AA370F900F900F900F90DF91CF91089565
:10815000CF92DF92EF92FF92CF93C82F809136108B
:108160008150823008F069C00E945540109236104C
:108170000E947AC86093C2047093C3048093C404BD
:108180009093C504C0908704D0908804E09089043F
:10819000F0908A040E947835AB01BC0140938704BB
:1081A000509388046093890470938A048091BA057F
:1081B0009091BB05A091BC05B091BD058C199D099E
:1081C000AE09BF09840F951FA61FB71F8093BA057C
:1081D0009093BB05A093BC05B093BD05C1110AC027
:1081E000C1E00E94F8228C2FCF91FF90EF90DF909A
:1081F000CF9008958091B8059091B905019690931C
:10820000B9058093B8050E947835C090BE05D0901E
:10821000BF05E090C005F090C105C616D706E80678
:10822000F906F0F60E9478356093BE057093BF059D
:108230008093C0059093C105D3CFC0E0D2CF8F9279
:108240009F92AF92BF92CF92DF92EF92FF920F93E5
:108250001F93CF93DF930E9486373AE0C32E30E21C
:10826000D32EE12CF12C15E002E846015701CAE0BB
:10827000D0E01092DA121092D9121093CD1200931E
:10828000D0128092D1129092D212A092D312B092B8
:10829000D4128DE792E10E94AA3721978FEF881AB6
:1082A000980AA80AB80A209721F78AE0C80ED11CBC
:1082B000E11CF11C82EDC81680E2D806E104F1044D
:1082C000A1F6C12C20E2D22EE12CF12CD5E0C2E89F
:1082D0001092DA121092D912D093CD12C093D0120C
:1082E000C092D112D092D212E092D312F092D41254
:1082F0008DE792E10E94AA371092DA121092D912F9
:10830000D093CD12C093D012D701C6018C529F4F8B
:10831000AF4FBF4F8093D1129093D212A093D3123C
:10832000B093D4128DE792E10E94AA378FEFC81A5A
:10833000D80AE80AF80A8AE0C81680E2D806E104FA
:10834000F10431F69EEDC92E90E2D92EE12CF12CEC
:10835000D5E0C2E81092DA121092D912D093CD1261
:10836000C093D012C092D112D092D212E092D31206
:10837000F092D4128DE792E10E94AA378FEFC81ACB
:10838000D80AE80AF80A86EEC81680E2D806E104A0
:10839000F10401F7CC24C39482E1D82EE12CF12C16
:1083A0000AE010E0D5E0C2E81093DA120093D91287
:1083B000D093CD12C093D012C092D112D092D212CB
:1083C000E092D312F092D4128DE792E10E94AA3784
:1083D0001093DA120093D912D093CD12C093D01219
:1083E000D701C6018096A11DB11D8093D112909333
:1083F000D212A093D312B093D4128DE792E10E94CF
:10840000AA378FEFC81AD80AE80AF80A85E1C81611
:1084100082E1D806E104F10439F682E190E090931C
:10842000DA128093D912D093CD12C093D01284E186
:1084300090E1A0E0B0E08093D1129093D212A0938B
:10844000D312B093D4128DE792E1DF91CF911F91B7
:108450000F91FF90EF90DF90CF90BF90AF909F90E3
:108460008F900C94AA374F925F926F927F928F9267
:108470009F92AF92BF92CF92DF92EF92FF920F93B3
:108480001F93CF93DF9300D000D01F921F92CDB7E0
:10849000DEB78091970481110AC480919504909170
:1084A00096049C012F5F3F4F3093960420939504D0
:1084B0008E3E924008F4FBC38091FD109091FE1017
:1084C0009093DA128093D91205E00093CD1212E84E
:1084D0001093D01286E390E1A0E0B0E08093D11237
:1084E0009093D212A093D312B093D4128DE792E15D
:1084F0000E94AA3780919210909193109093DA1273
:108500008093D9120093CD121093D0128CE390E196
:10851000A0E0B0E08093D1129093D212A093D31236
:10852000B093D4128DE792E10E94AA378091FF1098
:10853000909100119093DA128093D9120093CD128A
:108540001093D01284E390E1A0E0B0E08093D112C8
:108550009093D212A093D312B093D4128DE792E1EC
:108560000E94AA3780919410909195109093DA12FE
:108570008093D9120093CD121093D0128AE390E128
:10858000A0E0B0E08093D1129093D212A093D312C6
:10859000B093D4128DE792E10E94AA3781E08093D4
:1085A000970410929604109295048091B50B88233D
:1085B00039F10E94061D811123C0809194048F5FC0
:1085C0008093940480919404853620F01092940452
:1085D0001092B50BE091B50BE150E73008F06AC09E
:1085E0000E2E000CFF0B8827E750FD4B8F4F0D948C
:1085F000C433034352431E454A458B45C345564346
:1086000010929404DFCF0E946337882309F452C08C
:1086100081E08093670289EA9DE00E94A9F78AE0E1
:108620000E9481F780E190E09093DA128093D91252
:1086300085E08093CD1212E81093D01284E190E18E
:10864000A0E0B0E08093D1129093D212A093D31205
:10865000B093D4128DE792E10E94AA3781E09AE5A7
:108660009093DA128093D91286E390E09093DC1213
:108670008093DB1287E08093CD121093D01284E8B0
:1086800090E0A0E0B0E08093D1129093D212A0933A
:10869000D312B093D4128DE792E10E94AA371092C0
:1086A000B50B08C00E946337882321F00E94061D85
:1086B0008823A9F380916702882309F433C7809146
:1086C00098048111C0C284E096E09093DA128093FE
:1086D000D91280EA90E89093DC128093DB1217E0C5
:1086E0001093CD1202E80093D01280EA90E0A0E04F
:1086F000B0E08093D1129093D212A093D312B09392
:10870000D4128DE792E10E94AA3780916202909183
:108710006302A0916402B09165020097A105B105C2
:1087200009F03FC21092DA121092D91215E010939C
:10873000CD120093D0128AE890E1A0E0B0E08093DF
:10874000D1129093D212A093D312B093D4128DE78A
:1087500092E10E94AA3789E090E09093DA12809328
:10876000D9121093CD120093D0128CE890E1A0E0C2
:10877000B0E08093D1129093D212A093D312B09311
:10878000D4128DE792E10E94AA3780916202909103
:108790006302A0916402B09165020097F1E0AF0717
:1087A000B10508F441C2B093DA12A093D9129093A4
:1087B000DC128093DB1287E08093CD1282E88093F5
:1087C000D01288E890E1A0E0B0E08093D1129093BD
:1087D000D212A093D312B093D4128DE792E10E94EB
:1087E000AA378091620290916302A0916402B091D5
:1087F0006502BA2FA92F982F8827009721E0A2079A
:10880000B10508F417C2B093DA12A093D91290936D
:10881000DC128093DB1287E08093CD1212E8109374
:10882000D01281EA90E0A0E0B0E08093D112909362
:10883000D212A093D312B093D4128DE792E10E948A
:10884000AA3780914B0B882309F4FAC183E090E0AA
:108850009093DA128093D91285E08093CD12109311
:10886000D01285E490E1A0E0B0E08093D112909323
:10887000D212A093D312B093D4128DE792E10E944A
:10888000AA3780919804875E809398042091980479
:10889000822F90E0253608F021C29093DA1280935F
:1088A000D91285E08093CD1282E88093D01280E0C7
:1088B00090E1A0E0B0E08093D1129093D212A09307
:1088C000D312B093D4128DE792E10E94AA370E948E
:1088D000061D811114C20E94D8F3811105C0909128
:1088E000850491FD0E94061D9091850480FB91F9FD
:1088F0009093850491FD03C28091431382FDFFC1D3
:10890000809136108150823008F4F9C16091941042
:1089100070919510072E000C880B990B0F94042D65
:108920006B017C0120E030E0A9010F94FD2C88232D
:1089300009F4BBC66091921070919310072E000C41
:10894000880B990B0F94042D2B013C0120E030E0A3
:1089500040E050E4C701B6010F94CC33A30192016B
:108960000F942D3618160CF4C2C66091FD1070914C
:10897000FE10072E000C880B990B0F94042D6D83AD
:108980007E838F8398876091FF1070910011072E6E
:10899000000C880B990B0F94042D4B015C0120E017
:1089A00030E040E251E40F94CC332D813E814F8181
:1089B00058850F942D3618160CF499C620E030E037
:1089C00040E050E4C701B6010F94CD33A3019201FA
:1089D0000F94FD2C87FD10C020E030E040E251E410
:1089E000C501B4010F94CD332D813E814F8158854F
:1089F0000F94FD2C87FF6AC684E190E09093DA1211
:108A00008093D91285E08093CD1282E88093D012B2
:108A100084E190E1A0E0B0E08093D1129093D21273
:108A2000A093D312B093D4128DE792E10E94AA379B
:108A30008091B30B81117CC682E07AC68BE99DE000
:108A40000E94A9F78AE00E9481F781E09AE590935D
:108A5000DA128093D91280E490E09093DC12809334
:108A6000DB1217E01093CD1282E88093D01284E8D5
:108A700090E0A0E0B0E08093D1129093D212A09346
:108A8000D312B093D4128DE792E10E94AA371093CB
:108A9000B50B10CE8091A20B882309F40BCE0E9457
:108AA0006337882309F406CE0E94061D811102CE89
:108AB0008DE89DE00E94A9F78AE00E9481F78091ED
:108AC000A30B90E0B0E0A0E0895B9F4FAE4FB54AAA
:108AD00021E03AE53093DA122093D9129093DC1218
:108AE0008093DB1287E08093CD1282E88093D012CE
:108AF00084E890E0A0E0B0E08093D1129093D2128D
:108B0000A093D312B093D4128DE792E10E94AA37BA
:108B10001092A20BC4CD0E946337882309F4CACDFA
:108B20000E94061D8111C6CD81E0809367021092DC
:108B3000B50B8FE79DE00E94A9F78AE00E9481F7BC
:108B400081E09AE59093DA128093D9128EE490E056
:108B50009093DC128093DB1287E08093CD1282E841
:108B60008093D01284E890E0A0E0B0E08093D1122E
:108B70009093D212A093D312B093D4128DE792E1C6
:108B80000E94AA3797CD0E94061D811193CD1982AC
:108B90001A821B821C8262E0CE0101960E94E9BF0C
:108BA0007ECD0196A11DB11D35E0B695A79597958F
:108BB00087953A95D1F70197A109B1090097E1E0AE
:108BC000AE07B10548F1B093DA12A093D912909391
:108BD000DC128093DB121093CD1212E81093D012A6
:108BE0008AE890E1A0E0B0E08093D1129093D21295
:108BF000A093D312B093D4128DE792E10E94AA37CA
:108C000088E090E09093DA128093D91285E0809307
:108C1000CD121093D012A9CD9093DA128093D9126D
:108C200085E08093CD12D9CF9093DA128093D91238
:108C300085E0C2CD9093DA128093D91285E0ECCD15
:108C400082E090E005CE8A3F08F020CE8EEF809340
:108C500098048EE69DE00E94A9F78AE00E9481F7C1
:108C600081E08093670281E09AE59093DA12809325
:108C7000D9128DE290E09093DC128093DB1287E0B2
:108C80008093CD1282E88093D01284E890E0A0E037
:108C9000B0E08093D1129093D212A093D312B093EC
:108CA000D4128DE792E10E94AA3710929704289679
:108CB0000FB6F894DEBF0FBECDBFDF91CF911F91ED
:108CC0000F91FF90EF90DF90CF90BF90AF909F906B
:108CD0008F907F906F905F904F9008958456910988
:108CE0009093DA128093D91285E08093CD1282E8B6
:108CF0008093D01281E090E1A0E0B0E0DCCD8CE088
:108D000090E09093DA128093D91215E01093CD126F
:108D100082E88093D01284E190E1A0E0B0E08093FB
:108D2000D1129093D212A093D312B093D4128DE7A4
:108D300092E10E94AA370E94783520E13EE040E0AF
:108D400050E00F9441332115310581E0480751056A
:108D500008F470C05093DA124093D9123093DC12A9
:108D60002093DB1287E08093CD1212E81093D0128B
:108D700080E190E1A0E0B0E08093D1129093D21214
:108D8000A093D312B093D4128DE792E10E94AA3738
:108D90000E94783520E13EE040E050E00F944133FE
:108DA0002CE330E040E050E00F9441333093DA128E
:108DB0002093D91205E00093CD121093D01282E1D6
:108DC00090E1A0E0B0E08093D1129093D212A093F2
:108DD000D312B093D4128DE792E10E94AA370E9479
:108DE000761F882309F45CC48F5F80939304E82E78
:108DF000F12C833330F5EE0CFF1CF092DA12E09286
:108E0000D9120093CD121093D0128EE090E1A0E021
:108E1000B0E08093D1129093D212A093D312B0936A
:108E2000D4128DE792E10E94AA371092DA121092C2
:108E3000D9122BC03093DA122093D9121093CD128D
:108E400094CF84E690E09093DA128093D912009345
:108E5000CD121093D0128EE090E1A0E0B0E08093AC
:108E6000D1129093D212A093D312B093D4128DE763
:108E700092E10E94AA37A2E3EA1AA0E8FA0AEE0CED
:108E8000FF1CF092DA12E092D9120093CD121093E7
:108E9000D0128FE090E1A0E0B0E08093D1129093E7
:108EA000D212A093D312B093D4128DE792E10E9414
:108EB000AA370E94761F90E09093DA128093D9121D
:108EC00085E08093CD1282E88093D01286E190E114
:108ED000A0E0B0E08093D1129093D212A093D3126D
:108EE000B093D4128DE792E10E94AA3720E030E0DF
:108EF000A9016091921170919311809194119091B8
:108F000095110F94CD3320E030E048EC52E40F94FB
:108F1000632D0F9439357093DA126093D91205E0FE
:108F20000093CD1212E81093D01286E290E1A0E0F7
:108F3000B0E08093D1129093D212A093D312B09349
:108F4000D4128DE792E10E94AA3780915E0290913F
:108F50005F029093DA128093D9120093CD1210938E
:108F6000D01280E093E1A0E0B0E08093D112909322
:108F7000D212A093D312B093D4128DE792E10E9443
:108F8000AA3720E030E040E251E46091640B709138
:108F9000650B8091660B9091670B0F94632D0F9476
:108FA00040357093DA126093D9120093CD1210936A
:108FB000D01282E492E1A0E0B0E08093D1129093CD
:108FC000D212A093D312B093D4128DE792E10E94F3
:108FD000AA3720E030E040E251E46091680B7091E4
:108FE000690B80916A0B90916B0B0F94632D0F941A
:108FF00040357093DA126093D9120093CD1210931A
:10900000D01286E492E1A0E0B0E08093D112909378
:10901000D212A093D312B093D4128DE792E10E94A2
:10902000AA3720E030E040E251E460916C0B70918F
:109030006D0B80916E0B90916F0B0F94632D0F94BD
:1090400040357093DA126093D9120093CD121093C9
:10905000D0128AE492E1A0E0B0E08093D112909324
:10906000D212A093D312B093D4128DE792E10E9452
:10907000AA3720E030E040E251E46091700B70913B
:10908000710B8091720B9091730B0F94632D0F9461
:1090900040357093DA126093D9120093CD12109379
:1090A000D0128EE492E1A0E0B0E08093D1129093D0
:1090B000D212A093D312B093D4128DE792E10E9402
:1090C000AA3720E030E048EC52E460918A117091B8
:1090D0008B1180918C1190918D110F94632D0F94B1
:1090E00039357093DA126093D9120093CD12109330
:1090F000D01286E392E1A0E0B0E08093D112909389
:10910000D212A093D312B093D4128DE792E10E94B1
:10911000AA3720E030E048EC52E460918E11709163
:109120008F1180919011909191110F94632D0F9454
:1091300039357093DA126093D9120093CD121093DF
:10914000D0128AE392E1A0E0B0E08093D112909334
:10915000D212A093D312B093D4128DE792E10E9461
:10916000AA3780916E0290916F029093DA128093E9
:10917000D9120093CD121093D01282E592E1A0E0B3
:10918000B0E08093D1129093D212A093D312B093F7
:10919000D4128DE792E10E94AA3780916C029091DF
:1091A0006D029093DA128093D9120093CD1210932E
:1091B000D01284E592E1A0E0B0E08093D1129093C8
:1091C000D212A093D312B093D4128DE792E10E94F1
:1091D000AA3720E030E040E251E460910211709142
:1091E000031180910411909105110F94632D0F9438
:1091F00040357093DA126093D9120093CD12109318
:10920000D01286E592E1A0E0B0E08093D112909375
:10921000D212A093D312B093D4128DE792E10E94A0
:10922000AA372CEA35EC47E25EE3609106117091B3
:10923000071180910811909109110F94C73420E013
:1092400030E040E251E40F94632D0F944035709369
:10925000DA126093D9120093CD121093D0128AE5DE
:1092600092E1A0E0B0E08093D1129093D212A0934B
:10927000D312B093D4128DE792E10E94AA372CEA60
:1092800035EC47E25EE360910A1170910B11809119
:109290000C1190910D110F94632D20E030E040E20D
:1092A00051E40F94632D0F9440357093DA1260935C
:1092B000D9120093CD121093D0128EE592E1A0E066
:1092C000B0E08093D1129093D212A093D312B093B6
:1092D000D4128DE792E10E94AA3720E030E040E20C
:1092E00051E460919710709198108091991090912D
:1092F0009A100F94632D0F9440357093DA12609397
:10930000D9120093CD121093D01282E692E1A0E020
:10931000B0E08093D1129093D212A093D312B09365
:10932000D4128DE792E10E94AA372CEA35EC47E28D
:109330005EE360919B1070919C1080919D109091C4
:109340009E100F94C73420E030E040E251E40F94C7
:10935000632D0F9440357093DA126093D912009305
:10936000CD121093D01286E692E1A0E0B0E0809397
:10937000D1129093D212A093D312B093D4128DE74E
:1093800092E10E94AA372CEA35EC47E25EE3609155
:109390009F107091A0108091A1109091A2100F9435
:1093A000632D20E030E040E251E40F94632D0F94F0
:1093B00040357093DA126093D9120093CD12109356
:1093C000D0128AE692E1A0E0B0E08093D1129093AF
:1093D000D212A093D312B093D4128DE792E10E94DF
:1093E000AA378091AC0B811105C08091AE0B882308
:1093F00009F46DC06091FD107091FE10072E000CF5
:10940000880B990B0F94042D20E030E048EC52E4D7
:109410000F94632D6B017C016091FF10709100111E
:10942000072E000C880B990B0F94042D9B01AC01A7
:10943000C701B6010F94C7340F94403565367105E6
:1094400010F064E670E07093DA126093D91205E0D0
:109450000093CD1212E81093D01284E290E1A0E0C4
:10946000B0E08093D1129093D212A093D312B09314
:10947000D4128DE792E10E94AA376091FD1070919D
:10948000FE10072E000C880B990B0F94042D6B0116
:109490007C0120E030E04AE253E40F942D361816A8
:1094A00024F48091AC0B811146C16091FF10709142
:1094B0000011072E000C880B990B0F94042D9B01B3
:1094C000AC01C701B6010F942D3687FFAFC1809163
:1094D000A20B882339F18091A10B91E0980F909312
:1094E000A10B90E09093DA128093D91285E08093DB
:1094F000CD1282E88093D01282E490E1A0E0B0E047
:109500008093D1129093D212A093D312B093D4121D
:109510008DE792E10E94AA378091A10B8A3010F06A
:109520001092A10B0E94EE36882309F4B5C1609118
:109530009A0B70919B0BEE24E394F12C611571054D
:10954000A9F090E080E00F94022D20E030E040E8A8
:109550005EE30F94632D0F94AB3420E030E040E8DD
:109560005FE30F94CD330F9440357B0101E010E0B1
:1095700080919C0B811102C010E000E08091C1112C
:109580009091C2118F3F980711F40E948E7E9093A4
:10959000C2118093C111080F191FB80190E080E03B
:1095A0000F94022D20E030E040E85EE30F94632D3D
:1095B0000F94AB344B015C01F092DA12E092D912B5
:1095C00005E00093CD1212E81093D01280E193E1F0
:1095D000A0E0B0E08093D1129093D212A093D31266
:1095E000B093D4128DE792E10E94AA37C501B4016D
:1095F0000F9440357093DA126093D9120093CD1214
:109600001093D01282E193E1A0E0B0E08093D112F8
:109610009093D212A093D312B093D4128DE792E11B
:109620000E94AA370DE113E1AAE1FA2E80914304CA
:10963000909144042091910430919204891B8F737E
:1096400009F449C12A3131050CF0DBC19091430482
:10965000809144044FEF5FEF981749F0E82FF0E056
:10966000ED5BFB4F42818F5F8F7380934404F90160
:10967000E35EFC4E408380911D138A3509F0B3C12F
:1096800062E070E080E090E00E946B37809191048E
:109690009091920401969093920480939104C6CF86
:1096A0001092DA121092D912ACCB6091FF10709127
:1096B0000011072E000C880B990B0F94042D20E04D
:1096C00030E0A9010F94FD2C811134C98CE090E0A9
:1096D0009093DA128093D91285E08093CD1282E8BC
:1096E0008093D01284E190E1A0E0B0E0F3CB8DE074
:1096F00090E09093DA128093D91285E08093CD1296
:1097000082E88093D01284E190E1A0E0B0E0809301
:10971000D1129093D212A093D312B093D4128DE7AA
:1097200092E10E94AA378091B30B811101C081E0C0
:109730008093B30BDBCB1092AC0B20E030E040E227
:1097400051E46091A40B7091A50B8091A60B9091B0
:10975000A70B0F94632D0F9439357093DA12609331
:10976000D9120093CD121093D01284E590E1A0E0BD
:10977000B0E08093D1129093D212A093D312B09301
:10978000D4128DE792E10E94AA3720E030E040E257
:1097900051E46091A80B7091A90B8091AA0B909154
:1097A000AB0B0F94632D0F9439357093DA126093DD
:1097B000D9120093CD121093D01288E590E1A0E069
:1097C000B0E08093D1129093D212A093D312B093B1
:1097D000D4128DE792E10E94AA378DE49DE00E94A9
:1097E000A9F78AE00E9481F781E09AE59093DA1266
:1097F0008093D91281E490E09093DC128093DB1285
:1098000087E08093CD121093D01284E890E0A0E01E
:10981000B0E08093D1129093D212A093D312B09360
:10982000D4128DE792E10E94AA3751CE6091AE0B1F
:10983000662309F44CCE062E000C770B84E39DE0E2
:109840000E94FCF98AE00E9481F71092AE0B84E03E
:1098500090E09093DA128093D91285E08093CD1234
:1098600012E81093D0128EE890E1A0E0B0E080936F
:10987000D1129093D212A093D312B093D4128DE749
:1098800092E10E94AA3781E09AE59093DA128093E0
:10989000D91283E590E0B0CF1092DA121092D9126B
:1098A00005E00093CD1212E81093D01280E193E10D
:1098B000A0E0B0E08093D1129093D212A093D31283
:1098C000B093D4128DE792E10E94AA371092DA1277
:1098D0001092D91293CE121613060CF492C08091F6
:1098E000811290918212A0918312B09184128C34D3
:1098F000E0E19E07A105B10509F4D7C98A3490417A
:10990000A105B10509F4D1C920E030E040E251E4FD
:1099100060914A0270914B0280914C0290914D02ED
:109920000F94632D0F9439357093DA126093D91226
:1099300005E00093CD1212E81093D01288E490E174
:10994000A0E0B0E08093D1129093D212A093D312F2
:10995000B093D4128DE792E10E94AA3720E030E064
:1099600040E251E460914E0270914F0280915002AA
:10997000909151020F94632D0F9439357093DA1240
:109980006093D9120093CD121093D0128AE490E123
:10999000A0E0B0E08093D1129093D212A093D312A2
:1099A000B093D4128DE792E10E94AA3720E030E014
:1099B00040E251E46091520270915302809154024E
:1099C000909155020F94632D0F9439357093DA12EC
:1099D0006093D9120093CD121093D0128CE490E1D1
:1099E000A0E0B0E056C9121613060CF01FCEF80125
:1099F0002F2D11922A95E9F710929204109291045A
:109A000015CE90917E1280911D13981321C09091D4
:109A10007F1280911E1398131BC023303105C4F0B0
:109A200090911F1390937D12809120138093801248
:109A30009330D1F4982F9D7F9038B1F490912113F9
:109A40009F3409F059C0909122139B3409F054C0FF
:109A5000EDE1F3E18AE1DF011D928A95E9F71092C9
:109A60009204109291043BCF833809F045C0809155
:109A7000211390912213982789279827B0E0A0E01E
:109A80008093811290938212A0938312B0938412D8
:109A9000C0902313D12CF12CE12CC0928512D092CE
:109AA0008612E0928712F092881224E233E140E0BD
:109AB00050E0BA014C155D056E057F0508F04AC0FF
:109AC000DB01CA01B695A795979587950696880FED
:109AD000991FFC01E358FD4ED9018C9111969C9180
:109AE000892798278927918380834E5F5F4F6F4F27
:109AF0007F4F2E5F3F4FDECF813861F5809121137C
:109B000090E0B0E0A0E08093811290938212A09345
:109B10008312B093841280912213482F50E070E09A
:109B200060E0409385125093861260938712709381
:109B30008812A3E2B3E1E9E8F2E190E030E020E04E
:109B40008217930739F04D9150E0419351932F5F65
:109B50003F4FF6CFEDE1F3E18AE1DF011D928A95F7
:109B6000E9F710929204109291040E942AC9B7CE8C
:109B70006F927F928F929F92AF92BF92CF92DF921D
:109B8000EF92FF920F931F93CF93DF93CDB7DEB782
:109B900064970FB6F894DEBF0FBECDBF1092D00011
:109BA0008091D00082608093D0001092D50080E137
:109BB0008093D4008091D10080618093D100809106
:109BC000D10088608093D1008091D100806880931B
:109BD000D1008091D1008F7D8093D1008AE5809360
:109BE000CE1280937E1285EA8093CF1280937F12EB
:109BF000EDE1F3E18AE1DF011D928A95E9F78091B9
:109C0000B10B882309F474C283E090E09093DA12D8
:109C10008093D91285E08093CD1282E88093D01290
:109C20008FE190E1A0E0B0E08093D1129093D21246
:109C3000A093D312B093D4128DE792E10E94AA3779
:109C400084E690E09093DA128093D91205E00093B5
:109C5000CD1212E81093D01286E090E1A0E0B0E0BF
:109C60008093D1129093D212A093D312B093D412B6
:109C70008DE792E10E94AA378BE090E09093DA1290
:109C80008093D9120093CD121093D01280E092E10C
:109C9000A0E0B0E08093D1129093D212A093D3129F
:109CA000B093D4128DE792E10E94AA371092DA1293
:109CB0001092D9120093CD121093D01284E390E148
:109CC000A0E0B0E08093D1129093D212A093D3126F
:109CD000B093D4128DE792E10E94AA371092DA1263
:109CE0001092D9120093CD121093D0128AE390E112
:109CF000A0E0B0E08093D1129093D212A093D3123F
:109D0000B093D4128DE792E10E94AA378091FD10A2
:109D10009091FE109093DA128093D9120093CD1295
:109D20001093D01286E390E1A0E0B0E08093D112CE
:109D30009093D212A093D312B093D4128DE792E1F4
:109D40000E94AA3780919210909193109093DA120A
:109D50008093D9120093CD121093D0128CE390E12E
:109D6000A0E0B0E08093D1129093D212A093D312CE
:109D7000B093D4128DE792E10E94AA3782E090E07E
:109D80009093DA128093D9120093CD121093D012CF
:109D90008EE190E1A0E0B0E08093D1129093D212D6
:109DA000A093D312B093D4128DE792E10E94AA3708
:109DB00081E08093660270E6C72E70E1D72EE12C19
:109DC000F12C1092DA121092D9120093CD12109346
:109DD000D012C092D112D092D212E092D312F0924D
:109DE000D4128DE792E10E94AA37BFEFCB1ADB0AAB
:109DF000EB0AFB0AE4E7CE16E0E1DE06E104F1043B
:109E000001F7CE0101967C0184E1D7011D928A956C
:109E1000E9F781E08F9390E99F938F9390E69F936A
:109E20008F9388E68F9386EB93E09F938F93FF92B7
:109E3000EF920F94553720E630E140E050E063ECBC
:109E400073E08DE792E10E9407AC2AE630E140E042
:109E500050E060ED73E08DE792E10E9407AC24E7EB
:109E600030E140E050E0B7018DE792E10E9407AC9D
:109E70002EE730E140E050E06CED73E08DE792E1D9
:109E80000E9407AC1092DA121092D9120093CD12F0
:109E90001093D0128EE090E1A0E0B0E08093D11258
:109EA0009093D212A093D312B093D4128DE792E183
:109EB0000E94AA371092DA121092D9120093CD1292
:109EC0001093D0128FE090E1A0E0B0E08093D11227
:109ED0009093D212A093D312B093D4128DE792E153
:109EE0000E94AA370FB6F894DEBF0FBECDBF4AE07E
:109EF000C42E40E2D42EE12CF12C55E0752E62E800
:109F0000662E460157010AE010E01092DA12109214
:109F1000D9127092CD126092D0128092D11290928A
:109F2000D212A092D312B092D4128DE792E10E9485
:109F3000AA3701501109FFEF8F1A9F0AAF0ABF0A13
:109F40000115110511F78AE0C80ED11CE11CF11CA6
:109F500092EDC91690E2D906E104F10491F6C12C04
:109F600030E2D32EE12CF12C05E012E81092DA1247
:109F70001092D9120093CD121093D012C092D11228
:109F8000D092D212E092D312F092D4128DE792E1E5
:109F90000E94AA371092DA121092D9120093CD12B1
:109FA0001093D012D701C6018C529F4FAF4FBF4FB5
:109FB0008093D1129093D212A093D312B093D41263
:109FC0008DE792E10E94AA37AFEFCA1ADA0AEA0ACD
:109FD000FA0ABAE0CB16B0E2DB06E104F10431F68E
:109FE0002EEDC22E20E2D22EE12CF12C05E012E85B
:109FF0001092DA121092D9120093CD121093D0124F
:10A00000C092D112D092D212E092D312F092D41216
:10A010008DE792E10E94AA37EFEFCE1ADE0AEE0A30
:10A02000FE0AF6EECF16F0E2DF06E104F10401F7D6
:10A03000CC24C39482E1D82EE12CF12C9AE0A92EF5
:10A04000B12C05E012E8B092DA12A092D912009376
:10A05000CD121093D012C092D112D092D212E092AF
:10A06000D312F092D4128DE792E10E94AA37B092F7
:10A07000DA12A092D9120093CD121093D012D70108
:10A08000C6018096A11DB11D8093D1129093D2126A
:10A09000A093D312B093D4128DE792E10E94AA3715
:10A0A0008FEFC81AD80AE80AF80A95E1C91692E1B2
:10A0B000D906E104F10439F68DE19DE00E94A9F78B
:10A0C0008AE00E9481F764960FB6F894DEBF0FBE57
:10A0D000CDBFDF91CF911F910F91FF90EF90DF9057
:10A0E000CF90BF90AF909F908F907F906F9008958A
:10A0F00082E090E08BCD0E94B84D1092980481E0F0
:10A10000809367028FEC9DE00E94A9F78AE00C948F
:10A1100081F7AB01BC0140933F1350934013609310
:10A1200041137093421387EA94E10C94377ACF93EA
:10A13000DF93DB01F9019C919130C1F0943080F004
:10A1400094509C938830D1F480819181009771F074
:10A15000019791838083480F591FEA01188206C036
:10A160008C3539F49C5F9C93943041F4DF91CF910E
:10A1700008958B3339F781E08C93F8CF20813181BA
:10A18000B9016F5F7F4F71836083420F531FEA01F4
:10A190008883808191818F3591056CF7E7CF0F938C
:10A1A0001F9381E000913F131091401320914113C0
:10A1B0003091421340913B1350913C1360913D13F9
:10A1C00070913E13041715072607370708F480E03F
:10A1D0001F910F9108954F925F926F927F928F928D
:10A1E0009F92AF92BF92CF92DF92EF92FF920F9326
:10A1F0001F93CF931092900410928F042FE320931B
:10A200008E0410928D0410928C0410928B04109284
:10A210003E0410923F0410924004109241049C01AD
:10A22000F90190812F5F3F4F9032D1F39E34C9F4F2
:10A23000818190ED980F9A3020F08D3211F08B32A1
:10A2400081F432969F012F5F3F4F808180538A3087
:10A2500008F47EC09F012F5F3F4F8081803209F458
:10A2600079C0F093A906E093A8068F010F5F1F4FF6
:10A27000C0816AE270E0C8010F941B37009731F08B
:10A28000FC01319780818032E1F31182CD3429F0D5
:10A29000C43519F0C73409F04BC0F80180810F5F55
:10A2A0001F4F8032D1F380538A3008F041C0C093F1
:10A2B0008E0490E080E04AE0DF011196489F900113
:10A2C000499F300D1124C901C0972081820F911D33
:10A2D00027FD9A95218130ED320F3A30E8F19093C5
:10A2E0008D0480938C042E3261F4329630E04AE083
:10A2F000DF0131962C9150ED520F5A3078F13093A6
:10A300008B049D01D9012F5F3F4F4C914032D1F317
:10A31000CD34A1F58E31910539F030F587319105B5
:10A3200019F08C31910551F5B0939004A0938F04EE
:10A33000CF911F910F91FF90EF90DF90CF90BF9042
:10A34000AF909F908F907F906F905F904F90089507
:10A35000F90178CFF9017ECFFD01AECF349F200DFA
:10A36000112430ED320FC4CF8537910538F087378F
:10A370009105D0F2803A23E09207B1F25091A806FD
:10A3800070E060E0C12CD12C7601C394FD013196C0
:10A390004C91442309F492C04132A1F4CD3491F49C
:10A3A0008032910579F4F0939004E0938F0463E296
:10A3B00070E0CF010F941B37009709F4B9CFFC016F
:10A3C0001082B6CF41544A3108F073C0DF012D919D
:10A3D000203209F459C030ED320F3A3008F465C02C
:10A3E0002E3209F053C0218120532A3008F45DC079
:10A3F00030E020E06115710519F4BF016150710969
:10A40000A42FB0E02601370104C0440C551C661C83
:10A41000771C4A95D2F780903E0490903F04A0901C
:10A420004004B090410484289528A628B72880923B
:10A430003E0490923F04A0924004B0924104211542
:10A440003105A9F1251BAC5DBB4F2C932081215414
:10A45000DF012A3108F49ACFDF012191222309F488
:10A4600095CF30ED320F3A30B8F333ED320F323052
:10A4700098F32B3289F39D012F5F3F4F4C9140326F
:10A4800009F084CFD901F7CFFD01A0CF2D3219F00B
:10A490002B3209F0ADCF218130ED320F3A3028F068
:10A4A0002E3209F0A5CF22819FCF9F01A9CF20E0B6
:10A4B000CACF6115710551F6BD01C8CF70939004E4
:10A4C00060938F0435CFCF93DF93EC01899188237C
:10A4D00019F00E9481F7FACF8DE00E9481F78AE09F
:10A4E000DF91CF910C9481F7EF92FF920F931F931E
:10A4F000CF93DF93CDB7DEB762970FB6F894DEBF88
:10A500000FBECDBF0E940D2A882309F43FC04AEF39
:10A5100053E082FF02C04FEE53E02AEF33E081FFA9
:10A5200002C021EF33E080FD2EC08AEF93E05F93FD
:10A530004F933F932F939F938F9388EE9EE09F932B
:10A540008F938E010F5F1F4F1F930F930F94942CC7
:10A550000F94990BC8010E946352C8010E9464AF16
:10A560000FB6F894DEBF0FBECDBF81E062960FB686
:10A57000F894DEBF0FBECDBFDF91CF911F910F9139
:10A58000FF90EF90089583EF93E0D1CF80E0EECF7E
:10A59000AF92BF92CF92DF92EF92FF920F931F93F1
:10A5A000CF93DF93CDB7DEB7E6970FB6F894DEBF53
:10A5B0000FBECDBF00918F0410919004F80101905F
:10A5C0000020E9F731976F01C01AD10AF801CF01D5
:10A5D000801B910B8C159D053CF481918F32B9F74E
:10A5E000DF0111971C92F3CF8BE1E3E6F3E1DE018B
:10A5F0005C9601900D928A95E1F7F12CE12CEC1418
:10A60000FD040CF05DC0F801EE0DFF1D808181118D
:10A6100003C08FEFE81AF80A5801AE0CBF1CF50111
:10A620008081882309F44CC0FFEFEF1AFF0AF8017C
:10A63000EE0DFF1D7F01E01AF10A81918111FACF21
:10A64000CE014C960E94897E8BE1FE017C96DE0154
:10A65000119601900D928A95E1F7B501CE01019610
:10A660000E949776CE0101960E94C9EF8FE20E9468
:10A6700081F78091B11081113BC085EF93E00E947A
:10A68000F6798091431384FF1BC019821C8221E05C
:10A69000A501BE01645E7F4FCE0101960E94CB8072
:10A6A000811129C08AE00E9481F70F94990BB501AE
:10A6B0008DEC9CE00F948B0BCE0101960E94C9EFAC
:10A6C0008AE00E9481F7CE014C960E94C9EFE6967F
:10A6D0000FB6F894DEBF0FBECDBFDF91CF911F91B3
:10A6E0000F91FF90EF90DF90CF90BF90AF900895C3
:10A6F00081EB90E1C4CFCE014C960E94F87D8BE1B6
:10A70000FE013196DE015C9601900D928A95E1F78B
:10A71000CE0101960E94C9EF72CF3F924F925F9295
:10A720006F927F928F929F92AF92BF92CF92DF9261
:10A73000EF92FF920F931F93CF93DF93809140048A
:10A7400087FD38C0809141048370A1F5C0919611B6
:10A75000D0919711488159816A817B818EEB9CE071
:10A760000E94DAF94C815D816E817F8186EF94E2EF
:10A770000E94DAF9409192115091931160919411D5
:10A780007091951183EF94E20E94DAF98AE0DF91EB
:10A79000CF911F910F91FF90EF90DF90CF90BF90DE
:10A7A000AF909F908F907F906F905F904F903F9071
:10A7B0000C9481F760908A1170908B1180908C11AD
:10A7C00090908D11A0908E11B0908F1100919011EA
:10A7D00010919111C0909211D0909311E09094112A
:10A7E000F090951188E50E9476EEC82F882309F431
:10A7F0009AC00E94FEED362E472E582ED92F20E00B
:10A8000030E040EB53EC0F942D3687FD0DC020E077
:10A8100030E040EB53E4632D742D852D9D2F0F9474
:10A82000FD2C18160CF081C060E671E08BEA9CE00C
:10A830000E94FCF960E671E086EA9CE00E94FCF967
:10A8400083EA9CE00E94A9F7C0E089E50E9476EEC9
:10A85000882361F10E94FEED362E472E582ED92F07
:10A8600020E030E044EB53EC0F942D3687FD0DC013
:10A8700020E030E044EB53E4632D742D852D9D2FB3
:10A880000F94FD2C18160CF055C068E671E080E9B5
:10A890009CE00E94FCF968E671E08BE89CE00E9475
:10A8A000FCF988E89CE00E94A9F7C0E08AE50E94D4
:10A8B00076EE882309F443C00E94FEED6B017C0113
:10A8C00020E030E040E151EC0F942D3687FD0AC0C6
:10A8D00020E030E040E151E4C701B6010F94FD2CC7
:10A8E00018166CF567EF7FEF86E79CE00E94FCF995
:10A8F00069E070E081E79CE00E94FCF98EE69CE054
:10A90000DF91CF911F910F91FF90EF90DF90CF904B
:10A91000BF90AF909F908F907F906F905F904F907F
:10A920003F900C94A9F7C1E090CF632C742C852C38
:10A930009D2E8BCFA32CB42C052D1D2FB7CFCC2350
:10A94000E1F0C301D40180938A1190938B11A093FD
:10A950008C11B0938D11C501D80180938E11909305
:10A960008F11A0939011B0939111C0929211D09237
:10A970009311E0929411F0929511DF91CF911F9174
:10A980000F91FF90EF90DF90CF90BF90AF909F908E
:10A990008F907F906F905F904F903F900895CF92EF
:10A9A000DF92EF92FF928AE50E9476EE882309F407
:10A9B0005AC00E94FEED20E030E040E050EC0F94E1
:10A9C000FD2CC12CD12CE12C90ECF92E87FD0FC071
:10A9D0000E94FEED20E030E040E050E40F942D3680
:10A9E00018160CF462C00E94FEED6B017C012091F0
:10A9F0006C0B30916D0B40916E0B50916F0BC7013A
:10AA0000B6010F94632D0F943935CB010E94B3C862
:10AA100080E50E9428EE81114EC0A7019601609149
:10AA200092117091931180919411909195110F94BE
:10AA3000CD336093921170939311809394119093FE
:10AA400095110F94990B409192115091931160912F
:10AA50009411709195118FE59CE00E94DAF98AE0DB
:10AA60000E9481F705C083E50E9476EE8111A1CF97
:10AA70008091400487FD24C080914104837001F5DA
:10AA80000F94990B409192115091931160919411F0
:10AA90007091951180E59CE00E94DAF98AE0FF90C0
:10AAA000EF90DF90CF900C9481F7C12CD12CE12C4A
:10AAB00080E4F82E9CCF0E94EAED8111AECFD8CF72
:10AAC00082E50E9428EE8111DBCFFF90EF90DF90AE
:10AAD000CF9008954F925F926F927F928F929F9244
:10AAE000AF92BF92CF92DF92EF92FF92CF93DF931C
:10AAF000CDB7DEB72C970FB6F894DEBF0FBECDBF33
:10AB00004090F2075090F3076090F4077090F507BB
:10AB10002091300230913102409132025091330243
:10AB2000C301B2010F94CD3369837A838B839C83F5
:10AB30008090F6079090F707A090F807B090F9077B
:10AB40002091340230913502409136025091370203
:10AB5000C501B4010F94CD336D837E838F839887B5
:10AB6000C090FA07D090FB07E090FC07F090FD073B
:10AB7000209138023091390240913A0250913B02C3
:10AB8000C701B6010F94CD3369877A878B879C877D
:10AB900020913C0230913D0240913E0250913F0293
:10ABA000C301B2010F94CD332B013C01209140022F
:10ABB000309141024091420250914302C501B401DB
:10ABC0000F94CD334B015C0120914402309145023A
:10ABD0004091460250914702C701B6010F94CD3310
:10ABE0006B017C010F94990B88E894E00E94A9F70F
:10ABF00083E50E9428EE882321F00E94EAED8093ED
:10AC00002E0280912E02811151C08FE694E00E94A5
:10AC1000A9F780E894E00E94A9F749815A816B81E5
:10AC20007C8186EB93E10E94DAF94D815E816F8130
:10AC3000788586EF94E20E94DAF949855A856B851A
:10AC40007C8583EF94E20E94DAF98EE794E00E941B
:10AC5000A9F786E794E00E94A9F7B301A20186EB69
:10AC600093E10E94DAF9B501A40186EF94E20E9413
:10AC7000DAF9B701A60183EF94E20E94DAF98AE0DB
:10AC80002C960FB6F894DEBF0FBECDBFDF91CF91EB
:10AC9000FF90EF90DF90CF90BF90AF909F908F90FC
:10ACA0007F906F905F904F900C9481F783E794E0D2
:10ACB000AECF2F923F924F925F926F927F928F9280
:10ACC0009F92AF92BF92CF92DF92EF92FF920F933B
:10ACD0001F93CF93DF93CDB7DEB7E5970FB6F89408
:10ACE000DEBF0FBECDBF8DAB209123042CAB21E086
:10ACF0002093230480918E048D3409F4CBC48435D1
:10AD000011F40C94846A873409F091C180918C0409
:10AD100090918D048B31910509F430C208F079C10E
:10AD20008430910508F030C120910B0682309105E6
:10AD300008F4E1C1213009F0E4C111E0029709F003
:10AD400010E00E94B31F19821A821B821C821D828E
:10AD50001E821F82188682E50E9476EE882309F4FF
:10AD6000E3C10E94FEED6B017C0120E030E0A9010F
:10AD70000F94FD2C882309F4EAC040904A025090B9
:10AD80004B0260904C0270904D0280914E02909167
:10AD90004F02A0915002B09151028CA79DA7AEA77F
:10ADA000BFA78090960690909706A0909806B090C6
:10ADB000990680919A0690919B06A0919C06B0916D
:10ADC0009D0688AB99ABAAABBBABA5019401C301AF
:10ADD000B2010F94FD2C81110DC028A939A94AA9EF
:10ADE0005BA96CA57DA58EA59FA50F94FD2C88233E
:10ADF00009F4ADC0A3019201C501B4010F94CC3395
:10AE000020E030E040E05FE30F94632D68A779A76E
:10AE10008AA79BA72CA53DA54EA55FA568A979A9E2
:10AE20008AA99BA90F94CC3320E030E040E05FE397
:10AE30000F94632D2B013C0120E030E0A901C701F4
:10AE4000B6010F94FD2C881F8827881F181709F456
:10AE500062C180E090E0A0E8BFEB8CA79DA7AEA701
:10AE6000BFA728A539A54AA55BA5CA01B9010F94BA
:10AE7000632D4B015C01A3019201C301B2010F9448
:10AE8000632D9B01AC01C501B4010F94CD330F9428
:10AE90007B364B015C01AC019B01C701B6010F94ED
:10AEA000CC3368AB79AB8AAB9BABA5019401C701EE
:10AEB000B6010F94CD339B01AC0168A979A98AA989
:10AEC0009BA90F94632D6B017C0120E030E0A90168
:10AED0000F942D3687FD24C1C701B6010F947B3630
:10AEE0006B017C01C301B2019058A50194010F943C
:10AEF000C7342CA53DA54EA55FA50F94632DA701D2
:10AF000096010F94632D28A539A54AA55BA50F943A
:10AF1000CD3369837A838B839C83A501940168A5D3
:10AF200079A58AA59BA50F94C7342CA53DA54EA550
:10AF30005FA50F94632DA70196010F94632DA301C4
:10AF400092010F94CD336D837E838F83988720E0A9
:10AF500030E0A90169817A818B819C810F94FD2C5D
:10AF60008111F6C020E030E0A9016D817E818F81E2
:10AF700098850F94FD2C8111EBC00F94950B80E602
:10AF800095E00E94A9F7BDC08531910509F4B9C0CB
:10AF90008A31910509F4EFC0049709F048C080E5B3
:10AFA0000E9476EEC12CD12C7601882321F00E94DC
:10AFB0007BE86B017C0183E50E9476EE882361F0DB
:10AFC0000E94FEED20E030E04AE754E40F94632D48
:10AFD0000F9440356B017C010E94B22380913710A1
:10AFE000811105C060E086E795E00E947A3C0E94EE
:10AFF0007AC8C60ED71EE81EF91E0E947AC86C19C0
:10B000007D098E099F0997FF7CC080E00F94440F53
:10B01000F4CF8232910509F401C260F48D319105BB
:10B0200009F429C108F4C3C04E9709F47CC10E94F9
:10B0300065C467C08A35910509F4B5C208F58A97D9
:10B04000B1F780910B06813009F05BC089E40E9462
:10B0500076EE082FF12C882319F00E94FAEDF82ED5
:10B060008AE40E9476EEE82E882309F4DAC10E9471
:10B07000FAED182F0111D8C1153008F4DFC1D7C17E
:10B080008B35910509F492C28C35910581F680913A
:10B090008B04882309F48EC2893099F562EEA62EBE
:10B0A00062E0B62E7AE4C72E72E0D72EE12C00E0E3
:10B0B00010E0D5018D915D010E9476EEF82E882377
:10B0C00061F0133011F4082FFE2C0E94FEEDF60102
:10B0D0006083718382839383EF2C1F5FF4E0CF0E34
:10B0E000D11C143031F7EE2009F4B6C20E946E3143
:10B0F0000E94993106C0213021F40E94B31F0E94A2
:10B10000DB2A3DA9311102C00E948EDF8CA98093F9
:10B1100023040C94436380E090E0A0E8BFE39DCE5D
:10B12000C12CD12C7601DECE89E40E9476EE8823F4
:10B1300031F00E94FEED69837A838B839C838AE4DD
:10B140000E9476EE882309F402CF0E94FEEDFBCE2A
:10B15000412FBE016F5F7F4F86E996E00E94E1DFDD
:10B160000E947AC8609388107093891080938A1027
:10B1700090938B10C6CF0F945C03C3CF87E00E94DF
:10B1800074528111BECF8CE0E6EDF2E0DE01119643
:10B1900001900D928A95E1F770E060E080E50E94F1
:10B1A000A51FBE016F5F7F4F0E94C535AACF87E004
:10B1B0000E940D2A811106C060E08FE40E9415EF05
:10B1C00081119FCF0E94B22310922F0260914B0BEE
:10B1D0008CE40E9415EFE82E80E00E94BCF10E94F2
:10B1E0007AC8609388107093891080938A10909326
:10B1F0008B100E94A72D81E08093C7050E94023327
:10B200008AE50E9428EEF82E882369F081E00E94EA
:10B210000D2A182F82E00E940D2A11110C94F26B56
:10B2200011E0811101C010E088E50E9428EE811133
:10B230000C94996A112311F40C949C6A012F10E06C
:10B240000C94A96A60E070E080E890E40C94B26A23
:10B25000A3019201C501B4010C94FF6A60E081E989
:10B2600095E00E947A3C0F94990B8FE795E00E943D
:10B27000A9F70C94DB6B14E00E947AC860938810E5
:10B280007093891080938A1090938B1080914B0B50
:10B29000811127C08EE40E9428EE882321F082EAE3
:10B2A00095E00E94246C87E00E94745281111FC0B7
:10B2B0000F9470168823D9F0115001F130E020E08E
:10B2C00043E15EE06DEC75E085E00E9411F961E01C
:10B2D00080EC95E00E94B8F888EA95E00E94246C22
:10B2E000CBCF60E08FE40E9415EF882399F20E9493
:10B2F000E9F88BE696E00E94246C03CF61E08EE5CE
:10B3000096E00E94B8F889EE95E00E94246C61E016
:10B310008EEF9DE00E94B8F840E070E060E08AEDBA
:10B3200095E00F94730E0091961110919711D8012A
:10B330002D913D914D915C9160914A0270914B022B
:10B3400080914C0290914D020F94CD33AB01BC0122
:10B3500088E50E94E3EE69837A838B839C83F801FE
:10B36000248135814681578160914E0270914F0250
:10B3700080915002909151020F94CD33AB01BC01EA
:10B3800089E50E94E3EE6D837E838F839887BE01FB
:10B390006B5F7F4FCE0101960E94B4E8882309F4C9
:10B3A000B0CE80E00E94BCF10E94A72D61E085E450
:10B3B0000E9415EF182F01E021E0482FBE016B5FBE
:10B3C0007F4FCE0101960E94A2C46B017C01AC01AB
:10B3D0009B010F94BF36811119C049815A816B813D
:10B3E0007C818DE896E00E94DAF94D815E816F8163
:10B3F000788588E896E00E94DAF9B701A60183E82B
:10B4000096E00E94DAF98AE00E9481F70E948E2D70
:10B4100011110E949AE80E94993173CE0E94C3FED6
:10B4200070CE10E0002351F0F4E0FF1528F485E918
:10B4300096E00E94A9F765CEE1101ECE80E1EAE415
:10B44000F2E0A6E9B6E001900D928A95E1F70023BB
:10B4500019F16F2DFF0C770B880B990B0F94042DAE
:10B460002091F5043091F6044091F7045091F804CE
:10B470000F94632D2091ED043091EE044091EF0480
:10B480005091F0040F94CD33609396067093970615
:10B490008093980690939906EE2019F1612F110F71
:10B4A000770B880B990B0F94042D2091F9043091A0
:10B4B000FA044091FB045091FC040F94632D2091F9
:10B4C000F1043091F2044091F3045091F4040F948C
:10B4D000CD3360939A0670939B0680939C0690935D
:10B4E0009D0660E080E50E9415EF8823C1F10023EE
:10B4F000D1F0E0919611F091971120813181428134
:10B50000538160919606709197068091980690916C
:10B5100099060F94CC3360939606709397068093A8
:10B52000980690939906EE20D1F0E0919611F09153
:10B530009711248135814681578160919A067091D7
:10B540009B0680919C0690919D060F94CC3360934E
:10B550009A0670939B0680939C0690939D0640E00C
:10B5600050E0BA0186E40E94E3EE6B017C0120E02A
:10B5700030E0A9010F942D3618168CF420E030E04D
:10B5800040E752E4C701B6010F94C73469837A8358
:10B590008B839C83CE0101960E94C62DB2CD60E0C4
:10B5A00070E0CB01F3CF10921607ABCD8FE0809304
:10B5B0001607A7CD52EEC52E52E0D52EF12CE12C68
:10B5C00000E010E0D6018D916D010E9476EE382EDC
:10B5D0008823D9F10E94FEED4B015C01133059F034
:10B5E000F701EE50F84F20813181428153810F9451
:10B5F000CC334B015C01F701E65BFD4F20813181CB
:10B6000042815381C501B4010F94CC332B013C011D
:10B610002DEB37E346E855EB0F942D3687FD0AC036
:10B620002DEB37E346E855E3C301B2010F94FD2C3F
:10B6300018165CF41330C1F48092560290925702AF
:10B64000A0925802B0925902032D1F5FB4E0EB0E96
:10B65000F11C143009F0B6CF002309F449CD86E57A
:10B6600092E00E94832744CDF701E45EF84F5F012A
:10B67000A301920160817181828193810F94CD3306
:10B68000D5016D937D938D939C931397812F0E9489
:10B69000E61CDBCF80918C0490918D048937910555
:10B6A00011F40C94446508F0B7C18D34910509F488
:10B6B000F7C608F0CEC08A31910509F42CC608F00F
:10B6C00071C08431910509F472C508F04EC0813112
:10B6D000910509F431C508F042C0029708F0A7CCE3
:10B6E00080E50E9476EEC12CD12C7601882321F0D2
:10B6F0000E947BE86B017C0183E50E9476EE882343
:10B7000061F00E94FEED20E030E04AE754E40F943F
:10B71000632D0F9440356B017C010E94B223809110
:10B720008F0490919004892B09F401C50E9473C481
:10B7300080918C0490918D0466EB76E0892B11F456
:10B740006EEA76E030E020E04EEB56E082E00E94C8
:10B7500011F940E0C701B6010F94891ED2CC42977F
:10B7600009F065CC0E9483EECCCC8731910509F4B9
:10B7700053C570F48531910509F44AC5469709F01F
:10B7800056CC8091431382FDBCCC0E94127EB9CC72
:10B790008831910509F455C5499709F048CC0E94B4
:10B7A0001022AFCC8032910509F439C6C0F58D3135
:10B7B000910509F41DC670F48B31910509F4BEC5DD
:10B7C0004C9709F034CC80918F04909190040E94A2
:10B7D000048397CC8E31910509F411C64F9709F077
:10B7E00026CC0E9478356C8F7D8F8E8F9F8FBE0107
:10B7F0006F5F7F4FCE014C960E943E1ECE01019698
:10B800000E9464AF0F94990BBE016F5F7F4F82E37C
:10B8100097E00F948B0B8AE00E9481F772CC8934F9
:10B82000910509F429C650F48132910509F420C626
:10B83000C09709F0FCCB0E9406FA63CC8B349105CB
:10B8400009F42AC68C34910509F0F1CB0E94213904
:10B8500058CC8C36910509F454CC08F072C085356B
:10B86000910511F40C94316490F58235910509F439
:10B87000E8C720F58E34910509F416C68135910587
:10B8800009F0D5CB0E94AC890E94C3230E94E6F345
:10B890000E94E9F31092B1061092B0061092AF0622
:10B8A00068EE73E080E090E00E94D9F20E94EEF32F
:10B8B00060E08DEF97E00E947A3C23CC83359105C0
:10B8C00009F4C7C78435910509F44CCFB0CB89364C
:10B8D000910509F4C6C600F58C35910509F4E6C753
:10B8E0008836910509F0A3CB8091080B83FD09CC24
:10B8F0000E94E02087FD05CC83E50E9476EE882338
:10B9000041F00E94FAED0E94822361E080E00F94F2
:10B910001D210F947C20F5CB8A36910509F4CCC605
:10B920008B36910509F083CB60E080E50E9409EF3A
:10B93000823008F0E6CBE82FF0E0ED5DF74F1082A3
:10B94000E0CB8237910511F40C94F764A0F58F36A3
:10B95000910509F4DAC6C8F48D36910509F436C6A6
:10B960008E36910509F063CB8EE40E9476EE882333
:10B9700009F4C7CB0E94C6ED6093380C7093390C64
:10B9800080933A0C90933B0CBCCB8037910509F423
:10B99000B8CB8137910509F04ACB83E50E9476EE5A
:10B9A000882309F4F9C60E94D6ED8D3308F0EFC65E
:10B9B00080930002A6CB8637910511F40C9407659D
:10B9C000D0F48337910511F40C94FF648537910509
:10B9D00009F02DCB80918F0490919004009711F481
:10B9E0000C940365DC012C91222311F40C94036563
:10B9F0000E9464AF86CB8737910511F40C944065A3
:10BA00008837910509F013CB81E08093C7058093B7
:10BA1000C6050E94023375CB8239E1E09E0711F41E
:10BA20000C94976808F078C1833D910511F40C944B
:10BA3000246608F0C4C0883C910511F40C944C6550
:10BA4000D0F58C38910509F4B4C628F48D379105EA
:10BA500009F4A5CEECCA8B39910509F4CBC68E3B0F
:10BA6000910509F0E4CA8091080B83FD4ACB83E578
:10BA70000E9476EE182F882309F4B2C60E94FAEDD0
:10BA80000E947AED60E081E00F941D2120919410D6
:10BA90003091951080919210909193108217930796
:10BAA0000CF4A5C68FED97E060E00E947A3C812FF0
:10BAB0000E94508626CB8C3C910511F40C94A7650E
:10BAC00048F5893C910511F40C947D658B3C9105FA
:10BAD00009F0ADCA0E94E02087FD13CB12EEE12EE3
:10BAE00012E0F12E10E000E0D7018D917D010E945F
:10BAF00028EE882349F00E94FEEDF801E05BF44F48
:10BB000064A375A386A397A30C5F1F4F0031110593
:10BB100059F7F7CA8D3C910511F40C942066B8E2F0
:10BB2000EB2EB7E0FB2E10E08E3C910509F07FCAAA
:10BB300088E5810F0E9428EE882351F00E94FEEDD7
:10BB4000F7016083718382839383812F0E94E61CB7
:10BB50001F5FF4E0EF0EF11C133051F780914004A9
:10BB600087FDC6CA80914104837009F0C1CA409123
:10BB700028075091290760912A0770912B0785E2C9
:10BB800098E00E94DAF940912C0750912D076091BE
:10BB90002E0770912F0786EF94E20E94DAF9409108
:10BBA000300750913107609132077091330783EF6E
:10BBB00094E20E94DAF98AE00E9481F7A2CA8D32EB
:10BBC00021E0920711F40C94256708F06CC08831CD
:10BBD000A1E09A0711F40C94856608F045C08C3DED
:10BBE000910511F40C9428668D3D910509F01FCA4A
:10BBF0000E94E020082F87FD84CA83E50E9476EE2C
:10BC0000002E000C110B7801EE0CFF1C882311F4A0
:10BC10000C946B660E94FAEDF701E25AFD4F918396
:10BC20008083000F111F000F111F9801265A3D4FEE
:10BC30007901BC01990F880B990B0F94042D2AE010
:10BC400037ED43E25CE30F94632D045B144FD8019E
:10BC50002D913D914D915C910F94632DF70160837F
:10BC60007183828393834DCA8232E1E09E0711F48F
:10BC70000C9421678C32914009F0D9C964E071E0DD
:10BC800083E50E94A51F8C0168EE73E080E50E94A9
:10BC9000A51F893823E1920710F088E893E1B801E5
:10BCA0000E94E8392ECA803321E0920711F40C94E7
:10BCB000A76700F58E32A1E09A0711F40C941B6877
:10BCC0008F32914009F0B3C970E060E085E40E94D2
:10BCD000FAEEF82E3FEF831711F40C949068882346
:10BCE00011F40C9461688FEB98E00E94A9F70E9410
:10BCF0002AAE07CA8039E1E09E0711F40C949368DC
:10BD00008139914009F093C98091A6068111F0C94B
:10BD100081E00E941133ECC9883F31E0930711F4B0
:10BD20000C94956908F0E2C0863AB1E09B0711F4E3
:10BD30000C944C6A08F0B3C08D39F1E09F0711F400
:10BD40000C94606A78F58A3931E0930709F4D9C90F
:10BD50008C39914009F06BC980913E04887811F0CC
:10BD60000C949F6880914004867011F00C949F6839
:10BD70000F94990B83E099E00E94A9F780910F023C
:10BD80000E94BCF940910B0250910C0260910D028F
:10BD900070910E0283EE98E00E94DAF98AE00E9428
:10BDA00081F7AFC9843AB1E09B0711F40C94CF68D6
:10BDB000853A914009F03BC96FEF7FEF89E40E941B
:10BDC000FAEE082F6FEF7FEF8AE40E94FAEE182F49
:10BDD0008AE50E9476EED12C811108C081E50E948F
:10BDE00076EED82E882311F40C94EA6BC02E81E0F5
:10BDF000800F863010F00C94D668912E81E0810F70
:10BE0000863010F00C94D6680E94FEED2B013C01A8
:10BE1000F02E07FDF12C07FF02C004E0C02E812E9A
:10BE200017FD812C17FF02C014E0912EB5E03B2EC8
:10BE3000CF1408F466C9E82C3F9C500111249E14CD
:10BE400010F40C94D3680E2D10E020E030E0A9012E
:10BE5000DD2069F0F501E00FF11FEE0FFF1FEE0F7F
:10BE6000FF1FEE54F94F20813181428153810A0D29
:10BE70001B1D000F111F000F111F0E54194FC3017E
:10BE8000B2010F94CD33D8016D937D938D939C9324
:10BE900013976E2D8F2D0E9406C3E394D0CF853F5C
:10BEA000F1E09F0711F40C948D6968F48C3A31E04D
:10BEB000930711F40C94DE68843F914009F0B7C8F1
:10BEC0000E94C43C1EC9863FB1E09B0711F40C944C
:10BED0009169873F914009F0AAC861E083E50E941B
:10BEE00015EF91E089270E94A1A30BC98335F3E0E8
:10BEF0009F0711F40C94486A08F0CBC08B3532E0F0
:10BF0000930711F40C94B86968F48C30B2E09B0785
:10BF100011F40C94A7698835924009F088C80E94F2
:10BF20000521EFC88D3BF2E09F0711F40C94386AAD
:10BF30008E3B924009F07BC80E94E020182F87FDBD
:10BF4000E0C88AE50E9476EE812C912C90E2A92E21
:10BF500091E4B92E882379F040E050E0BA018AE5F7
:10BF60000E94E3EE4B015C0120E030E0A9010F9458
:10BF70002D3618167CF580E090E0A0EAB0E48983C5
:10BF80009A83AB83BC83209152023091530240913B
:10BF9000540250915502C501B4010F94CD336B0189
:10BFA0007C0120E030E048EC53E40F94FD2C87FD49
:10BFB00006C0C12CD12C88ECE82E83E4F82ECC8E60
:10BFC000DD8EEE8EFF8EBE016F5F7F4FCE014C96F1
:10BFD0000E94433085E50E9428EE882311F40C94DA
:10BFE0003C6A0E94FEED6B017C0120E030E0A9017B
:10BFF000C701B6010F942D3687FF04C0F7FAF094FD
:10C00000F7F8F094F7FAF094F7F8F094C982DA822E
:10C01000EB82FC8280E00F944F1C882321F0CE013C
:10C0200001960E94FDF220E030E0A901C501B401B3
:10C030000F942D3618160CF064C880E090E0A0EA4A
:10C04000B0E489839A83AB83BC83A501940160919A
:10C0500052027091530280915402909155020F94B4
:10C06000CC336B017C0120E030E0A9010F942D3628
:10C0700018161CF0C12CD12C7601CC8EDD8EEE8EE4
:10C08000FF8EBE016F5F7F4FCE014C960E94433002
:10C0900038C8873E33E0930711F40C94506AB8F423
:10C0A0008C36B3E09B0709F42CC8803A934011F01A
:10C0B0000C94175820918F04309190049091431361
:10C0C000926090934313C9010E9404831AC8883E6A
:10C0D000F3E09F0711F40C94796A893E934011F0C4
:10C0E0000C9417588091391381110C947D6A0E9429
:10C0F000A1EF0E94F9820E9478356D3371058105A8
:10C10000910520F085EC99E00E94246C81EC99E087
:10C110000E94246C84EE80939B048DEA99E00E9437
:10C12000A9F789EA99E00E94246C0C94815887EC65
:10C1300096E00E94C336FCCA80913E0484FD18C07C
:10C140008091400487FD14C080914104837081F484
:10C1500060E08AED96E00E947A3C5F988A98809130
:10C160000801817080930601479812980C948158B9
:10C1700088E50E9428EE81115F9889E50E9428EEEB
:10C1800081118A988AE50E9428EE882331F08091F7
:10C190000801817080930601479885E40E9428EE8B
:10C1A000882311F40C94815812980C948158809132
:10C1B000431383FF25C082EF96E00E94A9F7809188
:10C1C000431383FF17C083E693E10E94897E8BE1CE
:10C1D000E3E6F3E1DE01119601900D928A95E1F715
:10C1E00070E060E0CE0101960E944084CE0101968D
:10C1F0000E94C9EF83EE96E00E94A9F70C94815843
:10C200000F94990B83E097E00E94A9F70C94815852
:10C210000E94237E0C94815880918F049091900409
:10C22000FC012191222331F02032D9F7DF0111974F
:10C230001C92F7CF60E00E944D8310929B040C94F7
:10C24000815883E50E9476EE882321F00E94C6ED96
:10C250000E94895084E50E9476EE8823A9F00E940E
:10C26000C6ED6B017C010E94AA35C092BE04D0923B
:10C27000BF04E092C004F092C104CD28CE28CF289C
:10C2800019F081E080933610809135108823F9F001
:10C2900080E090E0A0EAB1E489839A83AB83BC8319
:10C2A0001C8E1D8E1E8E1F8E18A219A21AA21BA2F2
:10C2B00010E000E020E0AE014F5F5F4FBE01645E22
:10C2C0007F4FCE0180960F94B01C0C9481580E9431
:10C2D000D8F3882381F00E9400760E94743882E7A8
:10C2E00097E00E94B17D10929F0C1092A00C1092CA
:10C2F000A10C1092A20C61E086E29EE00E94B8F8C8
:10C3000043E15EE06DE077E085E00E9421AE0E94AF
:10C310009CAF0C9481588091431383FD02C00C9410
:10C32000815883E50E9476EE882311F40C9481589D
:10C330000E94C6ED0E9489500C94815883E40E94AB
:10C3400028EE882361F183E297E00E94A9F78091AB
:10C35000AA148823F9F0BE016F5F7F4F87EA94E14A
:10C360000E94447DCE0101960E94F679CE0101968D
:10C370000E94CF7E8091B110882339F080E20E9424
:10C3800081F781EB90E10E94F6798AE00E9481F7C3
:10C390000C94815889E197E00E94A9F7F6CF83E5D4
:10C3A0000E9476EE882301F10E94D6ED182F8C337F
:10C3B00008F08CE3809318040E947AC86B017C011A
:10C3C000212F30E0A8EEB3E00F949533C60ED71EB0
:10C3D000E81EF91EC0921404D0921504E0921604CF
:10C3E000F09217040C9481580E94BE750C948158E9
:10C3F000809143138E7F809343130C9481588091D6
:10C40000431383FD02C00C9481580E944BC4809159
:10C410008F04909190040E9491820C948158809195
:10C42000431382FD0E94B2238091431383FD02C017
:10C430000C94815860E080E50E9415EF182F682F5A
:10C4400080918F04909190040E944D8383E50E9417
:10C4500076EE882321F00E94C6ED0E9489500E944A
:10C46000007611110C9481580E9474380C948158F4
:10C470000E94C8520C94815880E50E9428EE8823BF
:10C4800011F40C9481580E94D6ED853608F084E6AC
:10C4900080939B040C9481580E9474380C948158AA
:10C4A0000E94E6F30C94815870E060E083E50E94FE
:10C4B000FAEE8E34910531F40E9421230E949CAF44
:10C4C0000C9481588DE997E00E94A9F76091B60518
:10C4D0007091B70584E997E00E94C8F96091B805AA
:10C4E0007091B90587E897E00E94C8F96091B60598
:10C4F0007091B7058091B8059091B905681B790BCB
:10C5000080913610815021E030E0823010F030E030
:10C5100020E0621B730B8CE797E00E94C8F98AE069
:10C520000E9481F784E797E00E94A9F78091BA05FD
:10C530009091BB05A091BC05B091BD058C8F9D8FDE
:10C54000AE8FBF8FBE016F5F7F4FCE014C960E94B2
:10C550003E1EBE016F5F7F4F87E697E00F948B0B07
:10C560008091BE059091BF05A091C005B091C10515
:10C570008C8F9D8FAE8FBF8FBE016F5F7F4FCE01BF
:10C580004C960E943E1EBE016F5F7F4F87E597E08D
:10C590000F948B0B20E030E04AE754E46091C20531
:10C5A0007091C3058091C4059091C5050F94C7345F
:10C5B000AB01BC018FE397E00E94DAF98DE60E949F
:10C5C00081F78AE00E9481F70C9481588091080BD2
:10C5D00083FF02C00C9481580E94E020082F87FF3F
:10C5E00002C00C94815883E50E9476EE182F8823B0
:10C5F00059F10E94FAED0E94822361E081E00F94DC
:10C600001D212091FF10309100118091FD1090911B
:10C61000FE1082179307F4F480EB97E09F938F93BB
:10C620008BEB97E09F938F931F920E9431C40F94DE
:10C630007C200F900F900F900F900F90612F802F04
:10C640000E94C7870C94815882E50E9476EE811182
:10C65000D0CF5FC985EA97E0112301F30F947C20C6
:10C66000EDCF0E94E020182F87FD0AC080EC97E0F4
:10C670000E94A9F7812F0E94DD858AE00E9481F740
:10C680003CA930932304E5960FB6F894DEBF0FBEA5
:10C69000CDBFDF91CF911F910F91FF90EF90DF9071
:10C6A000CF90BF90AF909F908F907F906F905F9052
:10C6B0004F903F902F90089560E080E50E9409EF31
:10C6C000F82E81E08F1510F40C94815881E40E94BB
:10C6D00028EE60912308062F811102C00FEF10E0B1
:10C6E00083E50E9476EE882349F00E94C6ED8B0117
:10C6F0006F3F710519F010F00FEF10E0EF2DF0E033
:10C70000ED5DF74F00830C94815883E50E9428EE7D
:10C71000882331F060E083E50E9409EF8093080BE5
:10C720000F94990B81ED97E00E94A9F78091080B77
:10C73000882351F110E000E020E08091080B90E0A8
:10C74000B0E0A0E0002E04C0B695A7959795879518
:10C750000A94D2F780FF12C0FF24F394F20E222332
:10C7600019F08CE20E9481F7F801EE0FFF1FE953E8
:10C77000F84F859194910E94A9F72F2D0F5F1F4FBD
:10C7800005301105D1F601CE83EC97E005CE8CE3A0
:10C79000809300020C9481580F94990B60910002D1
:10C7A00088ED97E00E94D2F98AE00E9481F70C940C
:10C7B00081588091080B83FF02C00C94815883E557
:10C7C0000E9476EE882311F40C9481580E94FAEDB1
:10C7D0000E947AED61E080E00F941D210C94815855
:10C7E00082E50E9476EE811149C90C9481588EEE43
:10C7F00097E05AC983E50E9476EE882311F40C94E1
:10C8000081580E94D6ED182F8C3308F08CE380936A
:10C810001D040E947AC86B017C01212F30E0A8EE34
:10C82000B3E00F949533C60ED71EE81EF91EC092D2
:10C830001904D0921A04E0921B04F0921C040C9488
:10C840008158809116078F7D8061809316070C9424
:10C850008158809116078F7E8062809316070C9412
:10C86000815883E50E9428EE882311F40C948158A6
:10C870000E947AC8609388107093891080938A1000
:10C8800090938B100E94FEED20E030E04AE754E4E4
:10C890000F94632D0F94403560931E0470931F0412
:10C8A00080932004909321040C9481580E94E020EE
:10C8B00087FF02C00C94815880913E0484FD09C01A
:10C8C0008091400487FD05C080914104837009F484
:10C8D00089C022EEC22E22E0D22E30E5E32E3BE0CC
:10C8E000F32E10E0D6018D916D010E9476EE882323
:10C8F00009F465C0133009F06DC00E94FEED4B01D4
:10C900005C0120E030E040EA51E40F94FD2C87FF09
:10C910004EC0A50194016091700B7091710B8091D4
:10C92000720B9091730B0F94C7342B013C01AC0137
:10C930009B0160910B0870910C0880910D089091FB
:10C940000E080F94632D60930B0870930C0880936E
:10C950000D0890930E08A30192016091800B7091D5
:10C96000810B8091820B9091830B0F94632D6093C8
:10C97000800B7093810B8093820B9093830B60915B
:10C980001B0870911C0880911D0890911E080F943F
:10C99000022DA30192010F94632D0F9440356093F3
:10C9A0001B0870931C0880931D0890931E088092AA
:10C9B000700B9092710BA092720BB092730B1F5F71
:10C9C000F4E0EF0EF11C143009F08CCF0E948E239E
:10C9D0000C9481580E94FEEDF701648B758B868B59
:10C9E000978BEDCF81E00E94D8C30C9481580E94B0
:10C9F00069C18DE991E10E9439910C9481580E949E
:10CA00006B1D0C9481580E949CAF0C94815800912E
:10CA10008F041091900494E0F12C40E09150F9F0D3
:10CA2000F8018081282F2B7F213499F42181213333
:10CA3000B1F4813411F1853409F441E098012E5F9D
:10CA40003F4F89012F5F3F4FF80180818032C9F34A
:10CA5000E5CF803521F4818180538A3078F341110C
:10CA60000F94990BFF2021F08FE098E00E94A9F726
:10CA7000C8010E9463520C948158FF24F394DECFC6
:10CA80000E941D1F0C9481581092C7051092C60574
:10CA90000E9402330C9481580E94E020182F87FFD7
:10CAA00002C00C94815800911B0784E40E9476EE2A
:10CAB000F82E8823B1F00E94FEED4B015C0120E0CE
:10CAC00030E0A9010F94FD2C8823A9F024E0120284
:10CAD000F0011124E95EF84F80829182A282B38234
:10CAE0000F2D602F83E50E9415EF80931B070E9496
:10CAF0000B240C94815880E0F8CF0E94E02087FF3F
:10CB000002C00C94815802EE12E080E5E82E8BE022
:10CB1000F82E96EEC92E92E0D92ED8018D918D0176
:10CB20000E9428EE882359F00E94FEED0F944035B4
:10CB3000F70160837183828393830E94981CF4E0E1
:10CB4000EF0EF11CC016D10641F70C94815880916C
:10CB50003F0487FD2DC0809140048E7049F54091BF
:10CB6000840B5091850B6091860B7091870B85E14A
:10CB700098E00E94DAF94091880B5091890B6091FE
:10CB80008A0B70918B0B82E198E00E94DAF9409158
:10CB90008C0B50918D0B60918E0B70918F0B85E4F7
:10CBA00094E10E94DAF98AE00E9481F70C9481589E
:10CBB00083E50E9476EE882391F00E94FEED60935B
:10CBC000840B7093850B8093860B9093870B6093F7
:10CBD0008C0B70938D0B80938E0B90938F0B80E555
:10CBE0000E9476EE882351F00E94FEED6093840B44
:10CBF0007093850B8093860B9093870B82E50E9440
:10CC000076EE882351F00E94FEED6093880B7093BE
:10CC1000890B80938A0B90938B0B84E50E9476EEB0
:10CC2000882311F40C9481580E94FEED60938C0BC4
:10CC300070938D0B80938E0B90938F0B0C94815877
:10CC40000E94B7F70C9481580E946A550C94815841
:10CC500082E40E9428EE882341F080916002909146
:10CC60006102909302028093010282E50E9428EE05
:10CC7000882341F080910102909102029093610219
:10CC80008093600283E50E9476EE882331F00E9453
:10CC9000FAED909361028093600280913E0490913E
:10CCA0003F04A0914004B0914104892B8A2B8B2B27
:10CCB00011F00C94815860916002709161028CE2D5
:10CCC00098E00E94FCF985E20E9481F78AE00E94C8
:10CCD00081F70C9481580F94990B85E40E9481F799
:10CCE00080E3800F0E9481F7F701E25AFD4F6081D7
:10CCF000718180E398E00E94FCF985E20E9481F74F
:10CD00008AE00E9481F70C94815880E50E9428EE09
:10CD1000882311F40C9481580E94FAED8C01892B20
:10CD200009F082C083E50E9428EE882391F00E94DA
:10CD3000FAED8F3F980731F487E891E10E94F3F311
:10CD40000C948158BC0187E891E10E9461F40C9435
:10CD500081580F94990B70E060E08BE398E00E949B
:10CD6000FCF98091891158E5C52E52E0D52EC81ADC
:10CD7000D10887FDD394CC0CDD1CCC0CDD1C0D2C14
:10CD8000000CEE08FF088091881178E8872E912C1E
:10CD9000881A910887FD9394880C991C880C991C1B
:10CDA000092C000CAA08BB088091871190E08F3FE6
:10CDB000C9F1FC01EE0FFF1FE80FF91FE25CFE4E08
:10CDC0008181928133E0880F991F3A95E1F7B0E0B5
:10CDD000A0E044E0B595A795979587954A95D1F73A
:10CDE00002969C012F5F3F4F032E000C440B550B06
:10CDF000281939094A095B09A4EBB0E00F94823382
:10CE0000A7019601281939094A095B090F94633370
:10CE1000B90188E398E00E94FCF98AE00E9481F75A
:10CE20000C94815880E0DDCF0F94950BB80182E51A
:10CE300098E00E94FCF983E498E00E94A9F70C9422
:10CE400081580E94CF540C94815860E085E40E9480
:10CE500009EF811174C080E50E9428EE882351F00B
:10CE60000E94FEED609302117093031180930411F0
:10CE70009093051189E40E9428EE882381F00E9496
:10CE8000FEED2CEA35EC47E25EE30F94632D6093F0
:10CE9000061170930711809308119093091184E48F
:10CEA0000E9428EE882381F00E94FEED2CEA35ECEA
:10CEB00047E25EE30F94C73460930A1170930B113D
:10CEC00080930C1190930D110F94990B40910211C6
:10CED00050910311609104117091051181E698E061
:10CEE0000E94DAF92CEA35EC47E25EE36091061124
:10CEF0007091071180910811909109110F94C73416
:10CF0000AB01BC018DE598E00E94DAF92CEA35EC22
:10CF100047E25EE360910A1170910B1180910C1150
:10CF200090910D110F94632DAB01BC0189E598E040
:10CF30000E94DAF98AE00E9481F70C9481580F94DC
:10CF4000950B85E698E00E94A9F70C94815880E53E
:10CF50000E9428EE882351F00E94FEED6093971006
:10CF6000709398108093991090939A1089E40E947E
:10CF700028EE882381F00E94FEED2CEA35EC47E292
:10CF80005EE30F94632D60939B1070939C108093CD
:10CF90009D1090939E1084E40E9428EE882381F0D7
:10CFA0000E94FEED2CEA35EC47E25EE30F94C734B5
:10CFB00060939F107093A0108093A1109093A21083
:10CFC0000F94990B4091971050919810609199107F
:10CFD00070919A108FE798E00E94DAF92CEA35EC0C
:10CFE00047E25EE360919B1070919C1080919D10D0
:10CFF00090919E100F94C734AB01BC018BE798E071
:10D000000E94DAF92CEA35EC47E25EE360919F106A
:10D010007091A0108091A1109091A2100F94632D97
:10D02000AB01BC0187E798E00E94DAF98AE00E9430
:10D0300081F70C94815883E50E9428EE182F8823ED
:10D0400069F00E94FAED9C01909349028093480296
:10D0500091E0232B09F090E09093250880E50E9451
:10D0600028EE882361F02091480230914902232B59
:10D0700011F00E94EAED809325080C94815811115B
:10D080000C9481580F94990B8FE998E00E94A9F7AE
:10D0900080912508882391F087E898E00E94A9F7FD
:10D0A00060914802709149028EE898E00E94FCF974
:10D0B0008AE898E00E94A9F70C94815883E898E0E8
:10D0C000EDCF04EB10E083E50E9476EE882319F0A3
:10D0D0000E94FAED8C0165E070E083E40E94FAEEB4
:10D0E000E82E60E085E50E9415EFD82E60E082EB27
:10D0F00098E00E947A3CB801110F880B990B0F94AD
:10D10000042D69837A838B839C832D2D4E2D6F2D67
:10D11000CE0101960E948D9E0E949CAF0C94815876
:10D1200006E410E0D0CF0E94B2230C9481580E94F4
:10D1300091E80E949AE80E9499310C94815888E401
:10D140000E9428EE882321F00E94EAED80932204B9
:10D1500082E50E9428EE082F83E50E9428EE182F12
:10D16000011102C0882341F00E948DF3112321F0A8
:10D170000E94EAED80930F0284E40E9428EE882347
:10D1800011F40C9481580E94FEED60930B02709391
:10D190000C0280930D0290930E020C9481580F9410
:10D1A0009D0B0C948158F3940C94185F0F94950B7D
:10D1B00084E399E00E94A9F70C94815887E00E94CB
:10D1C000745281110C9481587FE1C72E7FE0D72ED5
:10D1D000EAE4F2E0F9A7E8A79E012F5F3F4F1901AB
:10D1E000790110E000E0C6010E948BE8A8A5B9A56E
:10D1F0008D909D90AD90BD90B9A7A8A7A501940171
:10D200000F94CC332B013C01F701408251826282A2
:10D21000738220E030E040EA51EC0F942D3687FD18
:10D220000AC020E030E040EA51E4C301B2010F94AB
:10D23000FD2C181684F4F801ED5BF04FE4911E16F6
:10D2400054F4B7FAB094B7F8B094D7018D929D9288
:10D25000AD92BC921397F70181909190A190B190FB
:10D260007F0120E030E040EA51ECC501B4010F94A9
:10D270002D3687FD3FC020E030E040EA51E4C50193
:10D28000B4010F94FD2C1816ACF10F5F1F4FF4E0A2
:10D29000CF0ED11C0330110509F0A5CF68E2E62EB0
:10D2A00067E0F62E10E0F10181919191A191B19189
:10D2B0001F01F70181939193A193B1937F01812F76
:10D2C0000E94E61C1F5F133071F70E94993160E0E5
:10D2D0008DE499E00E947A3C63E972E084E690E094
:10D2E0000E94E8396AEB72E084E690E00E94E83937
:10D2F0000C9481580F94950B8BE699E00E94A9F746
:10D3000061E08DE599E00E947A3C68E270E088EC8B
:10D3100090E00E94E8390C9481580E94AFAA0C94C6
:10D3200081580E941F9D0C948158209301050E94F2
:10D33000DD2210920105882311F40C9481580F947A
:10D34000990B89E899E00E94A9F70C948158809183
:10D35000431382FF05C08064809343130C9481586B
:10D3600083FD02C00C9481580E944BC40C948158D8
:10D370000E94E020082F87FF02C00C94815885E5A9
:10D380000E9428EE882359F10E94FEED4B015C01BA
:10D39000E02E002E000CFF0820E030E0A9010F94E1
:10D3A0002D3687FF04C0B7FAB094B7F8B09420E0E8
:10D3B00030E84BE354E4C501B4010F942D369701D6
:10D3C00053E0220F331F5A95E1F72C523B4F1816AA
:10D3D000D4F1D9018D929D92AD92BC9213978CE4B9
:10D3E0000E9428EE882311F40C9481580E94FEEDCF
:10D3F0006B017C01002E000C110B20E030E0A90134
:10D400000F942D3687FF04C0F7FAF094F7F8F094E4
:10D4100020E030E84BE354E4C701B6010F942D3609
:10D42000980143E0220F331F4A95E1F72C523B4FFE
:10D4300018169CF0D9011496CD92DD92ED92FC92D3
:10D4400017970C94815880E090E8ABE3B4E4F901BD
:10D4500080839183A283B383C2CF80E090E8ABE363
:10D46000B4E4F90184839583A683B7830C9481582F
:10D470000E94662E0C94815828E01202F0011124BB
:10D48000EC52FB4FC080D180E280F3800C94F55FBA
:10D490000E948D530C9481580E94DEFD0C9481589B
:10D4A00081E080930B061092771060E083E50E9484
:10D4B00015EF81110C9481580E947CB20C94815814
:10D4C00083E50E9428EE882341F00E94EAED8093D4
:10D4D000DC040E94A9EF0C9481580F94990B84E905
:10D4E00099E00E94A9F78091DC040E94BCF90C9499
:10D4F00081580E94966C0C9481580E94FA81811187
:10D500000C9481580C94776010918C040E947AC816
:10D51000609388107093891080938A1090938B1079
:10D52000112311F40C948158812F0E9427850C94AB
:10D530008158111107C011E089E50E9428EE082FDB
:10D54000811307C0012FF11204C011E001E0FF2494
:10D55000F39482E50E9476EE882311F40C9422590C
:10D560000E94FEED6CA37DA38EA39FA320E030E07C
:10D57000A9010F94FD2C882381F0111105C0011120
:10D5800003C0FF2009F417C160E0CE0184960E9419
:10D5900062300E949BF50E9465F5112309F47EC05C
:10D5A000002309F478C010924A0210924B021092A4
:10D5B0004C0210924D0210924E0210924F021092A5
:10D5C0005002109251020E946E318BE29FE00E9445
:10D5D0008BE84B015C018FE29FE00E948BE82B01FE
:10D5E0003C01AC019B01C501B4010F942D36181606
:10D5F00014F00C942859A5019401C301B2010F94B1
:10D60000C7349B01AC010F94632D20E030E040E86B
:10D610005FE30F94CD330F947B3620E030E048E495
:10D6200052E40F94632D68A379A38AA39BA320E0FF
:10D6300030E040EC5FE3C301B2010F94632D6983D6
:10D640007A838B839C8320E030E040EC5FE3C5016C
:10D65000B4010F94632D6C8F7D8F8E8F9F8FAE01E1
:10D66000405E5F4FBE016F5F7F4FCE014C960E94C0
:10D6700021300E94681F10924A0210924B021092B1
:10D680004C0210924D0210924E0210924F021092D4
:10D6900050021092510280E00E949733002319F04B
:10D6A00081E00E949733FF2009F485C010920A059B
:10D6B0001092090510920B0583E00E9474528111AB
:10D6C0007AC00E946E31209128073091290740913D
:10D6D0002A0750912B0760E070E080E393E40F94F9
:10D6E000CC332B013C0120912C0730912D07409128
:10D6F0002E0750912F0760E070E084E393E40F94CD
:10D70000CC334B015C018091520290915302A09165
:10D710005402B091550280939E0690939F06A09369
:10D72000A006B093A1060091961110919711D8010F
:10D730002D913D914D915C91C301B2010F94CC3379
:10D740006093960670939706809398069093990637
:10D75000F8012481358146815781C501B4010F94B8
:10D76000CC3360939A0670939B0680939C069093AB
:10D770009D0686E996E00E9485ED882311F40C94BD
:10D780002E591C8E1D8E1E8E1F8E88E0E6E9F6E057
:10D79000DE01119601900D928A95E1F7AE01445E8B
:10D7A0005F4FBE016B5F7F4FCE0101960E9421301B
:10D7B00082E00E9497330E946E318091C60580936B
:10D7C000C7058E2D0E94BCF10E948E2D0E949931BA
:10D7D0000C9481580F94950B84E199E00E94A9F76D
:10D7E0000C948158882309F4A6CEAFCEDF92EF9235
:10D7F000FF920F931F93CF93DF93EC01E090A80665
:10D80000F090A9068AE0D82E6AE070E0CE010F946D
:10D810001B378C01009711F0FC011082CE010E9491
:10D82000EB5081E00E9459560115110519F0E801ED
:10D83000D992EACFC701DF91CF911F910F91FF904D
:10D84000EF90DF900C94EB504F925F926F927F922B
:10D850008F929F92AF92BF92CF92DF92EF92FF9200
:10D860000F931F93CF93DF93CDB7DEB77C014DB6F7
:10D870005EB66090A8067090A9068DB69EB66AE066
:10D8800070E0C7010F94382C6C018C010E191F0930
:10D89000892B21F4C7010F944A2C8C01C8010196F1
:10D8A0002DB73EB7281B390B0FB6F8943EBF0FBEFD
:10D8B0002DBF8DB79EB701965C01A801B7010F94EB
:10D8C0006B2CF501E00FF11F1082C5010E94EB5097
:10D8D00081E00E945956C114D10451F076019FEFA6
:10D8E000E91AF90A0FB6F8949EBE0FBE8DBEC5CFD9
:10D8F0000FB6F8949EBE0FBE8DBEC3010E94EB50C2
:10D900000FB6F8945EBE0FBE4DBEDF91CF911F9152
:10D910000F91FF90EF90DF90CF90BF90AF909F90CE
:10D920008F907F906F905F904F9008954F925F928D
:10D930006F927F928F929F92AF92BF92CF92DF921F
:10D94000EF92FF920F931F93CF93DF93CDB7DEB784
:10D95000C059D1090FB6F894DEBF0FBECDBF0E94EB
:10D96000B7EF8823B9F183E50E9428EE882309F4F4
:10D9700049C088E994E00E94A9F78AE00E9481F7F3
:10D980008EEF8093980481E0809367021092970451
:10D9900081E09AE59093DA128093D9128CE490E0BA
:10D9A0009093DC128093DB1287E08093CD1282E8A3
:10D9B0008093D01284E890E0A0E0B0E08093D11290
:10D9C0009093D212A093D312B093D4128DE792E128
:10D9D0000E94AA37C057DF4F0FB6F894DEBF0FBEC4
:10D9E000CDBFDF91CF911F910F91FF90EF90DF900E
:10D9F000CF90BF90AF909F908F907F906F905F90EF
:10DA00004F90089583E40E9428EE882349F00E94F5
:10DA1000A1EF0E94F9820E944E820E945540DACF07
:10DA20008090DB079090DC07A090DD07B090DE07C8
:10DA30008091E40780FF05C09091080B9860909357
:10DA4000080B869581708093250882E495E00E94FA
:10DA5000246C80916A0790916B079E012F5F3F4F66
:10DA60007901009799F09F938F9389E395E09F93B5
:10DA70008F933F932F930F94942CC7010E94F66BC2
:10DA80000F900F900F900F900F900F90809168075C
:10DA900090916907009799F09F938F9380E395E0A9
:10DAA0009F938F93FF92EF920F94942CC7010E9443
:10DAB000F66B0F900F900F900F900F900F906E01DC
:10DAC00031E8C30ED11C60914707709148078091DF
:10DAD000490790914A07860123E041E00F94CA2745
:10DAE0009F938F938EE195E09F938F93FF92EF9298
:10DAF0000F94942CC7010E94F66B86E195E00E947A
:10DB0000246C87E080934A0B809386040F900F90DB
:10DB10000F900F900F900F90809163078823F9F07A
:10DB2000609164077091650780916607909167071F
:10DB300023E041E00F94CA279F938F938DE095E0F7
:10DB40009F938F93FF92EF920F94942CC7010E94A2
:10DB5000F66B0F900F900F900F900F900F90809199
:10DB60006C078823A1F01F928F931F921F9280E071
:10DB700095E09F938F93FF92EF920F94942CC7019F
:10DB80000E94F66B0FB6F894DEBF0FBECDBF80913A
:10DB90006D078823A9F01F928F931F9281E08F93C6
:10DBA00080E095E09F938F93FF92EF920F94942CD7
:10DBB000C7010E94F66B0FB6F894DEBF0FBECDBF53
:10DBC00040906E0750906F076090700770907107DB
:10DBD00020E030E0A901C301B2010F94FD2C8111B6
:10DBE00004C08091E40782FF20C0860121E041E06B
:10DBF000C301B2010F94CA279F938F938091E407CA
:10DC000082FB882780F91F928F9383EF94E09F9384
:10DC10008F93FF92EF920F94942CC7010E94F66BA2
:10DC20000FB6F894DEBF0FBECDBF6091390770917B
:10DC30003A0780913B0790913C078E010F581F4F88
:10DC400023E041E00F94CA27782E692E60913507B2
:10DC5000709136078091370790913807860123E04D
:10DC600041E00F94CA276F927F929F938F9382EE29
:10DC700094E09F938F93FF92EF920F94942CC7019F
:10DC80000E94F66B60913D0770913E0780913F07BF
:10DC90009091400723E041E00F94CA2787ED94E07C
:10DCA0000E94246CDF92CF928DEC94E09F938F932F
:10DCB000FF92EF920F94942CC7010E94F66B809113
:10DCC00046078F93809145078F9386EC94E09F934E
:10DCD0008F93FF92EF920F94942CC7010E94F66BE2
:10DCE00060914107709142078091430790914407EA
:10DCF00023E041E00F94CA279F938F938CEB94E02D
:10DD00009F938F93FF92EF920F94942CC7010E94E0
:10DD1000F66B8CE0EBE4F7E0A8E2B7E001900D923F
:10DD20008A95E1F78CE0E7E5F7E0ACE1B7E0019038
:10DD30000D928A95E1F780E00E94E61C81E00E9446
:10DD4000E61C82E00E94E61C8091E30780931607A0
:10DD500081E08093DC040E94A9EF82E797E09F9323
:10DD60008F938BED90E29F938F93FF92EF920F949E
:10DD7000942C0FB6F894DEBF0FBECDBFC7010E9432
:10DD8000F66B8091E2078F938091E1078F938091EA
:10DD9000E0078F938091DF078F93BF92AF929F929E
:10DDA0008F928EEA94E09F938F93FF92EF920F945D
:10DDB000942CC7010E94F66B0FB6F894DEBF0FBE1D
:10DDC000CDBF08CECF93DF93C091A40CC093FE07C4
:10DDD00081E6C89FE0011124CA55D34F8091080BFA
:10DDE00080FF05C00F94990BCE010E946352CE01B3
:10DDF0000E94EB5080E0DF91CF910C9459568BE15B
:10DE0000E3E6F3E1AEE7B3E101900D928A95E1F725
:10DE1000809143138062809343130895CF93809140
:10DE20003210C1E08823C9F08091331090913410F2
:10DE300040912A1050912B1060912C1070912D1050
:10DE4000DC01ED91FC910288F389E02D2AE23EE0AD
:10DE50001995C82F811104C0C0E08C2FCF9108956F
:10DE600040912E1050912F10609130107091311010
:10DE70004115510561057105B9F0809133109091FC
:10DE80003410DC01ED91FC910288F389E02D2AE247
:10DE90003EE01995882301F310922E1010922F1056
:10DEA000109230101092311010923210D6CF0F9382
:10DEB0001F93CF93DF93CDB7DEB760970FB6F8947B
:10DEC000DEBF0FBECDBF8C01DC01ED91FC91028065
:10DED000F381E02DBE016F5F7F4F1995882309F410
:10DEE00064C08981807CC9F56F81637070E0762F92
:10DEF0006627770F770F8885B4E08B9FC0011124C8
:10DF0000682B792B89858295869586958370682BF9
:10DF10006F5F7F4F90E080E02A852370220F3B8562
:10DF200037FB332730F9232B3E813F70230F3327F4
:10DF3000331F2750310904C0660F771F881F991FB0
:10DF40002A95D2F760960FB6F894DEBF0FBECDBF0C
:10DF5000DF91CF911F910F910895803419F5688555
:10DF60006695669570E090E080E0CB0177276627A4
:10DF70002A85622B098510E0102F0027012E000C46
:10DF8000220B330B602B712B822B932B6F5F7F4FF8
:10DF90008F4F9F4F4AE0660F771F881F991F4A9542
:10DFA000D1F7D0CF8BE0F801848360E070E0CB0143
:10DFB000C9CF0895FC01828108954F925F926F92BC
:10DFC0007F928F929F92AF92BF92EF92FF920F93A8
:10DFD0001F93CF93DF93B0E2A0E06A2F70E0AB0114
:10DFE0004B0F511D55954795411117C0E6E6FFE1CE
:10DFF00085919491282F822FDF91CF911F910F91BE
:10E00000FF90EF90BF90AF909F908F907F906F9018
:10E010005F904F900895B42FE2CFA41711F0B4137E
:10E0200003C0E2EEFFE1E4CF9A0121503109220F53
:10E03000331F220F331FF901EC59F04EE590F49095
:10E04000F901E859F04E059114918E159F051CF3C6
:10E05000A42F081719070CF4C0CFBC01F901EA5925
:10E06000F04EC591D491F901E659F04EA590B490C7
:10E070006E197F09072E000C880B990B0F94042D45
:10E080002B013C01B5016C1B7D0B072E000C880B8E
:10E09000990B0F94042D9B01AC01C301B2010F94A5
:10E0A000632D4B015C01B8016E197F09072E000C2E
:10E0B000880B990B0F94042D9B01AC01C501B40191
:10E0C0000F94C7344B015C01BE01DD0F880B990B27
:10E0D0000F94042D9B01AC01C501B4010F94CD3305
:10E0E0000F943935262F972F86CFEF92FF920F93FB
:10E0F0001F93E0920505F092060500930705109323
:10E1000008056093100570931105809312059FEF29
:10E11000FF27621B730B840B30F48095709561951B
:10E12000790B890B992790934815A6E06A9F009276
:10E130003C15512DEE277A9F500DE11D8A9FE00D71
:10E1400050933D15E0933E15AFE06A9F0092401555
:10E15000512DEE277A9F500DE11D8A9FE00D5093BF
:10E160004115E0934215AAE06A9F00924415512D93
:10E17000EE277A9F500DE11D8A9FE00D50934515C3
:10E18000E09346151F910F91FF90EF9008950000C6
:10E190008091C80580FF29C089988FEF80930C0675
:10E1A0008091C805869580FF23C08F988FEF80935C
:10E1B0000D068091C8058695869580FF1CC08091CC
:10E1C0000B0182708093090143988FEF80930E06B4
:10E1D0008091C80586958695869580FF15C016980E
:10E1E0008FEF80930F0600000895899A81E0D6CFC3
:10E1F0008F9A81E0DCCF80910B01809582708093B3
:10E200000901439A81E0E2CF169A81E0EACF0F93A9
:10E210001F93CF93811113C0C42F8B010F94990BBF
:10E2200080EC92E10E94A9F7C8010E94A9F7CC23D3
:10E2300031F08AE0CF911F910F910C9481F7CF912B
:10E240001F910F9108950F930091010521E002277E
:10E2500022E035E04CE050E0BC0182ED94E00E9409
:10E2600002F40F9108950F930091010521E0022718
:10E2700022E035E044E050E0BC0182ED94E00E94F1
:10E2800002F40F9108950F930091010521E00227F8
:10E2900022E035E041E050E0BC0182ED94E00E94D4
:10E2A00002F40F9108950F930091010521E00227D8
:10E2B00022E035E042E050E0BC0182ED94E00E94B3
:10E2C00002F40F9108950F930091010521E00227B8
:10E2D00022E035E041E050E0BC0182ED94E00E9494
:10E2E00002F40F9108950F930091010521E0022798
:10E2F00022E035E048E050E0BC0182ED94E00E946D
:10E3000002F40F9108950F930091010521E0022777
:10E3100022E035E04CE050E0BC0182ED94E00E9448
:10E3200002F40F9108950F9301E022E035E041E0FF
:10E3300050E0BC0182ED94E00E9402F40F91089538
:10E34000CF93DF93C9EFD0E18A819B810E94D1C036
:10E350009D838C83CEE8D0E18A819B810E94DD6F12
:10E360009D838C83A89510928406DF91CF910895A8
:10E370001F93CF93DF93182FEB010F94990B8AEF24
:10E3800091E20E94A9F786EE91E2113011F48CEE31
:10E3900091E20E94A9F7BE0182EF91E20F948B0BEC
:10E3A0008AE0DF91CF911F910C9481F7CF93DF9397
:10E3B000EC018D810F946B2060E08B81DF91CF9118
:10E3C0000C94E5C6DF92EF92FF920F931F93CF93C9
:10E3D000DF938C01C62FD22FF32EE42ED52E0E9470
:10E3E000D6710E940BE48C2F80640F945F208D2DDA
:10E3F0000F945F208E2D0F945F208F2D0F945F2040
:10E400008D2F0F945F2087E8C11101C085E90F941B
:10E410005F20CC3011F40F946420C0E00F9464208E
:10E42000F801868387FF04C0CF3F11F0CF5FF6CF9E
:10E43000DF91CF911F910F91FF90EF90DF900895A2
:10E4400061E0FC0183810E94E5C68FEF0D945F209F
:10E450000F931F93CF938C010E94D6710E940BE4FF
:10E46000C82F882371F08DEF0F945F200E940BE47A
:10E47000C82FC8010E9420728C2FCF911F910F913D
:10E48000089582E1F8018483F4CF8F929F92AF9236
:10E49000BF92CF92DF92EF92FF920F931F93CF9391
:10E4A000DF93EC016A017B01590120E030E0A90112
:10E4B00067E30E94E271A501980167E1CE010E9425
:10E4C000E271811127C08F81833039F089E0CC0C53
:10E4D000DD1CEE1CFF1C8A95D1F7A701960169E1AE
:10E4E000CE010E94E27111E0882319F010E087E06C
:10E4F0008C83CE010E942072812FDF91CF911F91DA
:10E500000F91FF90EF90DF90CF90BF90AF909F90D2
:10E510008F90089589E08C8310E0EBCFCF93DF9349
:10E52000EC016EBDFA01CA019E5F0DB407FEFDCF7E
:10E5300020812EBD0DB407FEFDCF21812EBD329668
:10E54000E817F90791F70DB407FEFDCF8FEF0F9491
:10E550005F208FEF0F945F200F9464208E838F7164
:10E56000853049F083E18C83CE010E94207280E0E7
:10E57000DF91CF91089581E0FBCF0F931F93CF934D
:10E58000DF93EC018B010E94D6710E940BE4811194
:10E590000CC085E18C8310E0CE010E942072812F97
:10E5A000DF91CF911F910F910895A8016CEFCE01DB
:10E5B0000E948E72182F882361F3EECF0F931F9362
:10E5C000CF93DF93EC0189018F81833039F089E0AB
:10E5D000440F551F661F771F8A95D1F79A01AB012B
:10E5E00068E1CE010E94E27181112AC0A8016EEF9C
:10E5F000CE010E948E72182F8823B1F00E940BE486
:10E60000182F8823D1F020E030E0A9016DE0CE0181
:10E610000E94E271882321F086E18C8310E004C01F
:10E620000F9464208111F8CFCE010E942072812FB7
:10E63000DF91CF911F910F91089587E18C83F4CFE3
:10E6400086E0EBCF1F93CF93DF93EC010E94D6714E
:10E6500020E030E0A9016CE0CE010E94E27111E0FF
:10E66000882319F010E083E08C83CE010E94207291
:10E67000812FDF91CF911F9108951F93CF93DF9347
:10E68000EC018F81833039F089E0440F551F661FFC
:10E69000771F8A95D1F79A01AB0162E1CE010E9402
:10E6A000E27111E0882319F010E085E08C83CE013F
:10E6B0000E942072812FDF91CF911F9108958F9238
:10E6C0009F92AF92BF92EF92FF920F931F93CF93BF
:10E6D000DF938C01EB017A010E947AC84B015C0147
:10E6E0002CE2820E21E0921EA11CB11C0F9464202A
:10E6F000F80186838F3F69F40E947AC86819790906
:10E700008A099B0997FDF2CF81E1F8018483C0E07B
:10E7100021C08E3F71F5F1E0EF1AF1088FEF8EBD49
:10E72000FE012FEF0DB407FEFDCF8EB581932EBDF8
:10E73000CF018C1B9D0B8E159F05A0F30DB407FE1A
:10E74000FDCF8EB5CE0DDF1D88830F9464200F940E
:10E750006420C1E0C8010E9420728C2FDF91CF910C
:10E760001F910F91FF90EF90BF90AF909F908F906F
:10E7700008958FE0CACF0F931F93CF93DF93EC01DF
:10E780008B010E94D67140E052E0B801CE01DF91CA
:10E79000CF911F910F910C945F730F931F93CF93A1
:10E7A000DF93EC0189018F81833039F089E0440FD8
:10E7B000551F661F771F8A95D1F79A01AB0161E15A
:10E7C000CE010E94E27181110AC040E052E0B8011E
:10E7D000CE01DF91CF911F910F910C945F7384E074
:10E7E0008C83CE010E94207280E0DF91CF911F9137
:10E7F0000F9108958F929F92AF92BF92CF92DF9226
:10E80000EF92FF920F931F93CF93DF93EC01162F9C
:10E810001F821C824B830E947AC86B017C0120ED11
:10E82000C20E27E0D21EE11CF11CA89561E08B818D
:10E830000E94E5C68B810E9434B2209A289A219AC0
:10E840002398229A81E00F946B2085E08D830F94AA
:10E850006B200AE08FEF0F945F200150D9F7A89545
:10E8600020E030E0A90160E0CE010E94E2718E83D9
:10E87000813081F00E947AC86C197D098E099F0948
:10E8800097FDEECF81E08C83CE010E9420721A8228
:10E8900080E06AC0A8952AEA31E040E050E068E0F4
:10E8A000CE010E94E271853041F581E08F83A89509
:10E8B0008F81812C912C5401823029F4812C912C50
:10E8C000A12C80E4B82E20E030E0A90167E3CE015E
:10E8D0000E94E271A501940169E2CE010E94E271F9
:10E8E0008E838823F1F00E947AC86C197D098E0905
:10E8F0009F0997FDE8CF8AE0C6CF04E00F9464201B
:10E900008E830150D9F78A3A11F482E0CFCF0E946A
:10E910007AC86C197D098E099F0997FDBCCF82E0EA
:10E92000B2CF8F818230C1F420E030E0A9016AE3E8
:10E93000CE010E94E271882311F088E0A4CF0F94E9
:10E940006420807C803C11F483E08F830F946420EA
:10E950000F9464200F946420CE010E94207281E005
:10E960008A83173070F41D83DF91CF911F910F912F
:10E97000FF90EF90DF90CF90BF90AF909F908F90DF
:10E98000089588E18C8384CF0F931F93CF93DF93F7
:10E99000EC018B0120E030E0A90169E00E94E27106
:10E9A00081110AC040E150E0B801CE01DF91CF9162
:10E9B0001F910F910C945F7380E18C83CE010E94B4
:10E9C000207280E0DF91CF911F910F9108951F92E7
:10E9D0000F920FB60F9211242F933F938F939F9313
:10E9E000AF93BF9380918E0690918F06A091900671
:10E9F000B091910630918D0623E0230F2D3758F505
:10EA00000196A11DB11D20938D0680938E069093D3
:10EA10008F06A0939006B0939106809192069091F4
:10EA20009306A0919406B09195060196A11DB11D83
:10EA30008093920690939306A0939406B0939506C4
:10EA4000BF91AF919F918F913F912F910F900FBEEA
:10EA50000F901F90189526E8230F0296A11DB11D57
:10EA6000D2CFCF92DF92EF92FF920F931F93CF936B
:10EA7000DF93CDB7DEB7A0970FB6F894DEBF0FBE19
:10EA8000CDBF442309F445C0611571058105910589
:10EA900079F100E0C42ED12CF12CE12CA7019601D4
:10EAA0000F94413311E0100FE1E0F0E0EC0FFD1F97
:10EAB000E00FF11D07FDFA956083B901CA01012F2E
:10EAC000611571058105910549F7115010F1E1E0DB
:10EAD000F0E0EC0FFD1FE10FF11D17FDFA9590819D
:10EAE00087E39A3008F480E3890F0E9481F7EDCF25
:10EAF00080E3A0960FB6F894DEBF0FBECDBFDF91C6
:10EB0000CF911F910F91FF90EF90DF90CF900C94D9
:10EB100081F7A0960FB6F894DEBF0FBECDBFDF9190
:10EB2000CF911F910F91FF90EF90DF90CF900895BC
:10EB3000809138138823C1F0815080933813E3E625
:10EB4000F3E1882351F08150990B2BE1289FF001CC
:10EB5000299FF00D1124E756FC4E8BE1AEE7B3E19F
:10EB600001900D928A95E1F780913813811105C0CB
:10EB7000909143139062909343130895CF92DF9244
:10EB8000EF92FF928091431382FF29C0C0903F1300
:10EB9000D0904013E0904113F090421381EB91E24A
:10EBA0000E94A9F74AE0C701B6010E9431758FE2C1
:10EBB0000E9481F760913B1370913C1380913D134B
:10EBC00090913E134AE00E9431758DE00E9481F7DA
:10EBD0008AE0FF90EF90DF90CF900C9481F783EC68
:10EBE00091E2FF90EF90DF90CF900C94A9F7BC01D9
:10EBF00085EE90E20F948B0B82EE90E20C94A9F7D5
:10EC00008091431383FF03C084608093431308956E
:10EC1000CF92DF92EF92FF920F931F93CF93DF93E8
:10EC2000CDB7DEB7EDB6FEB6DC010D900020E9F7FA
:10EC30009D01281B390B285F3F4FEDB7FEB7E21B44
:10EC4000F30B0FB6F894FEBF0FBEEDBF0DB71EB7A6
:10EC50000F5F1F4F9F938F938BED90E29F938F9346
:10EC60001F930F930F94942C6801F4E0CF0ED11CE6
:10EC70000F900F900F900F900F900F90D6018D91E5
:10EC80006D01882349F0082E000C990B0F94DF3694
:10EC9000F60131978083F2CF66ED70E2C8010F94E0
:10ECA0002D2C4FE350E0B8018AEC95E00F943B37F0
:10ECB0000FB6F894FEBE0FBEEDBEDF91CF911F914F
:10ECC0000F91FF90EF90DF90CF900895FC01938516
:10ECD00091FD13C0987121E0903109F020E08091FE
:10ECE000431320FB84F980934313903141F08085D6
:10ECF000873419F481858E3711F480E0089581E01E
:10ED00000895FC0120E03EE2DB014D91BD0140325F
:10ED100049F0283011F430833196DB0111974C9182
:10ED2000408331962F5F2B3079F710820895EF9250
:10ED3000FF920F931F93CF93DF93CDB7DEB7A097CA
:10ED40000FB6F894DEBF0FBECDBF7C018B01BE01B4
:10ED50006F5F7F4FC7010E9468AC1816A4F4CE0104
:10ED600001960E946676882391F3BE016F5F7F4F04
:10ED700084EA90E10E94817664EA70E1C8010F9410
:10ED8000FD36892B21F7A0960FB6F894DEBF0FBE93
:10ED9000CDBFDF91CF911F910F91FF90EF9008951C
:10EDA000CF92DF92EF92FF92CF936B017C01C42F41
:10EDB00080912A1090912B10A0912C10B0912D10C1
:10EDC0008C159D05AE05BF0529F10E940E6F8111BE
:10EDD00008C0C0E08C2FCF91FF90EF90DF90CF90D4
:10EDE00008958091331090913410DC01ED91FC91E5
:10EDF0000088F189E02D2AE23EE0B701A6011995CD
:10EE0000882339F3C0922A10D0922B10E0922C1054
:10EE1000F0922D10CC2321F081E080933210DACFD4
:10EE2000C1E0D8CF4F925F926F927F928F929F9264
:10EE3000AF92BF92CF92DF92EF92FF920F931F9308
:10EE4000CF93DF93EC01423051056105710590F4D9
:10EE500080E0DF91CF911F910F91FF90EF90DF90B5
:10EE6000CF90BF90AF909F908F907F906F905F906A
:10EE70004F90089589859A85AB85BC850196A11D23
:10EE8000B11D84179507A607B70710F38F89803146
:10EE9000C9F5852E962EA72EBB248B899C89AD891A
:10EEA000BE89880E991EAA1EBB1E280139016A015F
:10EEB0007B0141E0C501B4010E94D076882341F274
:10EEC0009F89903181F5DD24EE24FF24F601EE0FB9
:10EED000FF1FE65DF14F118300839A89923008F499
:10EEE000B8CF4D815E816F817885840E951EA61EF8
:10EEF000B71E80922E1090922F10A0923010B092D8
:10EF00003110A7CF803209F0A3CF8B899C89AD89BE
:10EF1000BE894A015B01E7E0B694A7949794879471
:10EF2000EA95D1F7BECFE894C7F8DD24EE24FF249C
:10EF3000F601EE0FFF1FEE0FFF1FE65DF14F40825F
:10EF4000518262827382C9CFCF92DF92EF92FF9299
:10EF50000F931F93CF93DF93FC0181859285A38547
:10EF6000B4850196A11DB11D84179507A607B707A3
:10EF700050F480E0DF91CF911F910F91FF90EF90BF
:10EF8000DF90CF90089587898031A9F5BB27A72FFF
:10EF9000962F852FC388D488E588F6888C0D9D1D13
:10EFA000AE1DBF1DE9016A017B018F0140912A104E
:10EFB00050912B1060912C1070912D108417950793
:10EFC000A607B70749F5F8018789803169F5B701C8
:10EFD000A601552766277727440F551F465D514FD9
:10EFE000FA0180819181B0E0A0E088839983AA83AF
:10EFF000BB8381E0BFCF803209F0BBCFC388D48808
:10F00000E588F688DB01CA01C7E0B695A795979514
:10F010008795CA95D1F7C2CF40E0BC01CD010E94CF
:10F02000D0768111D0CFA5CFB701A6014F77552754
:10F0300066277727440F551F440F551F465D514FD4
:10F04000FA0180819181A281B381BF70CECF4F92AE
:10F050005F926F927F92AF92BF92CF92DF92EF92C8
:10F06000FF920F931F93CF93DF9300D01F92CDB7E2
:10F07000DEB78C0149835A836B837C835901C12C91
:10F08000D12C7601412C82E0582E612C712C4981C3
:10F090005A816B817C819E012F5F3F4FC8010E9486
:10F0A000A477882319F1F8018585A301920104C092
:10F0B000220F331F441F551F8A95D2F7DA01C90169
:10F0C000C80ED91EEA1EFB1E49815A816B817C81C4
:10F0D00087898031F1F481E0483F5F4F6105710518
:10F0E000B0F2F501C082D182E282F3820F900F90DC
:10F0F0000F900F90DF91CF911F910F91FF90EF90A4
:10F10000DF90CF90BF90AF907F906F905F904F90C7
:10F11000089581E0483F5F4F6F4F7F4008F4B7CFBD
:10F12000E0CF0F931F93CF93DF93FC012381222322
:10F1300031F080E0DF91CF911F910F9108958B0105
:10F14000EC01FB018789803139F582E08B831D8AD0
:10F150001E8A1F8A188E808D918DB0E0A0E025E078
:10F16000880F991FAA1FBB1F2A95D1F7898B9A8BED
:10F17000AB8BBC8B1A8F098F81E089831886198627
:10F180001A861B861C821D821E821F82188A1C867C
:10F190001D861E861F86CECF803259F683E08B8374
:10F1A000428D538D648D758D4D8B5E8B6F8B788FFB
:10F1B0009E012F5E3F4FC8010E9427788111DACF50
:10F1C000B8CF3F924F925F926F927F928F929F92B1
:10F1D000AF92BF92CF92DF92EF92FF920F931F9365
:10F1E000CF93DF93CDB7DEB72C970FB6F894DEBF81
:10F1F0000FBECDBF5C01DC0159968D909C90F4014F
:10F2000081859285A385B4859C01AD012F5F3F4F19
:10F210004F4F5F4F29873A874B875C87D5011496FC
:10F220004D905D906D907C9017974114510461044E
:10F23000710409F459C0BFEF4B1A5B0A6B0A7B0AD1
:10F24000312C730162011D821E821F821886F40117
:10F2500081859285A385B4852D813E814F81588516
:10F26000281739074A075B0708F056C089859A8531
:10F27000AB85BC858C159D05AE05BF0550F482E0BD
:10F28000C82ED12CE12CF12C92E0492E512C612C6E
:10F29000712C9E012F5F3F4FB701A601C4010E9450
:10F2A000A4778823C9F189819A81AB81BC81892B9C
:10F2B0008A2B8B2B01F1260137019FEF491A590A3E
:10F2C000690A790A2D813E814F8158852F5F3F4F12
:10F2D0004F4F5F4F2D833E834F8358873FEFC31AB5
:10F2E000D30AE30AF30AB3CF40805180628073806F
:10F2F00033243394A6CFC414D504E604F70411F7DD
:10F300000FEF1FEF2FEF3FE0B701A601C4010E94EE
:10F310001277782E81111AC0712C872D2C960FB67A
:10F32000F894DEBF0FBECDBFDF91CF911F910F913B
:10F33000FF90EF90DF90CF90BF90AF909F908F9015
:10F340007F906F905F904F903F900895F5014481BA
:10F35000558166817781411551056105710539F047
:10F3600097018601C4010E9412778823A9F2D50172
:10F370001496CD92DD92ED92FC921797332051F0C6
:10F38000D701C6010196A11DB11DF40180839183AF
:10F39000A283B383F50185899689A789B08D892BCE
:10F3A0008A2B8B2B09F0B9CFC58AD68AE78AF08ED3
:10F3B000818180688183B1CFCF93DF93EC01462FA9
:10F3C00041706C857D858E859F850E94D0768823CF
:10F3D00051F0888920E2829FC0011124865D914FFF
:10F3E000DF91CF91089590E080E0FACFCF93DF9343
:10F3F000EC018991882319F00E9481F7FACFDF91FF
:10F40000CF910895CF93DF93EC018B81882349F14D
:10F41000898187FF22C061E0CE010E94DC79FC0176
:10F42000892BF9F08081853EE1F08B81823040F4B8
:10F4300089899A89AB89BC89848F958FA68FB78F6C
:10F440008D899E89938F828F8D899E89AF89B88D92
:10F45000B58BA48B89818F778983DF91CF910C94B1
:10F460000E6F81E0888380E0DF91CF9108958F92C5
:10F470009F92AF92BF92CF92DF92EF92FF920F9343
:10F480001F93CF93DF93EC018B8181110EC080E03D
:10F49000DF91CF911F910F91FF90EF90DF90CF9070
:10F4A000BF90AF909F908F90089509891A892B89FA
:10F4B0003C89041715072607370748F34A015B0103
:10F4C000823031F488869986AA86BB8681E0E0CFB7
:10F4D00081149104A104B10449F4188619861A868E
:10F4E0001B861C821D821E821F82F0CF0885198513
:10F4F0002A853B85E98DFA8D858590E00996B901CD
:10F50000A8014150510961097109082E04C076957E
:10F510006795579547950A94D2F775016401E1E024
:10F52000CE1AD108E108F10804C0F694E794D79404
:10F53000C7948A95D2F7C416D506E606F70620F0DA
:10F54000012B022B032B11F58D899E89AF89B88D74
:10F550008C839D83AE83BF838E010C5F1F4FC114CC
:10F56000D104E104F10409F4ADCF4C815D816E81D9
:10F570007F819801898D9A8D0E94A47791E0C91AA4
:10F58000D108E108F1088111EACF81CFC41AD50A68
:10F59000E60AF70AE1CF2F923F924F925F926F9265
:10F5A0007F928F929F92AF92BF92CF92DF92EF9213
:10F5B000FF920F931F93CF93DF9300D01F92CDB78D
:10F5C000DEB78C014B011A01DC0113968C91139765
:10F5D000813009F0CFC011968C9181FFCBC082FDA4
:10F5E000B5C06101D80118964D915D916D917C91E6
:10F5F0001B97C114D10409F41BC159968D919C919C
:10F600005A97FC0174802FEF270D2A013B0139E046
:10F6100076946794579447943A95D1F7722E742054
:10F620007A01F1E0FF22711020C0E114F104E9F445
:10F6300014964D915D916D917C91179741155105EF
:10F640006105710509F09CC055968D919D910D90B5
:10F65000BC91A02D0097A105B10509F0AAC0C80171
:10F660000E94E178882309F485C0A12C82E0B82E9D
:10F67000AE18BF08CA14DB0408F45601D801599625
:10F680004D915C915A9714968D919D910D90BC91DE
:10F69000A02D0297A109B109FA01258504C0880FA0
:10F6A000991FAA1FBB1F2A95D2F7468557856089E7
:10F6B0007189840F951FA61FB71F9C01AD01270DEF
:10F6C000311D411D511D29013A01A11432E0B3063B
:10F6D00009F07DC080912A1090912B10A0912C10E0
:10F6E000B0912D10481659066A067B0669F41092EF
:10F6F00032108FEF9FEFDC0180932A1090932B1034
:10F70000A0932C10B0932D10809133109091341051
:10F71000DC01ED91FC910288F389E02D9401B301A5
:10F72000A2011995882331F1F80180859185A28580
:10F73000B3858A0D9B1DA11DB11D80879187A2876E
:10F74000B3878A0C9B1CCA18DB084CCFF80141898F
:10F7500052896389748980859185A285B38548170C
:10F7600059076A077B0709F43CCFC8010E94377A22
:10F77000811137CF81E0D8018C938FEF9FEF6EC05E
:10F780009E012F5F3F4F0E94A477882399F38981C0
:10F790009A81AB81BC81F801218D328DF9012789D5
:10F7A000203169F4883FFFEF9F07A105B10508F0FC
:10F7B00056CFF80184839583A683B78356CF883FBD
:10F7C0002FEF9207A2072FE0B20798F348CFE1147A
:10F7D000F10431F5F8014085518562857385818991
:10F7E0009289A389B489481759076A077B07C0F033
:10F7F0000E940E6F882309F4BDCF81E08093321000
:10F8000040922A1050922B1060922C1070922D1062
:10F81000A501B401C701865D914F0F94F43684CFE2
:10F8200041E0C301B2010E94D0768111F1CFA2CF95
:10F83000F80181899289A389B48984179507A6075D
:10F84000B70738F48181418B528B638B748B80684E
:10F850008183F801818183FD18C0C1010F900F9051
:10F860000F900F90DF91CF911F910F91FF90EF902C
:10F87000DF90CF90BF90AF909F908F907F906F90D0
:10F880005F904F903F902F900895C8010E94027A98
:10F890008111E3CF6FCF2F923F924F925F926F9281
:10F8A0007F928F929F92AF92BF92CF92DF92EF9210
:10F8B000FF920F931F93CF93DF93EC014B017A01DB
:10F8C0008B81811115C08FEF9FEFDF91CF911F9139
:10F8D0000F91FF90EF90DF90CF90BF90AF909F90EF
:10F8E0008F907F906F905F904F903F902F900895F2
:10F8F000898180FFE8CF89899A89AB89BC8948854D
:10F9000059856A857B85841B950BA60BB70BA701D0
:10F9100070E060E084179507A607B70708F47C013C
:10F9200067011E0124E0220E311CC114D10409F428
:10F93000A9C0488559856A857B855A0181E0B8222E
:10F94000898D9A8D2A013B0129E07694679457941A
:10F9500047942A95D1F72B81FC01223081F5628DE5
:10F96000738D848D958D640D751D861D971D00E02A
:10F9700012E00A191B09C016D10608F48601011508
:10F98000E2E01E0771F440902A1050902B10609016
:10F990002C1070902D10641575058605970509F0DB
:10F9A0004EC040E00E94D076882309F48CCFB50188
:10F9B000665D714FA801C4010F94F43652C01481E2
:10F9C00011501421A114B10471F411110CC0452B74
:10F9D000462B472B51F58D899E89AF89B88D8C8335
:10F9E0009D83AE83BF83E98DFA8D4C805D806E80F0
:10F9F0007F8022E0421A510861087108858504C0A1
:10FA0000440C551C661C771C8A95D2F78685978511
:10FA1000A089B189480E591E6A1E7B1EC301B2011E
:10FA2000610F711D811D911DA2CF4C815D816E8181
:10FA30007F8191010E94A4778111D5CF44CFA091FD
:10FA40003310B0913410ED91FC9111970088F18939
:10FA5000E02D9401AB01BC01CD011995882309F477
:10FA600032CF800E911E88859985AA85BB85800F2F
:10FA7000911FA11DB11D88879987AA87BB87C01ACE
:10FA8000D10A53CFC70121CFCF93DF93EB01FC0104
:10FA90002381211104C080E0DF91CF91089522508D
:10FAA000223028F48FE28883198281E0F5CF60E06C
:10FAB0000E94DC79009779F3DC0160E080E09EE24F
:10FAC0002D91203299F0883031F49E01260F311D9E
:10FAD000F90190836F5F9E01260F311DAD014150EA
:10FAE0005109FA014081F90140836F5F8F5F8B30CC
:10FAF00039F7FE01E60FF11D1082D7CFCF93DF93C8
:10FB0000EC01CB01E881F981608171810E94447D23
:10FB100028813981D901ED91FC91AA81BB818C9119
:10FB20009081992359F08936C8F4CF010196F901E3
:10FB3000918380838C918F5F8C93EACF893670F4A8
:10FB40008FE28083E881F9818081918101969183A0
:10FB50008083EA81FB8180818F5F8083DF91CF91F9
:10FB600008950F931F93CF93DF9300D000D01F927F
:10FB7000CDB7DEB79C012F5F3F4F3F832E832FE22F
:10FB8000FC01208381E08D83CE0106969A838983D0
:10FB900001979C838B8310E00BE180913813181739
:10FBA00058F4109FB001112467567C4ECE01019687
:10FBB0000E947E7D1F5FF1CF8D818B3558F467EAFF
:10FBC00074E1CE0101960E947E7D8E819F81019716
:10FBD0009F838E83EE81FF81108227960FB6F89463
:10FBE000DEBF0FBECDBFDF91CF911F910F91089562
:10FBF000CF93DF93EC010E94027A1B82DF91CF91B9
:10FC0000089510923510809143138F7B8B7F8093E2
:10FC100043130E94D8F3882321F087EA94E10C94DF
:10FC2000F87D08958091431382FF0AC08064809319
:10FC3000431380914313877F806280934313089519
:10FC40000E94017EF6CFCF93DF9380914313877F8D
:10FC50008093431380916613882321F083E693E118
:10FC60000E94F87D8091441390914513DC01ED9141
:10FC7000FC910190F081E02D45E360E01995811140
:10FC80000EC00F94990B8AEC90E20E94A9F7809124
:10FC9000431383FF30C0DF91CF910C94FF6EC0916E
:10FCA0004413D091451361E0CE010E94CEB0811182
:10FCB0000BC060E0CE010E94CEB0811105C00F9450
:10FCC000950B86EB90E2E1CF6EE071E183E693E184
:10FCD0000E949178811105C00F94950B85EA90E2FE
:10FCE000D4CF809143138860809343130F94990B72
:10FCF00089E990E2CACF80910B06882339F06FEF33
:10FD00008CE890E2DF91CF910C947A3CDF91CF9117
:10FD1000089540E050E0BA010C94377A0F931F9396
:10FD2000CF93DF93CDB7DEB7EB970FB6F894DEBF76
:10FD30000FBECDBF8091431300E010E083FF23C0CE
:10FD40008EE793E10E94897E8BE1EEE7F3E1DE012D
:10FD5000919601900D928A95E1F710E000E0BE01C6
:10FD60006F5F7F4FCE0181960E9468AC18163CF4FD
:10FD7000CE0101960E946676080F111DF0CFCE01CC
:10FD800081960E94C9EFC801EB960FB6F894DEBFCA
:10FD90000FBECDBFDF91CF911F910F9108950F93AB
:10FDA0001F93CF93DF93CDB7DEB76B970FB6F89461
:10FDB000DEBF0FBECDBF8C018EE793E10E94897E2E
:10FDC0008BE1EEE7F3E1DE01119601900D928A9549
:10FDD000E1F7B801CE0101960E949776CE01019617
:10FDE0000E94C9EF6B960FB6F894DEBF0FBECDBF71
:10FDF000DF91CF911F910F9108954F925F926F9273
:10FE00007F92AF92BF92CF92DF92EF92FF920F93C9
:10FE10001F93CF93DF931F92CDB7DEB78C017B0189
:10FE20005A01C22EDB0159968D919C91F801928F57
:10FE3000818FCB010E94897E712CF701808591858D
:10FE4000A285B3854189528963897489841795078E
:10FE5000A607B70708F052C055E0B695A795979545
:10FE600087955A95D1F7F82FFF70DF2ED70113969B
:10FE70008C91823010F480E0DBC041E050E0BE01A4
:10FE80006F5F7F4FC7010E944B7C0197A1F7F7017D
:10FE900080859185A285B3854F96A11DB11D808770
:10FEA0009187A287B387F0E2DF9EB0011124665DDF
:10FEB000714F61157105F9F2DB018C91882341F0D6
:10FEC000853E09F04CC0772029F077247394B5CF94
:10FED00071100EC080912A1090912B10A0912C10BF
:10FEE000B0912D10F80184879587A687B787D08AAF
:10FEF000DB018C918111E9CF772473948C2D82746E
:10FF0000823409F0B8CF772009F4A2C0F801D08874
:10FF100061E0C8010E94DC79009709F4ACCF20E2CF
:10FF2000DC011D922A95E9F72BE0F501DC01019037
:10FF30000D922A95E1F721E238E2FC01318B208B0A
:10FF400040E058E057874687338B228B318F208FD4
:10FF5000578B468B0E940E6F811109C08CCF4BE0EE
:10FF600050E0C5010F94E736892B09F066CFF0E227
:10FF7000DF9ED00111249D01265D314FF90183855B
:10FF8000817121F08C2D827109F001C1F801818D00
:10FF9000928D40912A1050912B1060912C107091ED
:10FFA0002D104487558766877787D08AFD01E65DE7
:10FFB000F14F44885588712C612C3201552444241A
:10FFC000D80155964D925D926D927C925897428DD4
:10FFD000538D70E060E044295529662977295596AC
:10FFE0004D935D936D937C935897D9011B962C91FB
:10FFF000287109F0BEC0848D958DA68DB78DF8014E
:020000021000EC
:10000000818B928BA38BB48B81E083838C2D8F703B
:10001000F801818314821582168217821086118658
:100020001286138681E0C4FE03C0C8010E948DAD14
:100030000F90DF91CF911F910F91FF90EF90DF9084
:10004000CF90BF90AF907F906F905F904F9008954A
:10005000D70113968C911397823009F40CCF5196E7
:100060008D919D910D90BC91A02D803E9F4FAF41F1
:10007000B10508F000CFC7010E94E178882309F498
:10008000FACE0E940E6F882309F4F5CED701599657
:10009000ED91FC915A9714964D905D906D907C90E7
:1000A0001797B2E04B1A510861087108858504C0A2
:1000B000440C551C661C771C8A95D2F7868597855B
:1000C000A089B189480E591E6A1E7B1E81E080936B
:1000D000321040922A1050922B1060922C10709285
:1000E0002D10EAE2FEE080E092E0DF019C011D922B
:1000F00021503040E1F7DD24D394D7015996ED919A
:10010000FC918481D816C0F4809133109091341002
:10011000DC01ED91FC910288F389E02D2AE23EE0BA
:10012000B301A2014D0D511D611D711D199588234B
:1001300009F4A1CED394E1CF258580E092E0A0E040
:10014000B0E004C0880F991FAA1FBB1F2A95D2F7E1
:10015000F7014189528963897489840F951FA61F0D
:10016000B71F818B928BA38BB48B8AE29EE0D12C3C
:10017000D6CE203161F498012F5E3F4F0E94277840
:10018000882329F084E0D80113968C933FCFD801BF
:1001900013961C9270CE2F923F924F925F926F9265
:1001A0007F928F929F92AF92BF92CF92DF92EF9207
:1001B000FF920F931F93CF93DF93CDB7DEB7C35456
:1001C000D1090FB6F894DEBF0FBECDBF4C015B0165
:1001D0006A01222E19821C821C8E1F8E61157105E8
:1001E00021F510E0CE014C960E94C9EFCE01019698
:1001F0000E94C9EF812FCD5BDF4F0FB6F894DEBFB1
:100200000FBECDBFDF91CF911F910F91FF90EF9067
:10021000DF90CF90BF90AF909F908F907F906F9026
:100220005F904F903F902F900895FC018381811142
:10023000D8CFFA0180818F32A1F18B01CE010196D6
:100240007C013C0180E2382E2E019CE1490E511CBC
:100250002396EFAE23972496FFAE249722963FAEC7
:10026000229721963FAE21973FAE3EAE3DAE3CAECB
:100270003BAE3AAE39AE38AE3FAA960190E047E0C9
:10028000D9018D91882309F447C08F3209F444C005
:100290008E3209F54A3009F4A4CF98E04AE09D0176
:1002A000EFCFFB01838182508B01823060F0618D42
:1002B000728DCE014C960E9491788E01045E1F4F84
:1002C000882309F48ECFC6016C010196F6012081C6
:1002D0002F32D1F3B3CFE8E6F0E22491222321F0CC
:1002E00031968213FACF7DCF491708F47ACF813245
:1002F00008F477CF8F3709F474CF3FE9380F3A31DC
:1003000008F420EEE7E3F0E0EC0FFD1FE90FF11D2C
:10031000820F80839F5FC3CF8FA9803209F461CFA2
:100320006901F90180812F5F3F4F8F32C9F3882324
:1003300001F121E0AE01495C5F4FB801C7010E94A5
:10034000FD7E882309F44DCF0A151B0519F0C8015D
:100350000E94F87D942D852D6E147F0431F0239634
:100360009FAD239724968FAD24978701E92EF82E11
:1003700075CF222DAE01495C5F4FB801C4010E94C8
:10038000FD7E182F2FCF1F93CF93DF93CDB7DEB70E
:100390006D970FB6F894DEBF0FBECDBF1D8E1C8EBD
:1003A000AC01BE01645E7F4F80E00E94CBAF10E0E5
:1003B0000097A9F019821C826C8D7D8D21E0AC0123
:1003C000CE0101960E94CB80182F882321F0CE0108
:1003D00001960E94F87DCE0101960E94C9EF812FFF
:1003E0006D960FB6F894DEBF0FBECDBFDF91CF91F3
:1003F0001F910895EF92FF921F93CF93DF9300D048
:1004000000D000D01F92CDB7DEB78091431383FF99
:100410000E94237E8091431383FF3CC00E94B7EF6C
:10042000811138C08091391390E08F969F938F93FC
:100430008FEF91E29F938F93CE0101967C019F9362
:100440008F930F94942C809143130F900F900F90E3
:100450000F900F900F9083FF1DC0C7010E94C381B2
:10046000182F8823B9F00E94FF6EC7010E940876FA
:10047000809139138F5F80933913812F2A960FB69D
:10048000F894DEBF0FBECDBFDF91CF911F91FF90DB
:10049000EF9008951092391310E0EFCF81E0809330
:1004A00039130C94FA81CF939091431393FF23C097
:1004B00090914B1391111FC02AE5811121E0C82FA3
:1004C00042EF52E063E673E188E493E10E94CB805F
:1004D000811105C082EF92E0CF910C94F775C111A4
:1004E0000AC062EF72E084ED91E20F948B0B8AE018
:1004F000CF910C9481F7CF910895CF9321E042EFF3
:1005000052E063E673E188E493E10E94CB80C82F58
:10051000882321F088E493E10E94F87D8C2FCF910D
:100520000895FF920F931F93CF93DF93CDB7DEB75C
:100530006D970FB6F894DEBF0FBECDBF2091431369
:1005400023FF2DC0AC01BE01645E7F4F80E00E949E
:10055000CBAF8C01009719F16C8D7D8D19821C82B7
:1005600022E0AC01CE0101960E94CB80811123C014
:10057000F12CCE0101960E94C9EFB801FF2081F154
:1005800083EA91E20F948B0B8AE00E9481F710922C
:100590003F131092401310924113109242136D9624
:1005A0000FB6F894DEBF0FBECDBFDF91CF911F9184
:1005B0000F91FF900895CE0101960E948DAD882382
:1005C000B9F261E0CE0101960E94DC79009781F2D8
:1005D00025EEFC0120831C820E940E6FF82EC9CFED
:1005E0008BE891E20F948B0B88E891E20E94A9F7C7
:1005F000D6CF0E947D82882331F00E94A1EF82EF46
:1006000092E00C94918208950F931F93CF93DF9300
:100610001F921F92CDB7DEB72091431323FF32C044
:100620008C01BC0182E00E94B87110923A130E94C2
:10063000017EA801BE016F5F7F4F80E00E94CBAFBB
:100640008C010097F9F069817A8126E5AC0187EA8F
:1006500094E10E94CB808823E1F080914313816074
:1006600080934313C8010E94CF7E10923713B801C4
:1006700084ED91E20F948B0B8AE00E9481F7C80110
:100680000E9464AF0F900F90DF91CF911F910F9157
:100690000895C8010E94F775F5CFCF92DF92EF92CF
:1006A000FF920F931F93CF93DF931F921F92CDB7AB
:1006B000DEB72091431323FF62C08C01613009F43F
:1006C00070C008F467C0623009F4CFC00E94017E98
:1006D000A801BE016F5F7F4F81E00E94CBAF8C010C
:1006E000009709F44CC069817A8121E0AC0187EA66
:1006F00094E10E94CB80882309F4BEC08091B81495
:100700009091B914A091BA14B091BB1480933B138B
:1007100090933C13A0933D13B0933E1310923F135C
:10072000109240131092411310924213B80180E1CD
:1007300091E20F948B0BC0903B13D0903C13E09050
:100740003D13F0903E1388E091E20E94A9F74AE041
:10075000C701B6010E9431758AE00E9481F789EFD6
:1007600090E20E94A9F7C8010E94CF7E8091B1104B
:10077000882311F001EB10E1C8010E9464AF0F90D3
:100780000F90DF91CF911F910F91FF90EF90DF902D
:10079000CF900895BC0182E00E94B87110923A1384
:1007A00095CF0E94D8F3811105C0B80181E00E9465
:1007B000B8718CCF80913A13882391F00F94950BE8
:1007C00061E070E089E691E20E94FCF98AE00E9413
:1007D00081F740E070E060E088E591E20F94730EED
:1007E00083E495E00E94B17DE0913A1384E0E89FB4
:1007F000F0011124E15CFA4F80913F139091401376
:10080000A0914113B091421380839183A283B3835B
:100810000F94990BB8018FE391E20F948B0B6091C9
:100820003A1389E6689FB00111246D5B7A4F84E327
:1008300091E20F948B0BC0903F13D0904013E09047
:100840004113F09042138EE291E20E94A9F74AE030
:10085000C701B6010E9431758AE00E9481F780913C
:100860003A138F5F80933A1331CF0F94990B8EE137
:1008700091E20E94A9F72ACFC8010E94F7757FCFA5
:100880006F927F928F929F92AF92BF92CF92DF92A0
:10089000EF92FF920F931F93CF93DF93CDB7DEB705
:1008A000C356D1090FB6F894DEBF0FBECDBF5C01B1
:1008B0008B016DB67EB67E0187E5E80EF11CBE01A8
:1008C0006F5F7F4FC5010E9468AC18160CF0A4C082
:1008D0008C858871803109F076C08DB69EB6BE01D8
:1008E0006F5F7F4FC7010E9481760115110509F4E2
:1008F00066C0F8018081882309F461C0019000205E
:10090000E9F73197CF01801B910B20E0F7010190AF
:100910000020E9F73197EE19FF09E80FF91F329629
:100920008DB79EB78E1B9F0B0FB6F8949EBF0FBE60
:100930008DBFEDB7FEB731966F01B801222311F0DC
:1009400069EF73E0C6010F942637B701C6010F9413
:10095000103769EF73E0C6010F94103719A21CA27B
:1009600021E0A701B501CE0181960E94CB808111C3
:100970000AC00F94990BB70188E790E20F948B0B94
:100980008AE00E9481F78BE1FE01B196DE01DC96E0
:1009900001900D928A95E1F7B601CE01CC960E94A6
:1009A0004084CE01CC960E94C9EFCE0181960E9470
:1009B000C9EF0FB6F8949EBE0FBE8DBE80CF21E06A
:1009C00081E090E0A3CFCE0101960E946676882355
:1009D00009F475CFBE016F5F7F4F84EA90E10E94FA
:1009E00081760115110519F0C8010E94F67984EA93
:1009F00090E10E94F67980E20E9481F76D8D7E8DF4
:100A00008F8D98A14AE00E9431758DE00E9481F798
:100A10008AE00E9481F753CF0FB6F8947EBE0FBED6
:100A20006DBECD59DF4F0FB6F894DEBF0FBECDBF00
:100A3000DF91CF911F910F91FF90EF90DF90CF90BA
:100A4000BF90AF909F908F907F906F900895CF93BD
:100A5000C82F0F94990B84E50E9481F78C2F0E9478
:100A60005AAC80E20E9481F786E590E2CF910C9427
:100A7000A9F78F929F92AF92BF92CF92DF92EF929F
:100A8000FF92CF936B017C01B42E20E030E0A901EE
:100A90000F94FD2C87FF07C08DE20E9481F7F7FAC3
:100AA000F094F7F8F094C0E060E070E080E09FE33D
:100AB000CB1541F02DEC3CEC4CEC5DE30F94632D39
:100AC000CF5FF6CFA70196010F94CD336B017C0168
:100AD0000F9440354B015C014AE00E943175CC23F4
:100AE00079F1C501B4010F94022D9B01AC01C7013E
:100AF000B6010F94CC336B017C018EE20E9481F72A
:100B0000C150F0F020E030E040E251E4C701B6010E
:100B10000F94632D6B017C010F9440354B015C01F8
:100B20004AE00E943175C501B4010F94022D9B016A
:100B3000AC01C701B6010F94CC336B017C01E0CF4F
:100B4000CF91FF90EF90DF90CF90BF90AF909F90AC
:100B50008F900895EF92FF920F931F93CF937C0194
:100B60008B01C2E44F3F09F0C4E580E20E9481F7A7
:100B70008C2F0E9481F78AE30E9481F7F701608140
:100B800071818281938142E00E94398582E490E202
:100B90000E94A9F7F801608171818281938142E00E
:100BA0000E94398562E070E080E090E0CF911F9173
:100BB0000F91FF90EF900C9447C81F93CF93DF9352
:100BC00000D000D01F921F92CDB7DEB7182F6091D2
:100BD000FF1070910011072E000C880B990B0F94D9
:100BE000042D6D837E838F8398876091FD107091B3
:100BF000FE10072E000C880B990B0F94042D6983AF
:100C00007A838B839C834AEFBE016B5F7F4FCE015B
:100C100001960E94AA856091941070919510072EFC
:100C2000000C880B990B0F94042D6D837E838F83AA
:100C300098876091921070919310072E000C880B8A
:100C4000990B0F94042D69837A838B839C834FEFD8
:100C5000BE016B5F7F4FCE0101960E94AA85609115
:100C600096101F3F39F085E11802F0011124E7507A
:100C7000FF4E608570E08AE490E20E94FCF960918A
:100C8000961070E085E490E20E94FCF928960FB679
:100C9000F894DEBF0FBECDBFDF91CF911F910895B5
:100CA0002F923F924F925F926F927F928F929F927C
:100CB000AF92BF92CF92DF92EF92FF920F931F936A
:100CC000CF93DF93CDB7DEB763970FB6F894DEBF4F
:100CD0000FBECDBF898B81E0809325021A821B82D3
:100CE0001C821D8219861A861B861C861D862CE393
:100CF0002E873CE13F8746E4488B312C212C50E87D
:100D00005A8B8FEB8B8B198291E09887812C912CD9
:100D100054010091941010919510B801012E000C0F
:100D2000880B990B0F94042D6B017C01232D322D20
:100D30004A895B890F94FD2C882389F08091921059
:100D400090919310A989A111E4C0B1E0B98308176B
:100D500019070CF019823C2C2D2CEA8AFB8A0E9480
:100D60007AC86B017C01DC01CB0129853A854B8572
:100D70005C85821B930BA40BB50BB7FD2FC0D7016D
:100D8000C60188519C4FAF4FBF4F89879A87AB8769
:100D9000BC8780E00E94DD8582E590E20E94A9F791
:100DA00081149104A104B10409F4DFC0C501B401A8
:100DB00068577C4E8F4F9F4F6C197D098E099F0994
:100DC00028EE33E040E050E00F944133CA01B9010E
:100DD0004AE00E9488F78AE00E9481F780E00F9441
:100DE000440F0E947AC86093881070938910809392
:100DF0008A1090938B106091921070919310072E2F
:100E0000000C880B990B0F94042D6E837F838C014B
:100E10009B01AC01632D722D8A899B890F94CC3381
:100E20002B013C0120E030E0A9010F942D3687FF13
:100E300004C077FA709477F8709481149104A10437
:100E4000B10409F096C020E030E040E85FE3C30160
:100E5000B2010F94FD2C87FF10C09885812C912C36
:100E60005401992331F082E8882E86E0982EA12C37
:100E7000B12C8C0C9D1CAE1CBF1CA981AA2391F126
:100E80002A813B814C815D81211531054105510548
:100E900041F0D701C601821B930BA40BB50BB7FD24
:100EA00021C02E813F81A8016D857E858F8598891F
:100EB0000F94CC3320E030E040E85FE30F94FD2C4A
:100EC00087FD2AC0D701C601805A9541AF4FBF4F59
:100ED0008A839B83AC83BD839E819D87AF81AE87D0
:100EE0000F87188B809125028823B1F0811491041B
:100EF000A104B10461F0B8E8CB1AB3E1DB0AE10860
:100F0000F108C818D908EA08FB08F7FE05C01886DA
:100F100000CF081719071CF52091250229832223E9
:100F200021F0109225020E949CAF898163960FB632
:100F3000F894DEBF0FBECDBFDF91CF911F910F910F
:100F4000FF90EF90DF90CF90BF90AF909F908F90E9
:100F50007F906F905F904F903F902F9008953C2C22
:100F60002D2CEA8AFB8A1982FACE8FE30E9481F740
:100F700032CF20E030E040E450E4C301B2010F94EE
:100F80002D3618160CF079CF4601570176CF2F92E7
:100F90003F924F925F926F927F928F929F92AF9209
:100FA000BF92CF92DF92EF92FF920F931F93CF9356
:100FB000DF93CDB7DEB765970FB6F894DEBF0FBEEF
:100FC000CDBF8A8B6B8B20913E05298B10923E05FD
:100FD00081E0809325021A821B821C821D82198661
:100FE0001A861B861C861D863CE33E874CE14F8794
:100FF00056E4588B312C212C80E88C8B9FEB9D8BF9
:101000001982A1E0A887812C912C54010091FF1036
:1010100010910011B801012E000C880B990B0F9450
:10102000042D6B017C01232D322D4C895D890F9499
:10103000FD2C882389F08091FD109091FE10BB89D2
:10104000B111E4C021E02983081719070CF01982B7
:101050003C2C2D2CEC8AFD8A0E947AC86B017C0105
:10106000DC01CB0129853A854B855C85821B930B7E
:10107000A40BB50BB7FD2FC0D701C60188519C4FFB
:10108000AF4FBF4F89879A87AB87BC878A890E94F9
:10109000DD858EE490E20E94A9F781149104A104F9
:1010A000B10409F4E2C0C501B4016053784F8F4F19
:1010B0009F4F6C197D098E099F0928EE33E040E0AF
:1010C00050E00F944133CA01B9014AE00E9488F709
:1010D0008AE00E9481F780E00F94440F0E947AC852
:1010E000609388107093891080938A1090938B106E
:1010F0006091FD107091FE10072E000C880B990B6B
:101100000F94042D6E837F838C019B01AC01632DB2
:10111000722D8C899D890F94CC332B013C0120E0EA
:1011200030E0A9010F942D3687FF04C077FA709440
:1011300077F8709481149104A104B10409F099C066
:1011400020E030E040E85FE3C301B2010F94FD2CE2
:1011500087FF10C09885812C912C5401992331F080
:101160008AE9882E82E0982EA12CB12C8C0C9D1C33
:10117000AE1CBF1CA981AA2391F12A813B814C811D
:101180005D81211531054105510541F0D701C601A9
:10119000821B930BA40BB50BB7FD21C02E813F81A1
:1011A000A8016D857E858F8598890F94CC3320E0CA
:1011B00030E040EC5FE30F94FD2C87FD2AC0D7019F
:1011C000C601805A9541AF4FBF4F8A839B83AC8342
:1011D000BD839E819D87AF81AE870F87188B8091DD
:1011E00025028823B1F081149104A104B10461F0B7
:1011F000B0EDCB1AB7E0DB0AE108F108C818D9084E
:10120000EA08FB08F7FE05C0188600CF0817190783
:1012100034F5309125023983332321F010922502D1
:101220000E949CAF298920933E05898165960FB65F
:10123000F894DEBF0FBECDBFDF91CF911F910F910C
:10124000FF90EF90DF90CF90BF90AF909F908F90E6
:101250007F906F905F904F903F902F9008953C2C1F
:101260002D2CEC8AFD8A1982F7CE8FE30E9481F73C
:101270002FCF20E030E040E450E4C301B2010F94EE
:101280002D3618160CF076CF4601570173CF0F9309
:101290000FB70F9300916E000B7F00936E00789450
:1012A0000F930BB70F930CB70F921F922F933F938F
:1012B0004F935F936F937F938F939F93AF93BF935E
:1012C000EF93FF9311240E94288AFF91EF91BF9121
:1012D000AF919F918F917F916F915F914F913F91CE
:1012E0002F911F900F900CBF0F910BBF0F910460B7
:1012F000F89400936E000F910FBF0F9118952091F5
:1013000094103091951021153105E9F080919210DB
:1013100090919310029624503109821793079CF400
:1013200090937F0680937E060E947AC8605E704428
:101330008D4F9F4F60938006709381068093820645
:101340009093830608951092800610928106109261
:101350008206109283060895CF93DF9310923E0584
:10136000C9EFD0E11F821E820E9486C818862C9881
:10137000CEE8D0E11F821E820E947F89188680916C
:101380000201807280930001DF91CF910895EF9266
:10139000FF920F931F93CF93DF93C82F7B018A0196
:1013A00080910B068130A1F40F94950BC7010E9428
:1013B000A9F78AE19FE10E94A9F7C7FD33C08C2FEE
:1013C0000C2E000C990B0E9461AC8AE00E9481F700
:1013D0000E94AC89A89580915406811132C081E0A9
:1013E0008093540680E880930B060E94AC89D5E177
:1013F000D150409AE1F069E170E080E090E00E9415
:1014000047C8A895409868E270E080E090E00E94AC
:1014100047C8A89568E270E080E090E00E9447C865
:10142000A895E6CF86E19FE10E94A9F7CECF6FE0B5
:101430007FE1CF3F11F063E17FE140E0C8010F940D
:10144000730EDF91CF911F910F91FF90EF90089550
:101450000F931F93CF93DF9380911A028F3708F475
:1014600042C08F5790910111909388069923C9F13A
:101470002C9A2091961020938706909102012111B9
:1014800090959072909300018F5F80931A028091E3
:10149000860691E089278093860680911902C1E033
:1014A000C80F85300CF0C0E0823009F4D8C03CF59C
:1014B0008823D9F1813009F4C6C0C09319020E9473
:1014C0007C328091260890912708009729F0019797
:1014D0009093270880932608DF91CF911F910F9159
:1014E00008952C98C6CF90918806891708F02C98FB
:1014F00090918706891740F290910201C2CF843003
:1015000009F4C5C00CF4BEC08530B9F690918506CB
:10151000911102C080938506809185068150809349
:101520008506882351F2C5E0C8CF809118028F5FED
:1015300080311CF480931802C0CF10921802809161
:101540008406811113C08091F9109091FA10909344
:10155000FC108093FB1080918E1090918F109093CF
:1015600091108093901081E0809384061092FA107D
:101570001092F91010928F1010928E100091FB10A3
:101580001091FC108091FF1090910011D1E018167D
:1015900019062CF080910111811101C0D0E08091D9
:1015A0001F0290912002081719073CF444E050E212
:1015B00061E170E280E00E94C789DD2371F08091D3
:1015C0001D0290911E02801791073CF443E250E205
:1015D00060E370E280E00E94C7898091941090914E
:1015E0009510D1E0181619062CF0809196108111F3
:1015F00001C0D0E0209190103091911080918A0626
:1016000090918B06281739073CF444E050E261E1E1
:1016100070E28FEF0E94C789DD2309F44ECF20913D
:1016200090103091911080911B0290911C028217B2
:1016300093070CF042CF43E250E260E370E28FEF99
:101640000E94C7893ACF88E080937B0085E480932D
:101650007C0080917A00806480937A002ECF809104
:101660007A0086FD27C02091780030917900809122
:10167000F9109091FA10820F931F9093FA108093B3
:10168000F9101BCF88E080937B0086E4E0CF809147
:101690007A0086FD11C02091780030917900809108
:1016A0008E1090918F10820F931F90938F108093C4
:1016B0008E1003CFC2E001CFC4E0FFCE2F923F9245
:1016C0004F925F926F927F928F929F92AF92BF9252
:1016D000CF92DF92EF92FF920F931F93CF93DF93FE
:1016E00000D0CDB7DEB79B838A836B015A01298373
:1016F0001801870181E090E02F3F11F090E080E039
:1017000025E0289FF001299FF00D1124EC5CFA4F91
:101710008481882309F48FC0EA81FB8114821582B9
:10172000168217821086EA81FB8184818230B9F0AB
:10173000833009F400C1813009F067C0258136810A
:1017400047815085F60160817181828193810F9478
:10175000FD2C87FD5AC082E0EA81FB818483EA8107
:10176000FB8185809680A780B084F601C080D180FF
:10177000E280F380B801110F880B990B0F94042DB0
:101780002B013C01809117028823F9F0F981F111B6
:101790001CC0809123088823A9F020E030E040E8B5
:1017A0005EE3C301B2010F94632D9B01AC01C5013F
:1017B000B4010F94CC33A70196010F94FD2C181699
:1017C0000CF464C080E880931502A3019201C50166
:1017D000B4010F94CC33A70196010F94FD2C181679
:1017E0000CF499C00E947AC86B017C019101A8EEAB
:1017F000B3E00F949533C60ED71EE81EF91EEA819A
:10180000FB81C082D182E282F3820F900F900F9011
:10181000DF91CF911F910F91FF90EF90DF90CF90CC
:10182000BF90AF909F908F907F906F905F904F9000
:101830003F902F900895F501408051806280738021
:10184000A3019201EA81FB81658176818781908580
:101850000F94FD2C882309F466CFEA81FB81458231
:10186000568267827086FF24F39420E030E0A9015D
:10187000F50160817181828193810F942D36181654
:101880000CF0F12CEA81FB81F4824DCF23E830EC9F
:101890004AEA5EE3C301B2010F94632D9B01AC01E0
:1018A000C501B4010F94CC33A70196010F94FD2C10
:1018B000181614F080E687CF20E030E040E05FE3C8
:1018C000C301B2010F94632D9B01AC01C501B401AA
:1018D0000F94CC33A70196010F94FD2C181614F029
:1018E00080E471CF2DEC3CEC4CE45FE3C301B2012A
:1018F0000F94632D9B01AC01C501B4010F94CC334F
:10190000A70196010F94FD2C181614F080E25BCF0E
:10191000109215025ACF0E947AC8EA81FB81008199
:10192000118122813381601B710B820B930B97FD18
:101930006CCF83E0848344EE5FE164EF7FE18981D3
:101940000F900F900F90DF91CF911F910F91FF900B
:10195000EF90DF90CF90BF90AF909F908F907F904F
:101960006F905F904F903F902F900C94C7898F920B
:101970009F92AF92BF92CF92DF92EF92FF920F931E
:101980001F93CF93DF93EC018A01072E000C880B85
:10199000990B0F94042D4B015C01C880D980EA801B
:1019A000FB80A70196010F942D3618162CF488821F
:1019B0009982AA82BB8210C0B801110F880B990BC3
:1019C0000F94042D4B015C01AC019B01C701B601D2
:1019D0000F942D3618165CF3DF91CF911F910F9164
:1019E000FF90EF90DF90CF90BF90AF909F908F903F
:1019F00008952F923F924F925F926F927F928F92B3
:101A00009F92AF92BF92CF92DF92EF92FF920F938D
:101A10001F93CF93DF93CDB7DEB763970FB6F894DC
:101A2000DEBF0FBECDBF809133058111F3C0809121
:101A300032058111DEC080918406811119C0639640
:101A40000FB6F894DEBF0FBECDBFDF91CF911F91CF
:101A50000F91FF90EF90DF90CF90BF90AF909F904D
:101A60008F907F906F905F904F903F902F90089550
:101A70000E94A0710E947AC84B015C010091FD1088
:101A80001091FE10809123029091240280179107FB
:101A90000CF404C280913805882309F4E4C16091F4
:101AA000FF1070910011072E000C880B990B0F94FA
:101AB000042D6D837E838F839887B801110F880B67
:101AC000990B0F94042D69837A838B839C834AE05E
:101AD000E42EF12C0CE310E020E0AE014B5F5F4FF1
:101AE000BE016F5F7F4F8CE291E10E945E8B00919F
:101AF000FD101091FE10809121029091220280171A
:101B000091070CF48EC0F12CF09201118091F51028
:101B10009091F610A091F710B091F8100097A105E0
:101B2000B10539F1A5019401281B390B4A0B5B0B58
:101B3000DA01C901B7FD1DC08091F3109091F41036
:101B4000081719070CF437C38091FF10909100110A
:101B5000009739F00E5F1F4F0497081719070CF410
:101B600040C31092F5101092F6101092F7101092D8
:101B7000F8100091921010919310073911050CF094
:101B8000F0C18091800690918106A0918206B0916B
:101B900083060097A105B10509F48CC1A501940144
:101BA000281B390B4A0B5B0BDA01C901B7FD82C157
:101BB00080917E0690917F06081719070CF4EBC2FE
:101BC00060919410709195106115710549F0C801EC
:101BD00002969B0124503109821793070CF414C319
:101BE000109280061092810610928206109283064F
:101BF00065C1109232050E94F3290E94B2238EEF34
:101C00000E94E2300E946E3180918406882309F49C
